:020000040800F2
:100000000000022035F90008B19C0008B39C0008EC
:10001000B59C0008B79C0008B99C000800000000CF
:10002000000000000000000000000000BB9C000871
:10003000BD9C000800000000BF9C0008C19C000897
:1000400079F9000879F9000879F9000879F90008C8
:1000500079F9000879F9000879F9000879F90008B8
:1000600079F9000879F9000879F9000805660008AF
:1000700079F9000879F9000879F9000879F9000898
:1000800079F9000879F9000879F9000879F9000888
:1000900079F9000879F9000879F90008359F000816
:1000A00079F9000879F9000879F9000879F9000868
:1000B000B99E000879F9000879F9000879F9000873
:1000C00079F9000879F9000879F9000879F9000848
:1000D00079F9000879F9000849A0000879F90008C1
:1000E00079F9000879F90008C59C000879F9000839
:1000F00079F9000879F9000879F9000879F9000818
:1001000079F9000879F9000879F9000879F9000807
:1001100079F9000879F9000879F9000879F90008F7
:1001200079F9000879F9000879F9000879F90008E7
:1001300079F9000879F9000879F9000879F90008D7
:1001400079F9000879F9000879F90008F59C0008A8
:1001500079F9000879F9000879F9000879F90008B7
:1001600079F9000879F9000879F9000879F90008A7
:1001700079F9000879F9000879F9000879F9000897
:0801800079F9000879F9000883
:10018800BCA4050800000020A40B0020A80B002038
:10019800704F0020064B07481A68074B1A60074B38
:1001A80000221A70064B01221A7001F018BD00BF18
:1001B800503C00206C0E002054420020383C0020A7
:1001C800F03B002008B5034801F009FD024B00226E
:1001D8001A7008BDFC100020F03B002008B5054B44
:1001E800012200201A7004F03FFD0348BDE80840D2
:1001F80001F0F5BC68420020A01100202DE9F04173
:10020800144C204603F075F800201349134A02F0F5
:1002180027FE1349134A0746002002F021FE12491F
:10022800124A0646002002F01BFED22105463A4635
:1002380023460A2002F02CFFD22132462346FA2018
:1002480002F026FF5A20D2212A462346BDE8F04173
:1002580002F01EBFB40F002032940508CD0100083B
:100268003B940508E5010008439405089D01000832
:1002780008B5054B012200201A7004F0F5FC03486C
:10028800BDE8084001F0ABBC68420020A011002086
:10029800044B054800221A70044B02221A7001F020
:1002A8009EBC00BF383C0020B40F0020F03B00206B
:1002B80008B5034801F093FC024B00221A7008BDF0
:1002C800FC100020F03B00202DE9F041144C2046A2
:1002D80003F00FF800201349134A02F0C1FD134937
:1002E800134A0746002002F0BBFD1249124A06468F
:1002F800002002F0B5FDD22105463A4623460A20E1
:1003080002F0C6FED221324623465A2002F0C0FE31
:10031800AA20D2212A462346BDE8F04102F0B8BE01
:100328006C0E002032940508B90200084C940508A8
:10033800990200085594050879020008002008B5BC
:1003480004F092FC064B00221A70064B1B78022B15
:100358000CBF05480548BDE8084001F040BC00BF97
:1003680068420020F03B0020B40F00206C0E0020F3
:1003780010B5084C204602F0BCFF00200649074A89
:1003880002F06EFDD22102462346E620BDE8104069
:1003980002F07EBEE81200205E94050845030008BE
:1003A80010B5074C4FF6E071206802F0ADF82068F0
:1003B800044902F057F8BDE8104003F0D3B900BF74
:1003C800A80B00206794050810B5074C4FF6E0719C
:1003D800206802F099F82068044902F043F8BDE863
:1003E800104003F0BFB900BFA80B00207C9405089B
:1003F80010B5074C4FF6E071206802F085F82068C8
:10040800044902F02FF8BDE8104003F0ABB900BF73
:10041800A80B0020919405082DE9F04F774C85B082
:10042800FFF7BEFF002004F01FFC23790BB9FFF78C
:10043800DFFF6379714D53B928684FF6E07102F018
:1004480063F828686E4902F00DF803F08BF9A37978
:100458000BB9FFF7B9FF694B5A79002A00F0C2803F
:100468001A79002A00F0BE80997900221A715A710F
:1004780001B19A71634BDFF8BCA1DFF8BC811A7037
:10048800614EDAF80010614CDFF8B0B1DFF8B091D6
:100498005F4F604D4FF4967006F025F9D8F80010BC
:1004A8004FF4987006F01FF931684FF49A7006F00F
:1004B8001AF921684FF49C7006F015F9564A4FF462
:1004C8009E701168019206F00EF9DBF800104FF4E7
:1004D800A07006F008F9D9F800104FF4A27006F0E1
:1004E80002F939684FF4A47006F0FDF829684FF452
:1004F800A67006F0F8F8494B4FF4A87019680293F3
:1005080006F0F1F8DFF83CC14FF4AA70DCF80010EF
:10051800CDF80CC006F0E7F8DFF808E14FF4AC704E
:10052800DEF8001006F0DFF8019AD4ED001A92ED1B
:10053800002A9AED000AD8ED000A96ED001A07F095
:10054800FDFD029B9BED000A93ED002AD9ED000A00
:1005580097ED001AD5ED001A07F0FEFD9BED007A25
:10056800DAED007A2E49DDF80CC0029B019A77EE8D
:10057800677A99ED007AC1ED0A7AD8ED007A77EEBC
:10058800677A97ED007AC1ED0B7AD6ED007A77EEAF
:10059800677A95ED007AC1ED0C7AD4ED007A77EEA2
:1005A800677A93ED007AC1ED0D7ADCF80030134CD0
:1005B800CB63D2ED007A1B4A2068136877EE677A1E
:1005C8000B64C1ED0E7A4FF6E07101F09DFF2068D3
:1005D800154901F047FF07F00CFE03F0C3F8134874
:1005E80003F004F9FFF7DCFE002007F0C3FD104814
:1005F80005B0BDE8F04F01F0F2BA00BFA80B00202B
:10060800A6940508F03B0020600E0020480E00204C
:100618005C0E00202C0E0020580E0020300E00200A
:10062800B0450020380E0020BB940508809698003D
:10063800FC100020440E00204C0E0020540E002018
:10064800640E0020680E002008B5002007F092FD17
:100658000248BDE8084001F0C2BA00BFFC10002003
:100668002DE9F04F494D4A4E85B000244FF6FF78EA
:10067800284602F03EFE414622462346454800945D
:10068800019401F005FF0427B060224623464FF687
:10069800E07141480097019401F0FAFE234630606A
:1006A800414622463D480097019401F0F1FE3C493D
:1006B800F0603C4A204602F0D3FB3B493B4A0746E0
:1006C800204602F0CDFB3A493A4A8046204602F0DD
:1006D800C7FB3949394A8146204602F0C1FB3849EF
:1006E800384A8246204602F0BBFB3749374A8346E0
:1006F800204602F0B5FB36490390364A204602F000
:10070800AFFB21468446B268CDF808C02B46204688
:1007180002F0BEFC214632682B467D2002F0B8FC70
:100728002321F2682B46B42002F0B2FC37213A4666
:100738002B46FA2002F0ACFC692142462B46FA20EF
:1007480002F0A6FC9B214A462B46FA2002F0A0FCA8
:10075800C82152462B46322002F09AFC5A462B46B4
:10076800C8216E2002F094FCDDF808C0C82162465A
:100778002B46AA2002F08CFC039AF020C8212B46B5
:1007880005B0BDE8F04F02F083BC00BF5810002050
:10079800A80B0020CF940508A6940508D79405084F
:1007A800DF940508B9090008E794050865090008F9
:1007B800EF94050875120008F79405089D0F0008C6
:1007C800FE940508610F0008059505085106000804
:1007D8000C9505082104000818B9044B93ED000A8C
:1007E8007047034B93ED000A704700BF440E00208A
:1007F800540E002018B9044B93ED000A7047034BC0
:1008080093ED000A704700BF4C0E0020640E0020D4
:1008180018B9044B93ED000A7047034B93ED000A97
:10082800704700BF600E00205C0E002018B9044B12
:1008380093ED000A7047034B93ED000A704700BF21
:10084800480E00202C0E002018B9044B93ED000A26
:100858007047034B93ED000A704700BF580E002005
:10086800300E002070B52DED028B9FED108A0446E6
:100878000E460A25F0EE488A07F01EF978EE808ABF
:1008880007F020F90A4838EE008A02F0AFFF013D70
:10089800F2D1F2EE047AC8EEA78A88EE278AC4ED70
:1008A800008A86ED008ABDEC028B70BD0000000056
:1008B800A086010010B50E4C0E4802F097FF04F117
:1008C800140104F11000FFF7CDFF4FF6E07004F0BB
:1008D8009FF9FFF779FD5E220023DF206E2104F0E7
:1008E800A7FA01232371044B1A68044B1A6010BD40
:1008F800A80B0020A0860100503C00205442002094
:1009080010B5002007F052FC0F4B104C186010482F
:1009180002F06CFF04F11C0104F11800FFF7A2FFBC
:100928004FF6E07004F074F9FFF762FD5E220023D1
:10093800DF203C2104F07CFA01236371054B1A681F
:10094800054B1A6010BD00BF380E0020A80B002010
:10095800A0860100503C002054420020104908B5F0
:1009680001F120002431FFF77DFF4FF6E07004F01D
:100978004FF9FFF729FDB7206E215E22002304F00E
:1009880057FA084B1A68084B1A60084B02224FF0B6
:10099800804001211A70BDE808400DF0FEB900BF83
:1009A800A80B0020403C002054420020E00C00200E
:1009B80008B5002007F0EEFB114B1860114802F053
:1009C80015FF114901F128002C31FFF74BFF4FF6B5
:1009D800E07004F01DF9FFF70BFDB7203C215E2203
:1009E800002304F025FA094B1A68094B1A60094BD1
:1009F80001214FF080401970BDE808400DF0CDB9D5
:100A0800680E0020A0860100A80B0020403C0020B2
:100A180054420020E00C00202DE9F84380462DEDDB
:100A2800068B10EE100A11EE905A11EE109A10EE85
:100A3800904A0EF003F9064648460F460EF0FEF8B7
:100A480041EC100B41EC180B10F0C2F8304653EC97
:100A5800102B39460EF046F90EF026FCB0EE480A87
:100A6800F0EE680A454B186009EE900A10F0B0F9EC
:100A7800304653EC102B39460EF034F90EF014FCC6
:100A88003F4B09EE100A186020460EF0D7F80646CC
:100A980028460F460EF0D2F841EC100B41EC1A0B29
:100AA80010F096F8304653EC102B39460EF01AF930
:100AB8000EF0FAFBB0EE4A0AF0EE6A0A314B186003
:100AC80008EE100A10F084F9304653EC102B394622
:100AD8000EF008F90EF0E8FB08EE900A79EE688A45
:100AE80039EEC88A9FED287A68EEA87A48EE087A27
:100AF80028EE078A9FED257A68EE878A88EE278A8E
:100B0800234B1860C8EEA78A68EE897A17EE900A18
:100B18000EF094F800221F4B0DF032FF68EE297A90
:100B2800044617EE900A0D460EF088F802460B466A
:100B3800204629460DF022FF68EEA99A0EF0B4FB74
:100B480058EE499AB8F1000F09D1134B83ED008A8A
:100B5800124BC3ED008A124B1860124B08E0124B7F
:100B680083ED008A114BC3ED008A114B1860114BBD
:100B7800C3ED009ABDEC068BBDE8F883500E00204B
:100B88003C0E0020340E002000004842000048C2FD
:100B9800400E002000004940440E00204C0E00206A
:100BA800600E0020480E0020540E0020640E002025
:100BB8005C0E00202C0E00202DE9F84380462DED18
:100BC800068B10EE100A11EE109A11EE905A10EEE4
:100BD800904A0EF033F8064648460F460EF02EF8B7
:100BE80041EC100B41EC190B0FF0F2FF304653ECBF
:100BF800102B39460EF076F80EF056FBB0EE490A87
:100C0800F0EE690A624B186008EE100A10F0E0F87E
:100C1800304653EC102B39460EF064F80EF044FBC6
:100C28005C4B08EE900A186020460EF007F806465E
:100C380028460F460EF002F841EC100B41EC1A0B57
:100C48000FF0C6FF304653EC102B39460EF04AF829
:100C58000EF02AFBB0EE4A0AF0EE6A0A4E4B186014
:100C680009EE900A10F0B4F8304653EC102B3946D0
:100C78000EF038F80EF018FB09EE100A78EEC98A63
:100C8800464B38EE698A28EEA8AA186008EE08AA2A
:100C9800B8F1000F0CD1424B18680DF0CFFF38A304
:100CA800D3E900230EF01EF83E4B04460D460BE038
:100CB8003D4B18680DF0C2FF31A3D3E900230EF0B5
:100CC80011F83A4B04460D4618680DF0B7FF024676
:100CD8000B46204629460EF005F80EF0E5FA2AA341
:100CE800D3E900230AEE900A294620460DF0FAFFC0
:100CF8000EF0DAFA9FED2E7A6AEE87AAF7EE007AFE
:100D08004AEEAA7A6AEE87AA67EE876ACAEEA77AD7
:100D180006EE100A77EEC67A67EEA87A46EE887A6B
:100D280087EE8AAA5AEE086AB1EE4A7AC6EEA88A0F
:100D380068EE897A47EE297A68EEA99A57EE099AF9
:100D4800B8F1000F0AD11B4B83ED00AA1A4BC3ED73
:100D5800008A1A4BC3ED007A194B09E0194B83ED51
:100D680000AA194BC3ED008A184BC3ED007A184B43
:100D7800C3ED009ABDEC068BBDE8F883AFF30080A5
:100D88001F85EB51B81E1940000000E08E79353EF2
:100D9800500E00203C0E0020340E0020400E002093
:100DA800680E0020580E0020380E0020300E00205B
:100DB80000004842440E00204C0E0020600E002027
:100DC800480E0020540E0020640E00205C0E002007
:100DD8002C0E00202DE9F74F044610EE10AA10EE55
:100DE800907A11EE105A11EE906A12EE108A894626
:100DF80000284DD14FF6E07003F00AFF50460DF081
:100E08001DFF824638468B460DF018FF5246CDE945
:100E180000015B464A494B4812F010FC494A2346F8
:100E28000520372104F022F828460DF007FF8246F6
:100E380030468B460DF002FF5246CDE900015B4675
:100E48004149404812F0FAFB3E4A234605206921F1
:100E580004F00CF840460DF0F1FE37A3D3E9002367
:100E68000DF040FF02460B463648384912F0E6FBC3
:100E7800234605209B21334A03F0F8FF34493148C3
:100E88004A4612F0DBFB82209B212E4A23464CE087
:100E98004FF4FC6003F0BCFE50460DF0CFFE8246D6
:100EA80038468B460DF0CAFE5246CDE900015B4636
:100EB8002349244812F0C2FB224A0023052050216E
:100EC80003F0D4FF28460DF0B9FE044630460D461F
:100ED8000DF0B4FE2246CDE900012B461A49194807
:100EE80012F0ACFB174A00230520822103F0BEFF55
:100EF80040460DF0A3FE10A3D3E900230DF0F2FE47
:100F080002460B460F48114912F098FB00230520B2
:100F1800B4210C4A03F0AAFF0E490A484A4612F0C7
:100F28008DFB084A8220B421002303B0BDE8F04FAE
:100F380003F09CBFAFF30080000000A2941A6D423A
:100F480013950508D80B0020249505083595050844
:100F5800429505084B9505080C4A0D4B116C92ED0E
:100F6800092A92ED050AD2ED060A92ED071AD2ED8A
:100F7800081A012083ED132A83ED140AC3ED150A1C
:100F880083ED161AC3ED171A196623E7B04500203A
:100F9800A80B00200C4A0D4BD16B92ED042A92ED60
:100FA800000AD2ED010A92ED021AD2ED031A0020CE
:100FB80083ED132A83ED140AC3ED150A83ED161A7F
:100FC800C3ED171A196605E7B0450020A80B0020E5
:100FD800F0B52DED088B044683B06B4B002851D13A
:100FE80093ED0B1AD3ED091A93ED0A0AD3ED080A0B
:100FF800FFF712FD654BD3ED009A654B93ED008A20
:10100800644BD3ED008A644B684601A993ED00AAAE
:10101800FFF728FC00980DF011FE064601980F46D0
:101028000DF00CFE41EC100B41EC1B0B0FF0D0FD4A
:10103800304653EC102B39460DF054FE0EF034F9BF
:10104800B0EE4B0AF0EE6B0A09EE100A0FF0C0FE84
:10105800304653EC102B39460DF044FE0EF024F9BF
:1010680007EE100A68EE077A28EE098A59EE897A9F
:1010780009EE878A204677EEA88A38EE0A8A07F0B2
:1010880089F851E093ED071AD3ED051A93ED060A96
:10109800D3ED040A0120FFF7BFFC404BD3ED009AC3
:1010A8003F4B93ED008A3F4BD3ED008A3E4B684699
:1010B80001A993ED00AAFFF7D5FB00980DF0BEFD3E
:1010C800044601980D460DF0B9FD41EC100B41ECBA
:1010D8001B0B0FF07DFD204653EC102B29460DF01D
:1010E80001FE0EF0E1F8B0EE4B0AF0EE6B0A09EEE5
:1010F800100A0FF06DFE204653EC102B29460DF018
:10110800F1FD0EF0D1F807EE100A68EE077A28EE26
:10111800098A59EE897A09EE878A002077EEA88A2B
:1011280038EE0A8A07F042F8F1EE487A28EE088A83
:1011380008EEA88A064687EE888A18EE100A0DF08F
:101148007DFD07EE106AF8EEC77A044617EE900A9E
:101158000D460DF073FD0AA3D3E900230DF0C2FD7F
:1011680002460B46204629460DF0E6FE0EF09CF896
:1011780000EE100A03B0BDEC088BF0BDAFF30080A1
:101188001F85EB51B81E1940A80B0020440E002003
:101198004C0E0020600E0020480E0020540E002047
:1011A800640E00205C0E00202C0E002038B50120B3
:1011B800FFF70EFF1E4C4FF6E07084ED000A03F0B7
:1011C80027FD5E22DF20A021002303F031FE194B0A
:1011D80001259D71184B93ED000A184BD3ED000AB9
:1011E800174B93ED001A174BD3ED001A164B93EDDE
:1011F800002A164B00201968FFF7ECFD144B93EDFD
:10120800000A144BD3ED000A134B93ED001A134B4D
:10121800D3ED001A124B2846196894ED002AFFF7FF
:10122800D9FDFFF7BDF80F4B1A680F4B1A6038BD90
:10123800300E0020A80B0020440E00204C0E002089
:10124800600E0020480E0020580E0020680E002076
:10125800540E0020640E00205C0E00202C0E00208E
:10126800380E0020503C00205442002008B50020D1
:10127800FFF7AEFE0D4B4FF6E07083ED000A03F06A
:10128800C7FCB720A0215E22002303F0D1FD084B44
:101298001A68084B1A60084B03224FF0804001215E
:1012A8001A70BDE808400CF078BD00BF580E002049
:1012B800403C002054420020E00C0020AFF30080A6
:1012C800284B2948062210B51A704FF6E07400F032
:1012D80086FC0020214607F065FA3120214607F0F8
:1012E80061FA6320214607F05DFA9520214607F050
:1012F80059FAC7204FF4FC6107F054FA4EF29C707B
:1013080003F086FC052001210023184A03F0AEFDF6
:10131800052020210023164A03F0A8FD05205221AC
:101328000023144A03F0A2FD842100230520124A59
:1013380003F09CFD4FF4F06003F06AFCB6210F4AFD
:101348000023052003F092FD4FF6FF7003F060FCC8
:101358008720DC210A4A002303F088FDBDE81040FD
:1013680008F076BC68420020301400205495050827
:101378008B9505088395050858950508A59A0508CD
:101388005A95050838B5384B3848394D07221A7030
:101398004FF6E07400F023FC0020214607F002FA23
:1013A8003120214607F0FEF96320214607F0FAF9BB
:1013B8009520214607F0F6F92146C72007F0F2F9F3
:1013C8004EF29C7003F024FC052001210023294AD9
:1013D80003F04CFD052020210023274A03F046FD99
:1013E800052052210023254A03F040FD05208421D1
:1013F8000023234A03F03AFD2A460520B62100239C
:1014080003F034FD40F213144FF4F06003F000FCD5
:101418002046012100231B4A03F028FD20462021F5
:101428000023194A03F022FD204652212A460023B0
:1014380003F01CFD204684210023144A03F016FD06
:10144800B62100232046124A03F010FD4FF6FF7024
:1014580003F0DEFB7D20DC210E4A002303F006FDAD
:10146800BDE8384008F0F4BB684200203014002082
:101478008E9905085F950508639505086795050821
:101488006A950508739505086F9505086E95050812
:10149800729505087795050838B52B4B2B48052418
:1014A8001C704FF6E07500F09AFB0020294607F003
:1014B80079F92720294607F075F94F20294607F0C2
:1014C80071F97720294607F06DF99F20294607F022
:1014D80069F92946C72007F065F94EF29C7003F0B8
:1014E80097FB204601210023194A03F0BFFC204640
:1014F80016210023174A03F0B9FC20463E21002399
:10150800154A03F0B3FC204666210023134A03F072
:10151800ADFC20468E210023114A03F0A7FC20468B
:10152800B621104A002303F0A1FC4FF6FF7003F028
:101538006FFB7D20DC210C4A002303F097FCBDE8FB
:10154800384008F085BB00BF6842002030140020F6
:101558008E99050882950508869505088A950508D7
:101568008E9505089295050896950508394B3A48D1
:10157800042270B51A704FF6E07400F030FB0020BA
:10158800214607F00FF93120214607F00BF96320B7
:10159800214607F007F99520214607F003F92F4E59
:1015A8002F4D2146C72007F0FDF84EF29C7003F03E
:1015B8002FFB052001213246002303F057FC0520AC
:1015C80020210023274A03F051FC05205221002343
:1015D800254A03F04BFC052084210023234A03F00D
:1015E80045FC2A460520B621002303F03FFC40F2C3
:1015F80013144FF4F06003F00BFB20460121324630
:10160800002303F033FC204620210023184A03F06E
:101618002DFC204652212A46002303F027FC2046B1
:1016280084210023134A03F021FCB621002320461D
:10163800114A03F01BFC4FF6FF7003F0E9FA7D2016
:10164800DC210E4A002303F011FCBDE8704008F0CD
:10165800FFBA00BF6842002030140020B795050883
:101668008E990508A2950508B2950508A79505085D
:10167800AC950508B1950508B6950508BA9505080D
:10168800F8B5304B3048314F314E03221A704FF6BF
:10169800E07400F0A4FA0020214607F083F86320E4
:1016A800214607F07FF8B3204FF4F06107F07AF88D
:1016B8002146C72007F076F84FF6FF7003F0A8FA26
:1016C8004EF29C75DC2100237D20224A03F0CEFBDC
:1016D800284603F09DFA052001213A46002303F02D
:1016E800C5FB0520522100231B4A03F0BFFBB6218E
:1016F80032460023052003F0B9FB40F213144FF4DF
:10170800F06003F085FA204601213A46002303F0F1
:10171800ADFB204652213246002303F0A7FBB62139
:10172800002320460D4A03F0A1FB284603F070FA77
:101738000520A2210A4A002303F098FBBDE8F840DF
:1017480008F086BA6842002030140020D4950508B5
:101758008E990508C5950508CF950508D395050800
:101768009395050808B5064B064802221A7000F042
:1017780036FA06F00FFFBDE8084008F069BA00BF66
:101788006842002030140020002008B503F06CFAED
:10179800064B00221A70064B1B78022B0CBF05481B
:1017A8000548BDE8084000F01ABA00BF68420020AA
:1017B800F03B0020B40F00206C0E00202DE9F14F03
:1017C8002D4C204601F095FD00202C492C4A01F0B3
:1017D80047FB2C492C4A8146002001F041FB2B494C
:1017E8002B4A0746002001F03BFB2A492A4A0646B5
:1017F800002001F035FB2949294A0546002001F05F
:101808002FFB2849284A8046002001F029FB274958
:10181800274A8246002001F023FBD22183464A460C
:101828002346E62001F034FC28203A4623460146A8
:1018380001F02EFC462132462346282001F028FCE0
:1018480064212A462346282001F022FC82214246B0
:101858002346282001F01CFC524623462820A021BC
:1018680001F016FC28205A46BE21234601B0BDE8E7
:10187800F04F01F00DBC00BFA01100205E940508D8
:1018880091170008D89505086D170008C595050833
:1018980089160008BA95050875150008E395050826
:1018A800A1140008EE9505088D1300085A9505083F
:1018B800C9120008034B01224FF4FC601A7003F0B0
:1018C800A7B900BFD90C00200B4B10B50024204647
:1018D8001C7003F0C9F906F0C9FF06F083F9074B3D
:1018E8001C70074B01221A7006F0BAFF0548BDE8C4
:1018F800104000F074B900BFD90C002068420020E5
:10190800F03B00206C0E00200A4B10B50024204646
:101918001C7003F0A9F906F0A9FF074B1C70074BD0
:1019280002221A7006F09CFF0548BDE8104000F03E
:1019380056B900BFD90C002068420020F03B0020B7
:10194800B40F002008B5064B0020187003F08CF97E
:10195800044B054803221A70BDE8084000F03FB95F
:10196800D90C0020F03B0020581000200C4B10B57B
:1019780000220C4C1A7006F079FF04F001F906F009
:101988003EFC06F06DFF20684FF6E07100F0BCFDEC
:101998002068054900F066FDBDE8104001F0E2BE90
:1019A800D90C00200C0C0020F89505080E4B0022DD
:1019B80010B51A700088C83880B2042805D90B48B9
:1019C8000B4A0C4B872102F0F5F80B4CC0B204F01F
:1019D80061F920684FF6E07100F096FD206807492C
:1019E800BDE8104000F03EBDD90C00200C9605085B
:1019F8000CD503082C9605080C0C00205D960508EC
:101A08002DE9F04F5848594D87B0002401F071FC7A
:101A18004FF6FF712246234655480094019400F082
:101A280037FD042607464FF6E07122462346514803
:101A38000096019400F02CFD4FF6E0718046224696
:101A480023464D480096019400F022FD4FF6FF71A1
:101A580081462246234649480096019400F018FD25
:101A6800234628604FF6FF712246454800960194A8
:101A780000F00EFD43496860434A204601F0F0F942
:101A88004249434A8246204601F0EAF94149424A1E
:101A98008346204601F0E4F940490390404A204635
:101AA80001F0DEF93F4904903F4A204601F0D8F999
:101AB8003A46059021462C4B204601F0E9FA21468A
:101AC8004246294BC82001F0E3FA0A214A46264B30
:101AD800C82001F0DDFA2A68234B6421782001F040
:101AE800D7FA78206A68204B014601F0D1FAC82558
:101AF80005262827E0B203F0FDFF2C4A01462846B8
:101B080001F0AEF994FBF6F106FB114179431E3161
:101B1800024689B20020144B0134013501F0B8FAAD
:101B2800042CADB2E6D1D221524605200E4B01F06D
:101B3800AFFAD2215A464C200B4B01F0A9FAD22118
:101B4800039A094B9C2001F0A3FAD221049A064B70
:101B5800EC2001F09DFA059A034BEC20B42107B064
:101B6800BDE8F04F01F094BAFC1000200C0C0020E6
:101B78006D96050877960508849605088F960508DA
:101B880068940508A396050875190008AB9605081A
:101B98004D190008B496050811190008BD960508E6
:101BA800D1180008C6960508BD180008B519000820
:101BB80008B500F03DFAFEF721FBFEF751FDFEF7F0
:101BC80083FBFFF7FBFDFFF71BFFFEF7D1FB00F0E0
:101BD800D5FA00F0D9F8BDE8084000F0A1B910B571
:101BE800044628B90F48104A104B452101F0E2FF7E
:101BF8000F4B1868844213D010B1C369002198476D
:101C0800002003F031F8002003F018F84FF6FF70B9
:101C180002F0FEFFE369204601219847044B1C604F
:101C280010BD00BFCF9605081BD50308EB96050825
:101C3800140C00200048D2E7FC1000204FF6FF707B
:101C480070474FF6FF70704713B5002944D04FF224
:101C5800DE7003F009F8002003F0D0F80F2002F03E
:101C6800D7FF1E4C1E4A412101230A2003F0FEF82B
:101C7800042003F0C3F8236828209621042B21DCD4
:101C88000123184A03F0F2F801A90DF106022068B1
:101C980003F072FB0F2002F0BBFFBDF80400BDF893
:101CA800061014382822002380B202F0E1FFBDF8A4
:101CB8000610BDF80400143989B22822012302F065
:101CC800D7FF09E0084A012303F0D0F81E20A52118
:101CD800064A012303F0CAF81CBD00BF180C0020F7
:101CE800FB9605080E9705082A97050840970508EA
:101CF80037B51E4C2368042B05462BDC01A80DF1D3
:101D0800060103F037FBBDF80630BDF8042018497A
:101D180004200AF047F82368002B04DA1548164A0D
:101D2800164B592105E0042B05DD1248124A144BC5
:101D38005A2101F03FFF04EB8302BDF80410013380
:101D48009180BDF806102360052BD18008D1201D95
:101D580003F092FB00230B482360FFF740FF03E0EA
:101D680028460121FFF770FF3EBD00BF180C002078
:101D7800579705089C9705082DD50308BE970508B1
:101D8800D59705084412002037B50B4C204601F0C2
:101D9800B0FA0A4B0A49009300250120094A0A4B68
:101DA800019501F04EF9294602462346284603B01C
:101DB800BDE8304001F06CB9100F0020511C00083C
:101DC800451C00084B1C0008F91C00084FF6FF7062
:101DD80070474FF6FF7070471FB54FF6E07002F07E
:101DE80043FF002003F00AF80F2002F011FF002142
:101DF800294A2A4C01230A2003F038F8002002F06F
:101E080007FF042002F0FAFF0A201921244A0123BF
:101E180003F02CF82521234A01230A2003F026F891
:101E28001F2002F0F5FE01230A2037211E4A03F085
:101E38001DF8237873B301231E2096211B4A03F053
:101E480015F862881A49684611F0F8FB01231E202C
:101E5800A2216A4603F00AF8A2881649684611F0DA
:101E6800EDFBAE216A4601231E2002F0FFFF0F2082
:101E780002F0CEFE6088A188143880B228220023A0
:101E880002F0F6FEA1886088143989B2282201235D
:101E980002F0EEFE1FBD00BF03980508300C0020BD
:101EA800159805083598050855980508789805087F
:101EB8008A9805089798050801B18DE7704713B50A
:101EC8000DF1060101A803F009FA144B01221A705A
:101ED8005988BDF80420891A0E311C2919460AD8D8
:101EE8009C88BDF80600201A0E301C2803D8996873
:101EF8000131996001E000238B60084B9968012942
:101F080005DD00229A601A70FFF794FE05E05A80FA
:101F1800BDF806209A80FFF75FFF1CBD300C00203B
:101F280037B50B4C204601F0E4F90A4B0A490093F7
:101F380000250120094A0A4B019501F082F829463B
:101F480002462346284603B0BDE8304001F0A0B859
:101F580044120020C11E0008D51D0008DB1D000822
:101F6800C71E000808B507F0C7FD164A002302205F
:101F7800CA2102F07BFF144B1A68144B1A60144BE9
:101F88001B78023B052B1CD8DFE803F003070B1373
:101F9800170FBDE80840FFF7E5BBBDE80840FFF7AD
:101FA8006FBBBDE80840FFF7E1BABDE80840FFF79E
:101FB800E9B9BDE80840FFF76FBABDE80840FFF788
:101FC8007FB908BD67940508503C002054420020A2
:101FD8006842002038B50E4B0E4D00241C700E4B85
:101FE8001C7007F01BFE0D4B1A680D4B20461A603B
:101FF80002F03AFE0B4B1B78022B0CBF0A480B4829
:10200800FFF7EDFD2C70BDE8384007F06DBD00BF4F
:1020180068420020D4430020383C0020503C002077
:1020280054420020F03B0020B40F00206C0E00202A
:1020380070B5124C204601F05CF90020014622469A
:1020480000F086FA00200E490E4A00F009FF0E49FA
:102058000E4A0646002000F003FFD221054632460C
:1020680023464FF4827001F013F8DC20D2212A466F
:102078002346BDE8704001F00BB800BF30140020C3
:1020880005950508DD1F0008A49805086D1F0008C0
:1020980010B5064C4FF6FF71206800F035FA044B76
:1020A80020681968BDE8104000F0DCB93C0C00203D
:1020B8009801002008B5002002F0D6FD054B1868ED
:1020C800054B196800F0CEF90448BDE80840FFF751
:1020D80086BD00BF3C0C002094010020FC100020AD
:1020E80008B5FFF7D5FF0020014605F009FFBDE858
:1020F800084001F037BB0088A0F5C87080B20928F5
:1021080008B505D90748084A084B8F2101F052FD48
:10211800074B1880074BFF21197005F0F1FEBDE849
:102128000840B5E7A89805083FD50308CB980508E7
:10213800D4140020D61400200088A0F5967080B230
:10214800092808B505D90848084A094B832101F030
:1021580031FD084B1880084B0121197005F0D0FE9D
:10216800BDE8084094E700BFA898050854D50308BF
:10217800CB980508D4140020D61400202DE9F3418B
:1021880000243A483A4D01F0B4F8224623464FF667
:10219800FF7138480094019400F07AF90426224629
:1021A800234607464FF6FF7133480096019400F026
:1021B8006FF92346286022464FF6FF712E48009695
:1021C800019400F065F92D4968602D4A204600F019
:1021D80047FE2C492C4A0646204600F041FE21467F
:1021E80080463A462046214B00F052FF2A681F4B92
:1021F8002046282100F04CFF3246D2211B4B5A20A2
:1022080000F046FFAA20D2214246184B00F040FFBA
:102218000F254FF4967440F2351620461B491C4A88
:1022280000F01EFE01340246782128460F4BA4B266
:10223800233500F02DFFB442ADB2EED10F254FF497
:10224800C87440F2991620461249134A00F008FE55
:10225800013402469B212846044BA4B2233500F0E2
:1022680017FFB442ADB2EED1BDE8FC818C1300205B
:102278003C0C0020FC980508799405080899050885
:10228800E920000811990508BD2000081A990508D9
:10229800412100081C990508FF20000808B508B16D
:1022A80043682BB90348044A044B9B2101F082FC84
:1022B800586908BD1E99050868D50308409905089E
:1022C80008B5FFF7EBFF8068123080B208BD08B58B
:1022D800FFF7E4FF4068063080B208BD2DE9F84FEB
:1022E80004468846FFF7DAFF6689E589074606F15E
:1022F800030905F10F0AB8F1000F1FD01F2002F0E3
:1023080087FC2046FFF7DCFF83462046FFF7DFFF08
:10231800294603465FFA8BF2F0B202F0ADFC0420C6
:1023280002F06CFD0B364FF6FF70033502F070FCBF
:10233800B0B2A9B23A68012302F098FD3D6920467F
:1023480041464A465346A847BDE8F88F13B50446A8
:102358000DF1060101A802F0C1FF2046FFF79EFF1C
:102368006389BDF80410BDF80620C91AE389D21A9A
:102378000339C3680F3A204698471CBDF7B5044691
:1023880014200D4616461F4610F0E6FD089BC76050
:102398000361064B0649074A80E8700000930190E4
:1023A800054B002000F04DFEFEBD00BFE5220008F1
:1023B800D7220008C922000855230008704708B52D
:1023C80008B143682BB90448044A054BAD2101F014
:1023D800F1FB586908BD00BF5F99050880D503085F
:1023E80040990508F8B505460E46FFF7E8FF836BE8
:1023F80004461BB128463146984700E018466F89C5
:1024080094F83C30ED890EB9034310D0208E02F0C9
:10241800FFFB608E02F012FC94F8350002F0EEFC2F
:1024280094F8343038462946224602F01FFD00232E
:1024380084F83C30F8BD08B5FFF7C1FF90F83500C7
:10244800BDE8084002F0EFBC38B5FFF7B8FF044616
:1024580011F07AF9054694F8350002F0DFFC68437C
:1024680080B238BD38B50D46FFF7A9FF29462E22A0
:10247800044611F099F950B1204629462E2211F050
:10248800E5F9002384F82E30012384F83C3038BD68
:102498002DE9F743074640200E461546984610F0AA
:1024A8005BFD044628B91148114A124B4E2101F030
:1024B80081FB114B114A12498DE818000020114B7D
:1024C80000F0BFFD39468146FFF7CCFF9DF8283064
:1024D800268684F835300B9B6586A363002384F831
:1024E800348084F83C304846BDE8FE835F9905088F
:1024F80098D503087D990508ED2300083F240008B6
:1025080051240008C523000810B50C46FFF757FFF3
:102518000123048680F83C3010BD00BF4FF4A07042
:102528007047C82070477047074B1B78022B07B5C8
:1025380008D1064B1B78022B04D001A80DF1060127
:1025480002F0CCFE0EBD00BFD4430020684200203C
:1025580073B50A4B06460D461446009300200849F9
:10256800084A094B019000F06CFD294602462346B3
:10257800304602B0BDE8704000F08ABD2F25000843
:10258800252500082B2500083125000813B502ABC6
:1025980003E90600436843B1027C0124082A9C70C1
:1025A80004D11B692146984700E01C4620461CBD03
:1025B80030B500282BD0058B002425E0036A1A7C4F
:1025C800012A05D15B681A888A421BD1187F30BD61
:1025D800052A06D15B681A888A4213D193F82C0021
:1025E80030BD032A06D15B681A888A420AD193F85B
:1025F800250030BD062A05D15B681A888A4201D1B8
:10260800D87A30BD01340430AC42D7D3002030BD75
:1026180008B1817501207047F8B504460D46D0B160
:10262800E175D0F898309847012D0DD1274600263E
:1026380006E0F86900F10802436906CA98470136BE
:10264800238B04379E42F4D3D4F898302046294689
:1026580098470120F8BDF8BDF8B505460846174665
:102668000E4611F071F8013FB84234BF04463C46AB
:102678003CB128463146224611F0E8F800232B5594
:10268800F8BD2C70F8BDF7B5044600200090019005
:1026980000296CD00E8B68E000F1080351F8233054
:1026A8001D7C042D04D15D682D88954247D00130EA
:1026B80000F1080351F823301D7C012D04D15D6819
:1026C8002D8895423BD0013000F1080351F82330A2
:1026D8001D7C052D04D15D682D8895422FD00130D1
:1026E80000F1080351F823301D7C032D04D15D68E7
:1026F8002D88954223D0013000F1080351F823308A
:102708001D7C022D04D15D682D88954217D00130BB
:1027180000F1080351F823301D7C072D04D15D68B2
:102728002D8A95420BD0013000F1080351F823306F
:102738001D7C062D08D15D682D88954203D103F1D3
:102748000801204615E0013000F1080351F8235034
:102758002B7C082B09D16F683F88974204D105F17B
:10276800080120461A4605E00130B04294D32046BD
:102778006946082210F0A0FE2046FEBDF8B50546C1
:102788000F461646002830D04388032B2FD0202030
:1027980010F0E2FB044600282BD040F80C5B3946C9
:1027A8000C22FFF759FF1820E66110F0D5FB06460A
:1027B800B8B102230374012363760F4B446063604E
:1027C8000E4BA360002323766B8805EB830201334D
:1027D8009BB2012B50606B800CD16A6852681376EB
:1027E80008E0204610F0C0FB04E0064602E00026A0
:1027F80000E006463046F8BDE45404088251040857
:1028080037B5456802AB03E906003DB3037C0124F4
:10281800042B85F8314022D1688E02F0F9F995F839
:10282800300002F0EBFA95F8343043B9BDF80200F5
:10283800BDF80610AA1C234602F018FB0FE0012B76
:1028480003D1084840F2395104E0022B07D105486A
:1028580040F24151044A054B01F0ACF92C462046A0
:102868003EBD00BF90990508582004088E990508B8
:10287800F8B504460F46164610B3838A0A2B20D0B3
:10288800202010F069FB0546E8B14460102200F1F1
:1028980008003946FFF7E0FE4FF6FF73A08A2B8049
:1028A8001F236B8000232B76831D013080B2012803
:1028B800EE6144F82350A08207D1A3691876F8BDC9
:1028C800F8BD0020F8BD0120F8BD0120F8BD2DE9B4
:1028D800F0411D464B1C984280460C4617460CDDBD
:1028E80095420ADC013208F101035B1A521BC8B297
:1028F800D2B29BB2294602F0BDF9A8F10208BDF890
:102908001800C4EB080802F083F901261FFA88F8BA
:1029180008E0A919601C80B289B24246002302F07F
:10292800A7F901367B1B9E42F3D3BDE8F081F8B5C9
:10293800C7B2144638461E460D4602F09FF9621E7D
:1029480092B23846294602F099F9304602F060F909
:10295800022606E0A21B92B23846294602F08EF9FA
:102968000136A642F6D3F8BD70B5044600F11E0044
:102978003C22002380B20D4602F07AF91E3DA9B22E
:1029880020463C220123BDE8704002F071B970B5C1
:10299800044601380322002380B20D4602F068F98C
:1029A800013DA9B2204603220123BDE8704002F090
:1029B8005FB9F7B5089D2E7BEF7A1C463604AB7AD3
:1029C80006EB0726F618431A687B06EB00602D18FD
:1029D80000200190121B08462146009501F098FE40
:1029E800FEBD30B5456885B004AB03E906007DB18E
:1029F80001242C736D68BDF80800BDF80A109DF815
:102A08000C209DF80E300095FFF7D3FF204600E01C
:102A1800284605B030BD2DE9F04385B004AB03E985
:102A280006004468BDF80860BDF80C70002C41D061
:102A3800012384F8263094F825300BB9A26800E009
:102A48006268FFB2BDF80A109DF80E300092304659
:102A58003A46FFF7AEFF04F10C08022002F0CEF967
:102A6800404610F071FE054600B1451E0F3F002498
:102A7800153E1FFA87F90DE002F0CAF902F0CEF907
:102A880004FB106189B248462022002302F008FAAC
:102A98000134E4B2AC42EFD3002002F0B9F8B8B286
:102AA800B1B24246012302F0FBF9002002F0A6F978
:102AB800012000E0204605B0BDE8F0832DE9F04391
:102AC80085B004AB03E906004568BDF80860BDF8A9
:102AD8000C70002D3CD001236B762B7EBDF80A10BC
:102AE800012B0CBF6A68AA689DF80E300092FFB2ED
:102AF8003A463046FFF75DFF0C35022002F07EF9BA
:102B0800284610F021FE0E3F81460024163E1FFA8B
:102B180087F80DE002F07CF902F080F904FB1061FF
:102B280089B240462022002302F0BAF90134E4B207
:102B38004C45EFD9002002F06BF8B8B2B1B22A4682
:102B4800012302F0ADF9002002F058F9012000E05D
:102B5800284605B0BDE8F0832DE9F04F85B005465D
:102B6800DDF84090029148469046039310F0ECFD42
:102B7800DDF838A0DDF83CB00646294600242F468B
:102B880011E024B1B4420CBF5B46534600E0039BFE
:102B980001F10805ADB200932846029A4346FFF7B3
:102BA80008FF01342946B442EBDD002002F030F87A
:102BB800022002F023F97D1D08F10508A8B21FFACA
:102BC80088F14A46012305B0BDE8F04F02F04EB93E
:102BD80070B5406886B006AB03E9060000282ED021
:102BE800012380F82D308668164BF21A534243EBC6
:102BF800020390F82C205AB1002B134D134B144AA2
:102C080008BF1D46134B00F11C0418BF13460AE009
:102C1800002B0D4D0D4B0E4A18BF1D460D4B00F1F4
:102C28000C0408BF1346BDF81200BDF81410BDF817
:102C38001620009601950294FFF78EFF012006B03A
:102C480070BD00BFC829040804260408AA2B04087C
:102C5800E62704088C2D040870B5446886B006ABD6
:102C680003E9060004B301236377A668104B227FAB
:102C7800F11A4B4243EB01030AB10BB904E01BB94B
:102C880066680C4D0C4B01E00C4D0D4BBDF8120065
:102C9800BDF81410BDF8162000960C340195029466
:102CA800FFF75AFF012000E0204606B070BD00BFC4
:102CB800143504085031040832330408EA3604088D
:102CC800C03804082DE9F04385B004AB03E90600D9
:102CD8004468BDF80860BDF80A90BDF80C50BDF80E
:102CE8000E80002C00F08C800123A37402206768FA
:102CF80002F084F84FF6FF7001F0A0FF002001F009
:102D080087FFEDB25FFA88F8A6F1160189B230465E
:102D18002A4643460097FFF74CFE277A002F2ED10C
:102D2800A28A234600E00137974204D29969097EB6
:102D380004330029F7D002F06BF802F06FF8A9F11C
:102D480016091FFA89F90E2101FB10914FF6FF723F
:102D580008F101085FFA88F389B2009248462A46CA
:102D6800FFF7B5FD022002F049F81F2001F050FFDF
:102D7800A38A002B38D0103DE8B2303E2CE0E3683F
:102D88005C68A28A2346013A002700E0013797428F
:102D980004D29969097E04330029F7D002F038F883
:102DA80002F03CF80E2101FB10914FF6FF7208F17A
:102DB80001085FFA88F389B2009248462A46FFF76D
:102DC80086FD022002F01AF81F2001F021FFA38AD5
:102DD80053B1103DE8B21A3E0637B1B254F8272075
:102DE8000123083202F05CF8002002F007F84FF6E1
:102DF800FF7001F023FF1F2001F00AFF012000E00F
:102E0800204605B0BDE8F0832DE9F041054636209F
:102E1800884614461F4610F09FF80646E0B120F891
:102E2800025B41462E22FFF717FCBDF8183086F8E2
:102E3800344073861820012386F8307086F83130C4
:102E480010F08AF8044618B104234660037404E0BD
:102E5800304610F089F800E004462046BDE8F081CD
:102E6800F8B5064624200F46154610F075F80446B6
:102E7800D8B10F4B068083600E4B39464360102251
:102E880000F10C00FFF7E8FB01260023182025625B
:102E98002377667710F060F8054610B14460067431
:102EA80004E0204610F060F800E005462846F8BD2A
:102EB800143504086E2F0408F8B506462C200F4672
:102EC800154610F049F80446E8B120F80C6B39466D
:102ED8001922FFF7C1FB0D4BA562A3600C4B636081
:102EE800002384F825301820012384F8263010F0B8
:102EF80033F8054618B103234460037404E0204600
:102F080010F032F800E005462846F8BD204E0408C7
:102F1800BE4A040810B50446142010F01DF820B16C
:102F280000234380014B0480036110BD85270008FE
:102F380038B50546442010F00FF80446C0B10E4BD2
:102F4800058243600D4B03600123837400230372E1
:102F580083820B4B036418200FF0FEFF054618B15F
:102F680007234460037404E020460FF0FDFF00E0EF
:102F78000546284638BD00BFB4460408AA420408DE
:102F8800792800082DE9F041054634208846144682
:102F98001F460FF0E1FF064620B3144B05808360FF
:102FA800134B41464360102200F10C00FFF754FB1D
:102FB800214606F11C001022FFF74EFB002386F87D
:102FC8002C3018200123376386F82D300FF0C4FF0A
:102FD800044618B105234660037404E030460FF038
:102FE800C3FF00E004462046BDE8F081C829040874
:102FF800222404082DE9F041044614200D46164603
:1030080098460FF0A9FF0746B8B1069B04800361F4
:103018000023C37201234560068180F80A80037388
:1030280018200FF099FF044618B10623476003746F
:1030380004E038460FF098FF00E004462046BDE85B
:10304800F0812DE9F041044618200D4616469846B1
:103058000FF082FF0746B8B101238370069B0480F6
:103068000361079B45608660C0F80C8043611820A7
:103078000FF072FF044618B108234760037404E098
:1030880038460FF071FF00E004462046BDE8F081A5
:103098002DE9F34198461B8B1D2B05460C46174618
:1030A8004FF0000000F2B480B5F5A07F00900190C9
:1030B80000F2AE80F02900F2AB80127CADF8061069
:1030C800511EADF80250072900F28A80DFE801F0AE
:1030D80045595E04456A14767B684E4A7A611A88B7
:1030E80093F834303A80013BDBB2012B7FD8ADF83E
:1030F8000240ADF806507AE005F11602ADF800205E
:1031080004F11602ADF8042002AE434A16E90300A2
:103118007A6107F1080282E8030003F1080201332B
:1031280048F82270A8F818307B681A8A187A3A800A
:1031380000286CD1FFF7FCFE3849436859603849CC
:10314800DF600126163D196002461E72A8B2E1B280
:103158004346FFF79DFF30465AE0012A0CBF314B2A
:10316800314B78687B6130F80C3B3B8010F0ECFA0F
:10317800431CDB001A34ED18ADF80440ADF80050DC
:1031880035E07B68294A1B687A6102E0284A7B6837
:103198007A611B8814353B80ADF800501434ADF8C3
:1031A800044024E07B68234A7A611A883A801A89A5
:1031B8009B7AAD18ADF80050E418F0E77E681E4B16
:1031C8007B61338838463B8073689847013D4519D1
:1031D800ADF80050B36838469847013C0419DEE75B
:1031E8001648174A174B40F21A3100F0E3FC02AABE
:1031F80012E9030007F1080383E80300B8F8183060
:1032080003F10802013348F82270A8F818300120A9
:10321800BDE8FC8109280008CD2C0008A03E040860
:10322800963A0408612C0008D92B0008C52A000822
:103238001F2A0008EB290008952500089099050821
:10324800682004088E990508F8B51646002834D079
:103258001378002B2ED0028B002327E0046A257CEC
:10326800042D21D165682F888F421DD195F8313002
:1032780053B16F8E01F0F2FC04F1080268866369AD
:10328800204606CA98476F86A81C31462E22FFF7AB
:10329800E3F995F831307BB104F1080263692046FF
:1032A80006CA98470120F8BD013304309342D5D3AC
:1032B8000020F8BD1846F8BD0120F8BD70B5B8B1BA
:1032C800068B0446002310E0256A287C04280AD1CE
:1032D8006D682888884206D11046A91C2E22FFF75F
:1032E800BBF9012070BD01330434B342ECD3002094
:1032F80070BD38B5044620B3134BC361134BC0F8F7
:103308009830134BC0F89C30124B00257822C0F837
:10331800A0308575C5750583294600F1200010F099
:103328000DF9D4F898302046294698470A4A138858
:10333800312B07D8094941F8234001331380012074
:1033480038BD38BD284638BD212600081926000892
:10335800B92500088F260008440C0020D814002046
:103368002DE9F0410446002800F0B380078B02469F
:103378000025A8E0136A1E7C042E00F08780012E29
:1033880023D1586803888B4240F09B8005F10807D9
:103398000FF0EAFD54F827004FF00008C0F8048049
:1033A8000FF0E2FD228B531E9D4208D00732238383
:1033B80054F8221044F8271044F8228002E044F818
:1033C800278025833046BDE8F081052E5ED0032E88
:1033D8005CD0022E13D15B68186803888B4270D1C9
:1033E8004388013B9BB243800BB90FF0BDFD05F14B
:1033F800080654F8263058680FF0B6FD4EE0072E40
:1034080021D15E68338A8B425BD1002706E0BB1D61
:10341800013756F823000FF0A7FDFFB2B38ABB426D
:10342800F5D80027B78205F1080654F82630586801
:103438000FF09AFD54F8260033E044F826702583EF
:103448000120BDE8F081062E1ED1586803888B4202
:1034580037D105F108060FF087FD54F8260000273C
:1034680047600FF081FD228B531E9D4209D008331F
:10347800013A54F82310228344F8261044F82370A4
:10348800DEE744F826701AE0082E1AD15868038837
:103498008B4216D10FF068FD05F1080654F8260096
:1034A800002747600FF060FD228B531E9D42C4D059
:1034B800073254F8221044F8261044F82270238367
:1034C800BEE701350432BD42FFF454AF0020BDE829
:1034D800F081BDE8F08170B5044600282AD0068B3B
:1034E800751E083600EB86061EE056F8043D1A7C69
:1034F800042A13D0012A11D0052A0FD0032A0DD08F
:10350800022A02D15B681B6809E0072A02D15B68BE
:10351800198A05E0062A01D0082A04D15B681988AF
:103528002046FFF71DFF013D681CDED100232383E1
:10353800012070BD70BDF0B528B30023068B1A4674
:103548001EE0046A257C072D18D16468258A8D42FF
:1035580014D1A78A002504EB83040DE004EB050CC5
:103568000435DCF818C09CF818C0BCF1010F03F151
:10357800010301D1D8B2F0BDBB42EFD30132043010
:10358800B242DED30020F0BD70B508B3048B00232F
:103598001BE0026A157C072D15D15268158A8D42E9
:1035A80011D10023958A11461C46012007E013B962
:1035B8009669307601E08E69347601330431AB4286
:1035C800F5D3012070BD01330430A342E1D30020BC
:1035D80070BD2DE9F04128B30023078B1A461EE081
:1035E800046A257C072D18D16468258A8D4214D178
:1035F800B4F814C0002504EB83040CE06619043504
:10360800B66996F81880B8F1010F03D106F10800E1
:10361800BDE8F08101336345F0D301320430BA428A
:10362800DED30020BDE8F0812DE9F04700282FD037
:103638000023B0F818C01D4627E0046A267C072E30
:1036480021D16468268A8E421DD1B4F814800026E0
:1036580004EB830915E009EB0604A7693C7E012CFD
:103668000DD192F800A0BAF1000F08D007F10800B8
:1036780011461022FEF7F0FF2046BDE8F08701331F
:1036880004364345E7D3013504306545D5D30020DA
:10369800BDE8F087F0B5B0B1068B002510E0046AEC
:1036A800277C062F0AD1646827888F4206D1238198
:1036B8009DF814306260A3720120F0BD013504301A
:1036C800B542ECD30020F0BD10B500210446FEF74A
:1036D800A3FF20460121BDE81040FEF79DBF38B585
:1036E80098B1048B024600230CE0106A0588043266
:1036F8008D4206D100F10802436906CA98470120A5
:1037080038BD0133A342F0D3002038BD10B50C46B4
:103718000021FEF781FF20460121BDE81040FEF799
:103728007BBF13B502AC04E90C00BDF8023083423C
:1037380006D8BDF80030834234BF0020012000E0E5
:103748000020BDF806308B4206D8BDF804308B4205
:1037580034BF0021012100E00021002818BF0846DD
:10376800C0B21CBD38B5114B114A1988002319E0A5
:1037780052F8045FA87D012812D100240CE004F15E
:10378800080355F82300037C082B03D14368002164
:103798001B6998470134A4B22B8BA342EFD838BDDC
:1037A80001339BB28B42E3D138BD00BF440C0020EB
:1037B800D4140020704770B5094CA5787DB9094B21
:1037C8001E78012E0BD16368013363606268064B73
:1037D8009A4204D9284601F0D3FAA670656070BDF4
:1037E800440C00203000002040420F00054A906041
:1037F800134602E099680139996091680029F9D166
:10380800704700BF440C0020F0B585B001F064FD9E
:10381800002800F04981002502A80DF10A01ADF841
:103828000850ADF80A5001F059FD03A80DF10E013A
:10383800ADF80C50ADF80E5001F09CFDBDF80C1021
:10384800BDF808200091BDF80E10BDF80A300191AE
:103858002C46964D9649082008F0A4FAA878012825
:1038680003D101F08DFAAC7019E1924B5B78012B12
:1038780040F01581AB78002B40F011816B602988EE
:103888008D4A09E152F8046FB07D012840F00281A9
:103898000025FAE005F10803BDF8080056F82340B2
:1038A800BDF80A1004F108030CCBFFF73AFF002813
:1038B80000F0E980237C013B062B00F29F80DFE8C3
:1038C80003F00429159D1F9D4C006668012304F12F
:1038D8000805337795E80600636920469847002372
:1038E80033772046636995E8060086E0636893F8B5
:1038F800252012F1FF3218BF012283F8252077E036
:10390800636893F82C2012F1FF3218BF012283F864
:103918002C206DE06268137E1568002B6ED16E88CE
:103928002F462946184606E051F804EFDEF804E071
:1039380001338EF81800B342F6D30123137600261C
:1039480007E057F8040F00F10802436906CA9847D0
:1039580001366B889E42F4D350E0656820892E6852
:10396800A37B227B0096A0F1160189B2FFF721F80C
:103978001420FFF73BFF2B7AC3B9AF8A29461A46B2
:103988001E4609E0886990F818E00676BEF1010F36
:1039980008BF134604310132BA42F3D301220BB9EE
:1039A800AB6924E0053355F8233020E06368DB6811
:1039B8005A680023908A154619461F4609E0AE69E1
:1039C80096F818E03776BEF1010F08BF0B460435AC
:1039D80001318142F3D3411E8B4203D1053052F8A5
:1039E800203003E004D2073352F8233001221A763C
:1039F80004F1080206CA636920469847237C013B04
:103A0800072B4CD8DFE803F00410074B0A0D123AD5
:103A180063681B6A34E063689B6A2DE063681B6B0C
:103A28002AE063681B6927E0636824E063681A7A00
:103A38007AB9988A1946013800E00132824204D2E4
:103A48008C69247E0431002CF7D0063253F82230DA
:103A580011E0DB685A68908A11460138002300E0BB
:103A68000133834204D28C69247E0431002CF7D0C0
:103A7800063352F82330DB69984710E06368DB6847
:103A8800204698470BE00135ADB2338BAB423FF689
:103A980001AF04E001339BB28B427FF4F3AE01F037
:103AA80061FC0F20FFF7A2FE05B0F0BD440C00201A
:103AB800B699050830000020D4140020034B9A68FA
:103AC80012B19A68013A9A60704700BF440C00200E
:103AD8002DE9F3470120DFF8D080DFF8D0900146C8
:103AE80009F0FAFC0025012403234FF4807602270D
:103AF800404669468DF8053000968DF804708DF8BB
:103B080006508DF8074009F03FF940460821224643
:103B180009F0BAF9234BDFF898801A6844F2A243F7
:103B2800B2FBF3FA0AF1FF3A204621461FFA8AFA55
:103B380009F002FDC8F804A048464146A8F800501C
:103B4800A8F80250A8F8085088F80A500AF090F827
:103B58007023A8F80C300423A8F810300AF1FF3AB3
:103B68006323642203FB0AF3B3FBF2F39BB2C8F8A6
:103B7800143008F10C014846A8F80E40A8F818704F
:103B8800A8F81A50A8F81C60A8F81E500AF08EF978
:103B9800484621460AF001F9484621460AF007FC42
:103BA800BDE8FC879C0100200000024000000140A5
:103BB800540C002083B50E460746154910201C46B4
:103BC800154608F0EFF81020124908F0EBF810201D
:103BD800114908F0E7F810200E4908F0E3F800232F
:103BE80010200E49019308F0DDF8334610200C49E7
:103BF8003A4608F0D7F810200A492A4608F0D2F8C1
:103C080010200949224608F0CDF8019B0133E7E767
:103C1800F0990508F5990508159A0508259A0508E3
:103C2800359A05084A9A05085B9A050808B5164B9F
:103C38001A6A01321A621A6A012A1A4603D013480C
:103C48004FF4A0710FE05862194602E04B6A013B3D
:103C58004B62506A0C4B0028F8D11A6A012A06D028
:103C68000A4840F24B110A4A0A4BFFF7A3FF1A6AA7
:103C7800013A1A621B6A2BB10448054A064B40F206
:103C88004D11F2E708BD00BF540C00206C9A0508DE
:103C980046580408969A0508A79A05080C4B0D493A
:103CA8001A6844F2A2436428B2FBF3F3D4BF20EAB3
:103CB800E0706420013B9BB24B60013B5843642297
:103CC800B0FBF2F080B2486103480C310AF071B8D9
:103CD8009C010020540C00200000014010B5134B3B
:103CE80093F828202AB11248124A134B4FF40A714C
:103CF8000EE0012283F8282066234FF0C042013BE2
:103D0800DBB2108033B90A480A4A0C4B40F2322120
:103D1800FFF750FF1488A4B28442F0D1084B1980F1
:103D2800024B002283F8282010BD00BF540C00204D
:103D38006C9A050850580408B89A05088E99050821
:103D48000000026010B5FFF7C3FE6420FFF7A6FF6E
:103D5800E5204FF40041FFF7C1FF00200121FFF7E4
:103D6800BDFF01204FF48071FFF7B8FF02204FF428
:103D7800E061FFF7B3FF032041F23001FFF7AEFF28
:103D880004200021FFF7AAFF082040F20221FFF7D4
:103D9800A5FF09200021FFF7A1FF0A200021FFF756
:103DA8009DFF0C200021FFF799FF0D200021FFF750
:103DB80095FF0F200021FFF791FF10200021FFF74A
:103DC8008DFF11200021FFF789FF12200021FFF746
:103DD80085FF13200021FFF781FF102041F2B07109
:103DE800FFF77CFF37211120FFF778FF3220FFF71C
:103DF8001DFF122040F23B11FFF770FF3220FFF742
:103E080015FF13204FF4C051FFF768FF0F21292039
:103E1800FFF764FF3220FFF709FF20200021FFF79A
:103E28005DFF21200021FFF759FF30200021FFF717
:103E380055FF31200721FFF751FF322040F20311CF
:103E4800FFF74CFF352040F20741FFF747FF40F2EC
:103E58000444362040F60F11FFF740FF3720214673
:103E6800FFF73CFF38204FF48061FFF737FF392018
:103E78002146FFF733FF3C200021FFF72FFF3D20AD
:103E88004FF48061FFF72AFF50200021FFF726FF3B
:103E9800EF215120FFF722FF52200021FFF71EFFDC
:103EA800532040F23F11FFF719FF60204FF41C51D7
:103EB800FFF714FF61200121FFF710FF6A2000219E
:103EC800FFF70CFF80200021FFF708FF8120002169
:103ED800FFF704FF82200021FFF700FF8320002165
:103EE800FFF7FCFE84200021FFF7F8FE8520002163
:103EF800FFF7F4FE90201021FFF7F0FE922000213A
:103F0800FFF7ECFE93200321FFF7E8FE95204FF41E
:103F18008871FFF7E3FE97200021FFF7DFFE982066
:103F28000021FFF7DBFE072040F27311BDE81040C7
:103F3800D4E610B5FFF7CCFD6420FFF7AFFE2121D2
:103F48000720FFF7CBFE3220FFF770FE012100208B
:103F5800FFF7C4FE3220FFF769FE23210720FFF791
:103F6800BDFE3220FFF762FE00211020FFF7B6FEEB
:103F780041F28830FFF75AFE33210720FFF7AEFEE3
:103F88003220FFF753FE112046F63001FFF7A6FE58
:103F98003220FFF74BFE4FF4C0610220FFF79EFE70
:103FA8003220FFF743FE122046F6EB41FFF796FE5C
:103FB8003220FFF73BFE03204AF6A401FFF78EFEEE
:103FC8003220FFF733FE00210C20FFF787FE322056
:103FD800FFF72CFE0D2040F60C01FFF77FFE322084
:103FE800FFF724FE0E204FF42C51FFF777FE322006
:103FF800FFF71CFEB0211E20FFF770FE3220FFF7EE
:1040080015FE012042F63F31FFF768FE3220FFF728
:104018000DFE05200021FFF761FE3220FFF706FEA6
:1040280000210620FFF75AFE3220FFF7FFFD162079
:104038004EF61C71FFF752FE3220FFF7F7FD1720EE
:1040480040F20311FFF74AFE3220FFF7EFFD00218F
:104058000B20FFF743FE3220FFF7E8FD00210F2079
:10406800FFF73CFE3220FFF7E1FD41200021FFF77A
:1040780035FE3220FFF7DAFD42200021FFF72EFE41
:104088003220FFF7D3FD00214820FFF727FE40F23A
:104098003F143220FFF7CAFD21464920FFF71EFED4
:1040A8003220FFF7C3FD00214A20FFF717FE322018
:1040B800FFF7BCFD00214B20FFF710FE3220FFF771
:1040C800B5FD44204FF46F41FFF708FE3220FFF79B
:1040D800ADFD00214520FFF701FE3220FFF7A6FDC8
:1040E80021464620FFF7FAFD3220FFF79FFD3020DA
:1040F80040F20771FFF7F2FD3220FFF797FD3120FC
:104108004FF40171FFF7EAFD3220FFF78FFD3220EF
:104118004FF40171FFF7E2FD40F202543220FFF73D
:1041280085FD21463320FFF7D9FD3220FFF77EFDBC
:10413800342040F20751FFF7D1FD3220FFF776FD1A
:1041480035204FF40171FFF7C9FD3220FFF76EFDEE
:1041580036204FF40171FFF7C1FD3220FFF766FDED
:1041680021463720FFF7BAFDA4F500743220FFF787
:104178005DFD21463A20FFF7B1FD3220FFF756FDDD
:104188002F2041F2BE21FFF7A9FD3220FFF74EFD97
:1041980021463B20FFF7A2FD3220FFF747FD002113
:1041A8002320FFF79BFD3220FFF740FD002124204C
:1041B800FFF794FD3220FFF739FD25204FF4004129
:1041C800FFF78CFD3220FFF731FD00214F20FFF76C
:1041D80085FD3220FFF72AFD4E200021FFF77EFDE6
:1041E8003220BDE8104021E508B5124B93F829208C
:1041F8002AB11148114A124B40F242210FE0012224
:1042080083F82920222166234FF0C042013BDBB20C
:10421800118033B90848094A0A4B40F25B21FFF77D
:10422800C9FC108880B22228F0D1024B002283F802
:10423800292008BD540C00206C9A05085D58040814
:10424800B89A05088E99050810B5224B49F2203214
:10425800032823D8DFE800F0021A0B111C8846F661
:10426800280041F22801944218BF01461AE01C8830
:1042780041F2080046F6080104E01C8841F23000CB
:1042880046F63001944208BF01460BE0188846F60E
:104298002001904208BF4FF4815103E00E4840F2DC
:1042A800792113E01B8848F68912934205D049F218
:1042B8002032934207D1032000E01120FFF70EFDC2
:1042C800BDE8104090E7044840F28521034A044BBA
:1042D800FFF770FC320000206C9A05087258040839
:1042E8008E990508014B18800A209FE4000002609F
:1042F8004FF0C043188003F500331A881A881888CD
:1043080080B270472DE9F041022098B001210024C5
:1043180009F0E2F8012502268C488DF85C5016A9B0
:104328008DF85E408DF85F4016968DF85D6008F058
:104338002BFD1820294609F0CFF82846294609F010
:10434800E3F821460C22824808F09EFD29460C22FB
:104358007F4808F099FD04210C227D4808F094FD5F
:1043680005210C227A4808F08FFD07210C22784895
:1043780008F08AFD08210C22754808F085FD0921FE
:104388000C22734808F080FD0A2171480C2208F0BD
:104398007BFD0B216E480C2208F076FD0E210C22C5
:1043A8006B4808F071FD0F210C22694808F06CFD7C
:1043B80007210C22674808F067FD08210C22654890
:1043C80008F062FD09210C22624808F05DFD0A210F
:1043D8000C22604808F058FD0B210C225D4808F0BB
:1043E80053FD0C210A465B4808F04EFD0D210C22B6
:1043F800584808F049FD0E210C22564808F044FDA3
:104408000C2254480F2108F03FFD03274CF6B373E4
:104418004F48169316A98DF85D708DF85E408DF89B
:104428005F408DF85C6008F0AFFC4FF6807316A90A
:10443800484816938DF85D708DF85E408DF85F40A2
:104448008DF85C6008F0A0FC40F6B830FFF7EEFB92
:10445800224631463D4808F00CFD44F6FF70FFF750
:10446800E5FB2A463146394808F003FD40F6B830E6
:10447800FFF7DCFB4FF48053102709930DF13C083C
:104488004FF4002368460F941094129413951494D3
:104498001594009401940294049406940794089443
:1044A8000A9405940B940C9311960397CDF83480D5
:1044B80008F0E3F9042368461193109412941395B5
:1044C800149415940F96CDF8388008F0D6F929463B
:1044D800204608F052FA40F6B830FFF7A7FB20460E
:1044E800FFF706FF04461C491C4D3846224607F0D4
:1044F80059FC48F689139C421AD049F220339C4251
:104508000DD041F289239C4212D03846144907F055
:1045180049FC1448144A154BA621FFF74BFB3846B3
:104528001349224607F03EFC2C80FFF70BFC0AE0FB
:10453800FFF7FFFC48F689122A8010200D4941F246
:10454800892307F02FFC18B0BDE8F0810004024071
:10455800000C024000100240CD9A050832000020ED
:10456800E49A05086C9A05088A5804088E99050883
:104578001B9B0508509B05084FF0C04322221A8058
:1045880003F5003382B01A8892B2ADF806201B8872
:104598009BB2ADF80630BDF8060080B202B0704795
:1045A800134B1B8848F68912934210B504460BD06A
:1045B80049F22032934213D1C1F1EF01202089B290
:1045C800FFF78CFB212006E0C1F1EF014E2089B2F4
:1045D800FFF784FB4F202146BDE81040FFF77EBB64
:1045E8000448054A054B40F2F321FFF7E3FA00BF00
:1045F800320000206C9A0508935804088E99050823
:104608002DE9F0410D46C5F1F008411E5E18C2EBD8
:104618000802C5F1EF039BB292B2B6B29A422CBF20
:10462800904698469A4234BF11461946864234BF8E
:104638003746074640F23F13864238BF06469E4239
:1046480028BF1E461B4B1B8848F68912B8F1EF0F8E
:1046580028BF4FF0EF089342044610D049F22032A9
:1046680093421FD15020FFF739FB51204146FFF7F5
:1046780035FB52203946FFF731FB53200AE041EA67
:10468800082189B24420FFF729FB45203946FFF766
:1046980025FB46203146FFF721FB20462946BDE889
:1046A800F0417DE70448054A054B40F2DD21FFF75C
:1046B80081FA00BF320000206C9A0508A15804084E
:1046C8008E99050800200146F0224FF4A07397E761
:1046D800072040F27311FFF701BB07200021FFF705
:1046E800FDBA10B51446FFF75BFFFFF77DFD2046C6
:1046F800BDE81040F6E508B5FFF752FF4FF0C0439C
:1047080022221A8003F500331A88188880B208BD5F
:10471800F8B580B202FB03F589B292B29BB2069C4F
:104728009DF81C60FFF76CFF0020FFF78DFD002748
:1047380009E034F8020B1EB1030A43EA002080B2F4
:10474800FFF7D0FD0137AF42F3DBBDE8F840B9E72A
:104758002DE9F74F16469DF834200C9F0192054627
:10476800B2B280B20C46984689B29BB2FFF748FFB6
:104778004FF0000B0020FFF767FDDA463DE0002D03
:1047880030DB09EB050340F23F1293422ADC002C90
:1047980028DB0BEB0403EF2B24DC19F00F0F04D1FB
:1047A800B9F1000FC8BF0AF1010A174B09EA030360
:1047B800002B03DA013B63F00F030133019A0AB1BE
:1047C800C3F10F03012202FA03F337F81A2013404A
:1047D8001BB213B10D4B588D01E00D4A508880B2C1
:1047E800FFF780FD09F1010901E04FF00009C1451B
:1047F800C5DB0AF1010A0BF1010BB345F5DB03B088
:10480800BDE8F04F5EE700BF0F000080540C0020A9
:10481800320000202DE9F04F85B004469DF83C0099
:10482800029200278A46039088463E4640F23F1C83
:104838009B463AE0002C2FDBE1452DDCBAF1000F56
:104848002ADBB8F1EF0F27DC2A0702D1002DC8BFF9
:1048580001361B492940002903DA013961F00F01AB
:104868000131039A0AB1C1F10F010E9830F81620F0
:1048780003FA01F10A4012B272B112494A8D01934A
:1048880092B21FFA89F01FFA88F1CDF800C0FFF73D
:1048980028FFDDF800C0019B013509F101095D45DC
:1048A800C8DB0136013708F10108029A974203DA9A
:1048B800A14600250123F2E705B0BDE8F08F00BF4F
:1048C8000F000080540C002082B0044BADF80600A5
:1048D800BDF8062092B25A8502B07047540C0020E9
:1048E80082B0044BADF80600BDF8062092B25A809B
:1048F80002B070473200002070B50646FFF7E2FEAE
:104908000020FFF7A1FCF02409E0013D3046ADB2DC
:10491800FFF7E8FC002DF8D1013CA4B214B14FF424
:10492800A075F2E770BD70B51D461446FFF738FE56
:104938002846FFF789FC0025054E05E0708D80B2FA
:10494800FFF7D0FC0135ADB2A542F7D170BD00BF6D
:10495800540C00202DE9F0410C4616461F461A4615
:1049680000230546FFF7DFFF611E711828463A4607
:10497800002389B2FFF7D7FF284621463246012394
:10498800FFF7D1FF013D7F19B8B221463246012316
:10499800BDE8F041C7E770B580B202FB03F489B205
:1049A80092B29BB2FFF72CFE0020FFF74DFC0025CA
:1049B800054E04E0708D80B2FFF794FC0135A542E6
:1049C800F8DBBDE870407DE6540C0020F8B5561AB7
:1049D8000C46013189B21F460546FFF7E1FD01206B
:1049E800FFF732FC4FF0C04322221A800E4A0F49CB
:1049F8001388B6B2002304E01088013321F8020BB3
:104A08009BB2B342F8D121462846FFF7C9FD0120E1
:104A1800FFF71AFC002404E03846FFF763FC013472
:104A2800A4B2B442F8D1F8BD00000260D643002019
:104A380070B5194B194AD98D92F9004064180025B0
:104A4800A4B2AC4208BF0124C62C28BFC6240F2636
:104A580015704FF6FF7288B09E85DC855A8519203F
:104A68000A222B462146FFF75EFF21463046FFF714
:104A780042FE224603460A4968460EF0DFFD6A46B2
:104A880004A808490EF0DAFD3220D22104AA2B46E8
:104A980000F0ECF908B070BD540C00208C2B0020FD
:104AA8008F9B0508979B05082DE9F0431F2093B0BD
:104AB800FFF722FF4FF47840FFF71EFF4FF6E0752F
:104AC8004FF4FC60FFF718FF2846FFF715FF00209A
:104AD800494CFFF711FF00200146642203464FF6B8
:104AE800FF79A4F82A90FFF71EFF00200A2164220C
:104AF8000346FFF718FF00200146642201234FF404
:104B080078476585FFF70FFF7720EF21C82200233C
:104B18004FF4FC666785FFF706FFBD2132220123AB
:104B280040F23F106685FFF7FEFEA02032220023E8
:104B380078216785FFF7F7FEA0207821322201232C
:104B48004FF01F086685FFF7EEFEA020782132227D
:104B58000223A4F82A80FFF7E6FEA020782132225B
:104B680003236585FFF7DFFE244B2549A3F8028060
:104B780002AD3C2228460EF09FFCEB20C321052203
:104B8800302300950025A4F82A900195FFF7E0FD51
:104B980032210A2096220B466785FFF7DBFE322179
:104BA8003C2096220B466685FFF7D4FE32210B4641
:104BB80096226E20A4F82A80FFF7CCFEFFF78DFD21
:104BC800FFF786FD3220FFF769F82846FFF766F8F9
:104BD8006420FFF763F80B4B03F110028DE8240003
:104BE80028465A681B682946FFF792FD1195119BC4
:104BF80001331193FBE700BF540C00203200002062
:104C0800B6580408F87C010800487047A41500202D
:104C180082B0064BADF80600BDF8062092B21A80A5
:104C2800188880B202B0FFF74FBE00BFA015002061
:104C3800014B188880B27047A015002082B0064B3F
:104C4800ADF80600BDF8062092B21A80188880B226
:104C580002B0FFF745BE00BFA2150020014B18881F
:104C680080B27047A2150020FFF746BEFFF7C8BC08
:104C7800FFF759BEFFF76EBEFFF78DBE2DE9F04F67
:104C88004FEA420800253D4C85B082468B46C8F164
:104C9800030817462E461FFA87F909EB0B0C2288E2
:104CA80005EB0A031FFA8CFC9BB26146184692B2C8
:104CB800CDF804C00293FFF714FDC9EB0B0292B2C2
:104CC8000392029B22880399184692B2FFF709FDC6
:104CD800DDF804C02288C5EB0A039BB2614618467A
:104CE80092B20293FFF7FDFC029B228803991846B3
:104CF80092B2FFF7F6FC05EB0B0292B2039209EBB6
:104D08000A03228803999BB2184692B20293FFF7CE
:104D1800E8FC029B2288C5EB0B0C1FFA8CFC18469A
:104D2800614692B2CDF804C0C9EB0A09FFF7D9FC75
:104D3800228803991FFA89F992B24846FFF7D1FCF5
:104D48002288DDF804C092B248466146FFF7C9FCE4
:104D5800B8F1000F04DA08EB860808F1060805E048
:104D6800F31B08F10A0808EB8308013F01360135F7
:104D7800BE42ADB28FD905B0BDE8F08FA0150020B6
:104D880008B9FFF7AABC012801D1FFF7A1BC7047F9
:104D9800704700200146F0224FF4A073FFF730BCA3
:104DA800704708B505280CD8DFE800F01214030591
:104DB8000709094808BD094808BD094808BD094848
:104DC80008BD0948094A0A4B40F24111FEF7F2FEB4
:104DD800084808BD084808BD200000201000002031
:104DE80008000020000000209C9B0508F2580408D9
:104DF8008E990508280000201800002010B50446E8
:104E0800FFF7CFFF014B18601C7110BD3800002060
:104E1800014B1879704700BF3800002008B5FFF72C
:104E2800C0FF808808BD08B5FFF7BBFFC08808BD74
:104E3800F7B51F460B4B0C4E1D681446EA882B68C5
:104E4800203C5443A4B2AE1B03EB440418BF012614
:104E5800AB888DE8500017B1FFF7DCFC01E0FFF7E5
:104E680077FCFEBD38000020280000202DE9F04125
:104E78000F46984615460446084E08E02046434625
:104E88003946FFF7D5FF33689B88E418A4B215F8B4
:104E9800012B002AF2D1BDE8F08100BF38000020C4
:104EA80010B5044608462146BDE81040DEE7094B28
:104EB80070B5044618790E461546FFF7B4FFC6F1DB
:104EC800F001091A89B220462A460023BDE870403D
:104ED800CCE700BF38000020704700BF044B1A68B9
:104EE8000AB9044A1A601A68101818601046704700
:104EF800840C0020704F00204FF0FF30704708B539
:104F08000248034A034B3721FEF754FEBB9B0508B2
:104F1800085904088E9905080120704710B5044601
:104F28000A48022108F05EFD0028F9D0074821460A
:104F380008F021FD0548012108F054FD0028F9D0AA
:104F48000248BDE8104008F013BD00BF003800401B
:104F580010B51948022108F045FD0028F9D0164877
:104F6800002108F008FD1448012108F03BFD002845
:104F7800F9D0114808F0FCFC0402A4B2002301E0B7
:104F880001339BB2002BFBD00B48022108F02AFD0D
:104F98000028F9D00848002108F0EDFC0648012156
:104FA80008F020FD0028F9D0034808F0E1FC204370
:104FB800C0F3CB0010BD00BF003800402DE9F0471A
:104FC8008AB00AAF0A20012108F086FA4FF460433C
:104FD80047F8143D474EDFF824A1012400254FF07F
:104FE8000208304639468DF81A508DF818808DF829
:104FF80019808DF81B4007F0C7FE30460D210522A9
:1050080007F042FF30460E21052207F03DFF05223A
:1050180030460F2107F038FF21464FF4804008F052
:105028007FFA504608F05AFB4FF48273ADF802300D
:105038004FF40073ADF80A303823ADF80C30504601
:1050480007236946ADF81030ADF80050ADF80450AC
:10505800ADF80650ADF80850ADF80E5008F070FBEA
:105068005046214608F007FCA9468DF81A503046EC
:105078004FF48055394605958DF818408DF81980FC
:105088008DF81B4007F080FE3046294607F0EDFEFC
:105098004025394618488DF818908DF819808DF8F4
:1050A8001A908DF81B40059507F06EFE21464FF4C7
:1050B800804008F041FA0621032008F0CBFC0C23BD
:1050C80007A88DF8213007958DF820908DF822409B
:1050D80007F04EFB17238DF8243009A80F238DF80D
:1050E80025308DF826308DF8274002F041FB0AB0B4
:1050F800BDE8F08700040240000C02400038004080
:10510800014B1878704700BF880C0020024B5A8862
:105118009B8802800B807047880C0020014B00227E
:105128001A707047880C0020F0B593B068460021CB
:1051380048220EF003FA6D46002464484FF480516B
:1051480007F095FE002301E001339BB2002BFBD052
:105158009020FFF7E3FE002301E001339BB2002B10
:10516800FBD0FFF7F5FE4FF480510746574807F08C
:105178007CFE002301E001339BB2002BFBD0534897
:105188004FF4805107F073FE002301E001339BB216
:10519800002BFBD0D020FFF7C1FE002301E0013334
:1051A8009BB2002BFBD0FFF7D3FE4FF4805106468D
:1051B800464807F05AFE45F8047B01342E624448FD
:1051C8004021E4B207F03FFE10B9092CB5D101E047
:1051D800092C78D19DE80C00D218029B03980699F7
:1051E800D218049BC018059BC018079BCB180899B8
:1051F800032490FBF4F092FBF4F25B1893FBF4F3B6
:10520800151AC11A9C1A002DB8BF6D420029B8BFE3
:105218004942002CB8BF6442502D03DD502909DDF6
:10522800502C50DC8D4205DAAC424FF0020405DB0D
:10523800111806E08C424FF0020401DAD11800E0A0
:10524800C1180A9B099A0C980F9DD2180B9BD2186B
:105258000D9BC0180E9BC018109BEB18119D91FB5D
:10526800F4F1032492FBF4F290FBF4F05B1993FB46
:10527800F4F3161AC41A9D1A002EB8BF7642002CF1
:10528800B8BF6442002DB8BF6D42502E89B203DD0D
:10529800502C09DD502D16DCA64205DAB5424FF038
:1052A800020405DB131806E0A5424FF0020401DAF8
:1052B800D31800E0C318074A93FBF4F39BB293801A
:1052C80001235180137013B0F0BD00BF00040240E9
:1052D800000C0240880C0020FFF712BFF7B5054606
:1052E8000C4601A80DF10601FFF710FF1B4BBDF896
:1052F8000660BDF8040093E80600724301FB002233
:1053080099685218164992FBF1F207EE102AF8EE46
:10531800C77A40F23F17FCEEE77A17EE902A92B26E
:10532800B2F5207F28BF3A462A801D69DA685B6992
:105338006E4302FB0060C01890FBF1F107EE101AF3
:10534800F8EEC77AFCEEE77A17EE903A9BB2B3F51F
:10535800F07F28BFEF232380FEBD00BF900C002004
:1053680040420F00FFF7DABE014B187E704700BFBE
:10537800900C0020FFF7CABE042808B505D90748D5
:10538800074A084B7D21FEF715FC054B03EB80000F
:10539800038B0B80438B138008BD00BFDC9B050883
:1053A8000E590408FA9B050808B5082001F08CF985
:1053B80042F69643C31A584240EB030008BD10B5A5
:1053C8000A2001F0A9F90C4C20600E2001F0A4F984
:1053D8006060122001F0A0F9A060162001F09CF98D
:1053E800E0601A2001F098F920611E2001F094F97C
:1053F80001236061237610BD900C002010B5FFF7E3
:10540800DDFD01F02BFA044601F034FA07490346A2
:105418002246202006F0C6FCFFF7C6FF28B101F09F
:1054280037FA10B9BDE81040C9E710BD369C050829
:1054380010B5104C0A20216801F055F961680E205A
:1054480001F051F9A168122001F04DF9E168162028
:1054580001F049F921691A2001F045F961691E2016
:1054680001F041F9082042F69641BDE8104001F0EC
:105478001DB900BF900C00202DE9F04F0346A7B0DE
:10548800B0F800C01C898688DF885D89CDF810C017
:10549800B249B0F802C0B3F80C90B3F80E80CDF85A
:1054A80024C00FFA84FB30B201220FFA87FE0BEBFF
:1054B800000C0A7629B20FFA89FACDF888C001EBF8
:1054C8000E0C0FFA88F2CDF890C00AEB0B0CCDF851
:1054D80030C002EB010CCDF858C0B3F810C05B8A9D
:1054E800CDF800C00FFA8CFC06910CEB00010A9174
:1054F80002930CEB0A011BB2239103EB0E010E91F0
:1055080099182591049900FA81F058445044604450
:10551800DDF824C006990EFA8CFEDDF810C01FFADB
:1055280080FB1CFB0CF08E4416FB0600964414FB13
:105538000400009A19FB09009E4412FB02001FFA9E
:105548008EFA09F059FBDDF824C0029ACDE9120160
:105558001CFB0CF017FB070015FB050018FB0800E7
:1055680012FB020009F048FBDDF824C0029ACDE9DD
:10557800140104991CFB01F317FB063615FB04669E
:10558800009B18FB096612FB036009F035FBDDE997
:105598001423CDE90001DDE9120109F0A3FB04465B
:1055A8000D46DDE9000102460B4609F09BFB024669
:1055B8000B462046294609F0E1F9CDE9180158467D
:1055C80009F02AFBCDE91001DDE91023DDE900012E
:1055D80009F088FBCDE90601504609F01DFB80461D
:1055E80089464246DDE912014B4609F07BFBDDE9BD
:1055F8001023CDE91C01DDE9140109F073FB002239
:1056080006460F46564BDDE9180109F06BFB42468A
:1056180004460D464B46DDE9060109F063FB0246E8
:105628000B4609F0ADF902460B462046294609F01B
:10563800A7F9424604460D464B46DDE91C0109F030
:1056480051FB02460B462046294609F097F9DDE949
:10565800102304460D463046394609F043FB0246FE
:105668000B462046294609F089F9DDF828C0CDE91E
:1056780002014FEA8C10DDF830C000EB0C20DDF899
:1056880010C0A0241CFB040009F0B6FADDF838C0ED
:10569800CDE90A014FEA8C10DDF858C000EB0C2068
:1056A800DDF824C01CFB040009F0A6FACDE90C01C2
:1056B800504609F0A1FADDE91023CDE91601DDE92C
:1056C8000C0109F00FFB4246CDE91E014B46DDE90E
:1056D8000A0109F007FB4246CDE920014B46DDE906
:1056E800000109F0FFFA32463B4609F047F9CDE9D7
:1056F8000E01584609F080FADDE91C23CDE91A01AC
:10570800DDE9060109F03AF9DDF88CC0C024CDE9DD
:10571800060104FB0CF0DDF888C0302505FB0C0001
:10572800DDF810C078261CFB060009F065FADDF8E4
:1057380094C0824604FB0CF0DDF890C005FB0C0019
:10574800DDF824C01CFB06008B4609F055FADDE99C
:10575800102306460F4609F0C5FA03E0900C002016
:10576800000014404246CDE904014B4650465946D4
:1057780009F0B8FADDE9142380468946DDE90A0113
:1057880009F0B0FADDE9002304460D46DDE90C0115
:1057980009F0A8FA02460B462046294609F0EEF819
:1057A8000022A14B09F09EFADDE9202304460D46AC
:1057B800DDE91E0109F0E2F802460B46DDE91601B3
:1057C80009F090FA02460B462046294609F0D8F817
:1057D800002204460D46954BDDE90E0109F082FAD8
:1057E80002460B462046294609F0CAF8DDE902239D
:1057F80009F0A2FB88A3D3E9002309F073FA09F0A2
:105808000BFD8B490860DDE91223DDE90C0109F085
:1058180069FADDE9002304460D46DDE90A0109F0CD
:1058280061FA02460B462046294609F0A7F80022ED
:105838007D4B09F057FADDE91E2304460D46DDE9E4
:10584800200109F09BF802460B46DDE91A0109F030
:1058580049FA02460B462046294609F091F80022EB
:1058680004460D46714BDDE9060109F03BFA024694
:105878000B462046294609F083F8DDE9022309F0A2
:105888005BFB65A3D3E9002309F02CFA09F0C4FCFB
:10589800674A5060DDE90E23DDE90A0109F022FAC2
:1058A800DDE9062304460D46DDE90C0109F01AFA84
:1058B80002460B462046294609F062F800220446B3
:1058C8000D465A4BDDE9180109F00CFA02460B4661
:1058D8002046294609F054F8DDE9022309F02CFB9B
:1058E8004DA3D3E9002309F0FDF909F095FC504BCD
:1058F80059469860DDE91423504609F0F3F9DDE9CB
:10590800002304460D463046394609F0EBF90246B5
:105918000B462046294609F031F80022424B09F08F
:10592800E1F9424604460D464B46DDE9040109F01B
:1059380025F802460B46DDE9160109F0D3F90246BF
:105948000B462046294609F01BF835A3D3E9002366
:1059580004460D46DDE90E0109F0C4F902460B467E
:105968002046294609F00CF8DDE9022309F0E4FA9B
:1059780029A3D3E9002309F0B5F909F04DFCDFF8B4
:10598800B0C0DDE91223CCF80C003946304609F0E6
:10599800A9F9DDE9002304460D465046594609F0A9
:1059A800A1F902460B462046294608F0E7FF0022E7
:1059B8001D4B09F097F9DDE9042304460D464046DE
:1059C800494608F0DBFF02460B46DDE91A0109F0FB
:1059D80089F902460B462046294608F0D1FF10A354
:1059E800D3E9002304460D46DDE9060109F07AF9FA
:1059F80002460B462046294608F0C2FFDDE902238D
:105A080009F09AFA04A3D3E9002309F06BF909F025
:105A180003FC074908610DE00000000080842E4166
:105A28000000000000C082400000144000008940CF
:105A3800900C0020DDE90E235046594609F052F932
:105A4800DDE9062304460D463046394609F04AF991
:105A580002460B462046294608F092FF11A3D3E9D7
:105A6800002304460D46DDE9180109F03BF902461A
:105A78000B462046294608F083FFDDE9022309F09A
:105A88005BFA0AA3D3E9002309F02CF909F0C4FB57
:105A9800034A506127B0BDE8F04FC9E4AFF3008076
:105AA800900C00200000000000C0824000000000B0
:105AB80080842E41AFF30080064B074A5968116075
:105AC8001969064A1160D969054A11609A6A054B35
:105AD8001A60704740000020583C002074420020A3
:105AE8004C420020083C0020014B1878704700BF4A
:105AF800AC0C0020032808B505D90548054A064B13
:105B08007121FEF757F80C235843044B185808BD69
:105B1800719C05083A5904088B9C05084000002030
:105B2800032808B505D90648064A074B7621FEF72B
:105B380041F8064B0C2202FB0030406808BD00BF4C
:105B4800719C05084A5904088B9C050840000020F0
:105B5800034B044A1B780C2101FB03239868704708
:105B6800AC0C002040000020034B044A1B780C209A
:105B780000FB032399607047AC0C00204000002014
:105B8800144B1B78012B10B5134B144C0ED119680C
:105B9800C82000F0A8FD2168CC2000F0A4FD104B1F
:105BA800D020196800F09FFDD4200DE01968D82096
:105BB80000F099FD2168DC2000F095FD084BE020FD
:105BC800196800F090FDE420064B1968BDE8104004
:105BD80000F089BD280E0020583C002074420020A7
:105BE8004C420020083C0020144B1B78012B10B5B8
:105BF800134C0FD1C82000F08FFD2060CC2000F09E
:105C08008BFD104B1860D02000F086FD0E4B1860FD
:105C1800D4200EE0D82000F07FFD2060DC2000F0CA
:105C28007BFD084B1860E02000F076FD064B1860FD
:105C3800E42000F071FD054B186010BD280E00200F
:105C4800583C0020744200204C420020083C0020B0
:105C580008B502F0C3FA10B1BDE80840C4E7BDE8D2
:105C6800084029E70148FBF7BABF00BF8C130020A2
:105C78000148FBF7B4BF00BF8C1300200148FBF7B5
:105C8800AEBF00BF8C1300200148FBF7A8BF00BFC0
:105C98008C130020032808B505D91448144A154B5D
:105CA8004E21FDF787FF144B1870144B022818700B
:105CB800134B0FD0032813D0012805D0114A1268BE
:105CC8001A60BDE80840CDE70F4A12681A60BDE8BF
:105CD8000840CDE70D4A12681A60BDE80840CDE7D4
:105CE8000B4A12681A60BDE80840CDE7719C0508A8
:105CF8005B590408B59C0508AC0C00204E3C0020FC
:105D080098010020900100208C01002088010020CB
:105D180084010020064B07495960C02100221972EE
:105D28001E211A70D9601A745A611A76DA6170479E
:105D3800D015002040787D0110B50321FF22C02036
:105D480001F072F81F4C102120608022C02001F061
:105D58006BF8112120608022C02001F065F8122123
:105D680020608022C02001F05FF81321206080228B
:105D7800C02001F059F8142120608022C02001F0D1
:105D880053F8152120608022C02001F04DF88022B0
:105D980020601621C02001F047F82060C02017219C
:105DA800802201F041F82060074CC020227AB721F8
:105DB80001F03AF80023237463612376E361012339
:105DC800237010BD2C3C0020D015002038B5C02011
:105DD8000321FF2201F028F80B4D00242B19615DE7
:105DE8005A78C020023401F01FF8C82CF6D1B1212E
:105DF800AC22C02001F018F8C0200321002201F0D5
:105E080013F8002038BD00BF6F5904082DE9F34787
:105E180006460F4692461D461AB90C1FE4019146E4
:105E280035E005EE902A06EE903AB8EE657AF8EE7F
:105E3800667AFC01C7EE277AA4F500749FED5C7AB8
:105E480067EE877A17EE900A08F0F8FE41EC100B1F
:105E58000AF016FF59EC108B4946404609F004FA3F
:105E680024184FEACA1008F0C7FECDE900012846F9
:105E780008F0C2FE4B46424608F034FF02460B4685
:105E8800DDE9000108F07AFD09F0EEF98146002EFF
:105E980014BF4FF022084FF01A08C5F307224146F5
:105EA800C02000F0C1FF08F10101EAB2C02000F0F3
:105EB800BBFFC4F3014208F10201C02000F0B4FFA7
:105EC800C4F3072208F10301C02000F0ADFFE2B2DD
:105ED80008F10401C02000F0A7FFC9F3034305F44B
:105EE800702243EA123208F10501C02000F09CFF3D
:105EF80008F10601C9F30722C02000F095FF08F158
:105F080007015FFA89F2C02000F08EFFC020B1219E
:105F1800A02200F089FF07EE107A264CF8EEC77A27
:105F28000EBBD4ED015A06EE90AAB8EE657A05EEDE
:105F3800905AB8EE666AF8EE656A0123C6EE266ADC
:105F4800237477EEA67A67EE277A17EE900A08F0A0
:105F580075FE41EC100B0AF093FE51EC100B09F0A2
:105F680083F9606120E005EE90AAD4ED016AB8EEED
:105F7800656A05EE905AB8EE667AF8EE656A01230E
:105F8800C6EE266A237677EEA67A67EE277A17EEAC
:105F9800900A08F053FE41EC100B0AF071FE51EC28
:105FA800100B09F061F9E0610020BDE8FC8700BF33
:105FB80000000043D01500200022012326E7012815
:105FC80038B50D4604D002280CBF3C242C2400E030
:105FD80034242146C02000F0A1FF05F0070200F09C
:105FE8000F0040EA02122146C020BDE8384000F008
:105FF8001BBF2DE9F3470A9C1D4607468A461646ED
:10600800524B01E06D0864089C42FBD82DB906F19B
:106018000076043EF601A94634E006EE905AB8EE42
:10602800667A06EE904AF8EE667AF601C7EE277AA7
:10603800A6F500769FED467A67EE877A17EE900A06
:1060480008F0FCFD41EC100B0AF01AFE59EC108B1D
:106058004946404609F008F93618E80108F0CCFD31
:10606800CDE90001204608F0C7FD4B46424608F03E
:1060780039FE02460B46DDE9000108F07FFC09F015
:10608800F3F88146022F9BBF324BDB194FF0000813
:1060980093F8C880C4F307224146C02000F0C4FE2C
:1060A80008F10101E2B2C9B2C02000F0BDFE08F15A
:1060B8000201C9B2C6F30142C02000F0B5FE08F1E2
:1060C8000301C9B2C6F30722C02000F0ADFE08F1F3
:1060D8000401C9B2F2B2C02000F0A6FE04F4702494
:1060E800C9F3034308F1050143EA1432C9B2C020D9
:1060F80000F09AFE08F10601C9B2C9F30722C020D0
:1061080008F1070800F090FE5FFA89F25FFA88F15B
:10611800C02000F089FEBAF1010F0CBF2F220F2218
:106128000DB942F04002012F06D002D3022F0AD146
:1061380005E0C020102104E0C020112101E0C020AA
:10614800122100F071FE0020BDE8FC87FFFF0F0060
:10615800000000436F59040807B50123009300238A
:10616800FFF747FF0EBD00280CBFFF22002208B52D
:10617800C020032100F058FE002008BD08B5C0204B
:10618800B121AC2200F050FE002008BD08B5042063
:10619800012107F0A1F94FF480700121BDE8084002
:1061A80007F0CAB907B50223009303238DF804301A
:1061B8000348002369468DF8073006F0E5FD0EBD5B
:1061C8000008024030B5124D8BB0002406A8069492
:1061D80007940894099405F0A5FF00948DF80440ED
:1061E8008DF80540029403940494284601246946D6
:1061F8008DF8144005F067FF28460B212246062338
:1062080005F0DCFF2846214605F0A6FF0BB030BD9F
:106218000020014010B5002104460122302000F082
:1062280003FEC0B9012001F01FF8002CB8BF4034AC
:10623800E4B210212246302000F0F6FD012001F0E2
:1062480013F830201121224600F0EEFD0120BDE8B0
:10625800104001F009B810BD10B500210446012214
:10626800302000F0E1FDC0B9012000F0FDFF002C56
:10627800B8BF4034E4B212212246302000F0D4FDE9
:10628800012000F0F1FF30201321224600F0CCFD60
:106298000120BDE8104000F0E7BF10BD38B501226D
:1062A80005460C463020002100F0BEFDF0B9012063
:1062B80000F0DAFF25EAE5725F2AA8BF5F223B21DA
:1062C800D2B2302000F0B0FD012000F0CDFF24EA6A
:1062D800E4725F2AA8BF5F22D2B230203C2100F0CE
:1062E800A3FD0120BDE8384000F0BEBF38BD30280E
:1062F80010B504460ADC10F17F0F02DB002802DB30
:1063080005E06FF07E0404F5807400E0302400217D
:1063180030200A4600F088FDA8B90120E4B200F058
:10632800A3FF41212246302000F07EFD012000F02D
:106338009BFF30204221224600F076FD0120BDE877
:10634800104000F091BF10BD282810B5044609DCA4
:1063580010F1180F02DB002802DB04E06FF01704CD
:106368007F3400E02824002130200A4600F05CFD3C
:10637800A8B90120E4B200F077FF5321224630206B
:1063880000F052FD012000F06FFF3020542122461A
:1063980000F04AFD0120BDE8104000F065BF10BDC7
:1063A80008B530200021012200F03EFD60B901202F
:1063B80000F05AFF30203321402200F035FD012043
:1063C800BDE8084000F050BF08BD10B530200021DE
:1063D800012200F029FD044660B9012000F044FFC5
:1063E80030203321224600F01FFD0120BDE8104077
:1063F80000F03ABF10BD10B530200021012200F096
:1064080013FD0446A0B9012000F02EFF34212246D6
:10641800302000F009FD012000F026FF3020372150
:10642800224600F001FD0120BDE8104000F01CBF2D
:1064380010BD4020EEE640200EE708B500210122FD
:10644800302000F0F1FC012000F00EFF3020342154
:10645800024600F0E9FC012000F006FF3020372159
:10646800024600F0E1FC0120BDE8084000F0FCBE57
:1064780008B500210122302000F0D6FC012000F0F0
:10648800F3FE302034210C2200F0CEFC0120BDE8C0
:10649800084000F0E9BE0000184B1949D3ED006A26
:1064A80093ED017A00231A469FED166A03E0F0EE99
:1064B800476AB0EE677A505E05EE900AF8EEE57A24
:1064C8000133C7EE867A9BB218B204327F2877EE82
:1064D800E67AECDD27EE077A07EEA77A0A49074A3B
:1064E8000B80BDEEC77A002313605360C2ED027AB9
:1064F80017EE102A054B92001A607047B00C002066
:106508008C2700200000FA45BC3B002058180020CA
:106518002DE9F84F2E4B2F4A19682F4B19B92F49DF
:1065280011602F4A02E02F4911602F4A1A602F4B41
:10653800DFF8BCA0DFF8BC90DFF8BCB000221A80FE
:10654800244A9846176830E007EB84036500B3F9DE
:10655800023007EE103AF8EEC77A013617EE900AC5
:1065680008F06CFB18A3D3E9002308F0BBFB08F084
:1065780053FE29F815002AF8140037F9243007EEDD
:10658800103AF8EEC77A013517EE900A08F056FB74
:106598000DA3D3E9002308F0A5FB08F03DFE2BF876
:1065A800140029F81500A8F80060B8F8006034B2A3
:1065B800FF2CC9DD00F05EF800F06AF801F07CF904
:1065C800BDE8F84F68E700BF9A9999999999E93F0A
:1065D8004C18002040180020781600208E2F00202C
:1065E8008E2B00208E3700208E330020BC3B0020ED
:1065F8008C2300208C2700208C25002010B50B4C04
:10660800204606F00EF80A4B18600A4806F009F80A
:10661800094B1860FFF77CFF084B09490122204607
:106628009A81BDE8104006F07DB800BF10600240B6
:106638004C1800208860024068180020B00C002028
:1066480020800010014B1868704700BF58180020C0
:1066580008B5054B054819880022012309F002FBFB
:10666800034B187008BD00BF700000207423002081
:10667800901E002003480449044A4FF4807309F02F
:1066880069BB00BF740000208C2300207221002009
:1066980003480449044A4FF4807309F05BBB00BF08
:1066A800800000208C250020AC19002038B5054654
:1066B8000C460135C1F3072100F0E4FDA8B2E1B2B0
:1066C80000F0E0FD00B238BD38B5044600F0EEFC3D
:1066D80001340546A0B200F0E9FCEDB2C0B240EAD0
:1066E800052000B238BD37B50B0E8DF804300B0C01
:1066F8008DF805300B0A8DF806308DF80710002448
:1067080000E0284601AB451CE15C013400F0BAFD0D
:10671800042CADB2F5D13EBD37B5002400E02846C3
:10672800451C00F0C3FC01ABADB2E0540134042CAD
:10673800F5D19DF805009DF80430000440EA036097
:106748009DF8073018439DF8063040EA03203EBD07
:1067580038B50446642000F087FD25786068AD00F0
:10676800EDB2257006F075FB237A40FA03F000F0CD
:1067780003000543104B257005F00F055A5D63783B
:10678800D218D2B2D3B20132D2B2022A637001D87F
:106798000022A2705BB2012B03DD0123A37000234A
:1067A800637094F90130013303DAFF23A3700023E7
:1067B800637094F9020038BD3A5A0408F7B504200A
:1067C8000121234F06F088FE02AD01214FF48040DD
:1067D800012406F0B1FE00264FF4B073384669462E
:1067E80045F8083D8DF804608DF8074006F0CCFAAE
:1067F8001020214606F070FE78236946154800935C
:106808008DF804608DF8074006F0BEFA0420214692
:1068180006F062FE21464FF4804006F08DFE1C23F0
:106828003846694600938DF804608DF8074006F0F5
:10683800ABFA0220214606F04FFEB02306488DF839
:10684800046069468DF80740009306F09DFAFEBD86
:10685800000802400010024000040240802108B5F0
:10686800034806F0F0FAD0F1010038BF002008BD57
:106878000004024008B54FF48071044806F0E3FABA
:10688800D0F1010038BF002008BD00BF0008024059
:1068980008B5FFF7E3FF08B1FFF7ECFFC0B208BD8A
:1068A80010B5642000F0E0FC0F48FFF751FF0446E4
:1068B80010B90E4B187009E0FFF7DCFF30B9002C57
:1068C8000A4B01DD012200E0FF221A700848FFF799
:1068D8003FFF0028074B01D1187010BD01DD0122D0
:1068E80000E0FF221A7010BDC000002050420020B6
:1068F800CC0000208C2B002007B50220012106F0D7
:10690800EBFD012300938DF8043002238DF8053048
:106918000448002369468DF806308DF8073006F0E4
:1069280033FA0EBD0004024010B5084C01210022C4
:10693800204606F09EFA40F2FF4000F095FC012147
:1069480020460A46BDE8104006F093BA000402400B
:1069580008B5FFF7E9FF00210A46302000F064FA85
:10696800012000F081FC01210A46302000F05CFA89
:10697800012000F079FC00210122302000F054FAB7
:10698800012000F071FC01210822302000F04CFAAF
:10699800012000F069FC02210122302000F044FAB5
:1069A800012000F061FC00210A46302000F03CFA8A
:1069B800012000F059FC1B21CD22302000F034FAD0
:1069C800012000F051FC04210322302000F02CFAB1
:1069D800012000F049FC06210822302000F024FAAA
:1069E800012000F041FC07210A46302000F01CFA83
:1069F800012000F039FC08218022302000F014FA30
:106A0800012000F031FC1E21B022302000F00CFAE9
:106A1800012000F029FC05219122302000F004FA21
:106A2800012000F021FC0D210322302000F0FCF9A8
:106A3800012000F019FC0E210022302000F0F4F9AA
:106A4800012000F011FC14218022302000F0ECF924
:106A5800012000F009FC0B218822302000F0E4F925
:106A6800012000F001FC30200C21822200F0DCF92A
:106A7800012000F0F9FB12218822302000F0D4F91F
:106A8800012000F0F1FB13218C22302000F0CCF91A
:106A9800012000F0E9FB00210122302000F0C4F9B8
:106AA800012000F0E1FB0C210822302000F0BCF9A5
:106AB800012000F0D9FB0D210822302000F0B4F9A4
:106AC800012000F0D1FB0E210822302000F0ACF9A3
:106AD800012000F0C9FB0F210822302000F0A4F9A2
:106AE800012000F0C1FB00210A46302000F09CF98B
:106AF800012000F0B9FB40210222302000F094F977
:106B0800012000F0B1FB00224121302000F08CF977
:106B1800012000F0A9FB30203F21D42200F084F9A5
:106B2800012000F0A1FB00210122302000F07CF9B7
:106B3800012000F099FB10210F22302000F074F999
:106B4800012000F091FB11210F22302000F06CF998
:106B5800012000F089FB12210022302000F064F9A6
:106B6800012000F081FB13210022302000F05CF9A5
:106B7800012000F079FB09213C22302000F054F973
:106B8800012000F071FB00210122302000F04CF9B7
:106B9800012000F069FB30203421024600F044F95E
:106BA800012000F061FB30203721024600F03CF95B
:106BB800012000F059FB36210322302000F034F97F
:106BC800012000F051FB39210322302000F02CF97C
:106BD800012000F049FB3B213C22302000F024F941
:106BE800012000F041FB3C210A46302000F01CF94E
:106BF800012000F039FB00210A46302000F014F98A
:106C0800012000F031FB5121C022302000F00CF9A6
:106C1800012000F029FB30205221002200F004F965
:106C28000120BDE8084000F01FBB00BF2DE9F04F70
:106C3800454E464D93B001214FF4001006F04CFC30
:106C4800304605F0EFFB4FF0C0630293404B0393CF
:106C5800404B002404934FF400794FF400334FF471
:106C680080684FF400674FF4005A4FF4807B304639
:106C780002A90C9301930997CDF8189005940794ED
:106C8800CDF82080CDF828A0CDF82CB00D9405F0D3
:106C980055FC22463046304905F0ABFC3046012110
:106CA80005F0B1FC01210A464FF0402006F082FEB3
:106CB800284605F0B7FB294A019B0392284A0C9302
:106CC80004922846402202A9059209970294CDF819
:106CD80018900794CDF82080CDF828A0CDF82CB0D6
:106CE8000D9405F02BFC224628461E4905F081FC30
:106CF8002846012105F087FC42F210770122022183
:106D0800194806F057FE384600F0AEFA3046012121
:106D180005F04FFC0121284605F04BFC384600F0F1
:106D2800A3FA0B238DF8443011A801238DF84540B0
:106D38008DF846408DF8473000F01AFD384600F0CF
:106D480093FA13B0BDE8F08F1060024088600240EB
:106D58000C4000408E3700208E2F00200C3C004055
:106D68008E3300208E2B0020003C0040024810216A
:106D7800012205F095BC00BF1060024013B5022047
:106D8800012106F0A9FB4FF410730E4C0093022367
:106D98008DF804308DF8053001238DF80630204633
:106DA800002369468DF8073005F0EEFF20460621DE
:106DB800042206F069F820460921042206F064F846
:106DC8001CBD00BF0004024030B5154D85B001213F
:106DD8004FF4001006F0A4FB284606F06BF80023D9
:106DE800ADF804304BF6FF73ADF806303323ADF839
:106DF80008304FF48063ADF80A304FF48043ADF8A3
:106E08000C3004AC074B2846012144F8103D06F02D
:106E1800F3F82846694606F07BF805B030BD00BF98
:106E280000540040801A060073B54FF496130646C6
:106E38000D461446019304E0019B5A1E0192002B53
:106E480057D031484FF4003106F0EEF90028F3D15D
:106E58002D48012106F0DCF84FF48053019304E03B
:106E6800019B5A1E0192002B45D02748274906F05E
:106E7800C6F90028F4D024483146002206F0E0F88C
:106E88004FF48053019304E0019B5A1E0192002B9A
:106E980033D01D481E4906F0B2F90028F4D01A482C
:106EA800294606F050F94FF48053019303E0019B03
:106EB8005A1E01921BB31448164906F0A0F900287F
:106EC800F5D01148214606F03EF94FF49613019388
:106ED80003E0019B5A1E01929BB10B480E4906F034
:106EE800A3F90028F5D00848012106F09DF80020F4
:106EF80008E0012006E0022004E0032002E004206C
:106F080000E005207CBD00BF0054004001000300E4
:106F180082000700800007000400001037B54FF416
:106F2800961304460D46019305E0019B5A1E0192F3
:106F3800002B00F09B8056484FF4003106F074F99E
:106F48000028F2D15248012106F062F84FF480532C
:106F5800019305E0019B5A1E0192002B00F08880E6
:106F68004B484C4906F04BF90028F3D048482146D5
:106F7800002206F065F84FF48053019304E0019B6A
:106F88005A1E0192002B75D04148434906F037F943
:106F98000028F4D03E48294606F0D5F84FF480532F
:106FA800019304E0019B5A1E0192002B64D03848DB
:106FB8003A4906F039F90028F4D03548012106F09D
:106FC80027F84FF48053019304E0019B5A1E019265
:106FD800002B53D02E482F4906F011F90028F4D081
:106FE8002B482146012206F02BF84FF480530193D9
:106FF80004E0019B5A1E0192002B41D0244C2849E1
:10700800204606F011F90028F3D02046002106F0AA
:107018001FF820460121238B06F006F84FF4805311
:10702800019304E0019B5A1E0192002B2AD01848B4
:107038001C4906F0F9F80028F4D0154806F085F840
:107048004FF480530193124A03E0019B591E0191AA
:10705800D3B113889B05F8D4012104460C4805F0E8
:10706800F7FF0B48104906F0F9F80EE001240CE090
:1070780002240AE0032408E0042406E0052404E0CE
:10708800062402E0072400E0082420463EBD00BF95
:1070980000540040010003008200070004000010B3
:1070A80002000010400000100004001013B54FF457
:1070B80096130446019305E0019B5A1E0192002B8A
:1070C80000F0B08061484FF4003106F0ADF80028B8
:1070D800F2D15E48012105F09BFF4FF480530193E4
:1070E80005E0019B5A1E0192002B00F09D80574835
:1070F800574906F084F80028F3D05448A02100220C
:1071080005F09EFF4FF48053019305E0019B5A1E42
:107118000192002B00F08A804C484E4906F06FF827
:107128000028F3D0C4F30521484806F00CF84FF4C2
:107138008053019304E0019B5A1E0192002B77D0E3
:107148004248454906F070F80028F4D0E1B23F48BB
:1071580005F0F9FF4FF48053019304E0019B5A1E98
:107168000192002B66D039483B4906F05DF80028AB
:10717800F4D03648012105F04BFF4FF480530193BA
:1071880004E0019B5A1E0192002B55D02F4830492C
:1071980006F035F80028F4D02C48A121012205F08A
:1071A8004FFF4FF48053019304E0019B5A1E019254
:1071B800002B43D0254C2949204606F035F80028F5
:1071C800F3D02046002105F043FF20460121238B00
:1071D80005F02AFF4FF48053019304E0019B5A1EE7
:1071E8000192002B2CD019481D4906F01DF80028E3
:1071F800F4D0164805F0A9FF4FF480530193134AC1
:1072080003E0019B591E0191E3B113889905F8D455
:10721800012104460D4805F01BFF0C48114906F0F2
:107228001DF810E001240EE002240CE003240AE01B
:10723800042408E0052406E0062404E0072402E00C
:10724800082400E0092420461CBD00BF005400406B
:107258000100030082000700040000100200001073
:10726800400000100004001082B0002304E0019BDD
:1072780001330193009B01330093009B8342F6D3B3
:1072880002B0704737B54FF4805304460D4601935A
:1072980004E0019B5A1E0192002B6ED03D484FF42A
:1072A800003105F0C1FF0028F3D13A48012105F06B
:1072B800AFFE4FF48053019304E0019B5A1E0192E4
:1072C800002B5CD03348344905F099FF0028F4D0EE
:1072D8003048A021002205F0B3FE4FF480530193FB
:1072E80004E0019B5A1E0192002B4AD029482B49E1
:1072F80005F085FF0028F4D0C4F30521254805F0E2
:1073080022FF4FF48053019304E0019B5A1E01921F
:10731800002B38D01F48224905F071FF0028F4D00F
:10732800E1B21C4805F00FFF4FF48053019303E0CE
:10733800019B5A1E019243B31648194905F05FFF95
:107348000028F5D01348294605F0FDFE4FF49613A2
:10735800019303E0019B5A1E0192C3B10D481149E4
:1073680005F062FF0028F5D00A48012105F05CFE0F
:107378000D48FFF779FF00200AE0012008E002200D
:1073880006E0032004E0042002E0052000E00620D7
:107398003EBD00BF0054004001000300820007000A
:1073A8008000070004000010A0860100F7B54FF424
:1073B800805304460D461646019304E0019B5A1E6D
:1073C8000192002B75D041484FF4003105F02CFF95
:1073D8000028F3D13D48012105F01AFE4FF48053EF
:1073E800019304E0019B5A1E0192002B63D0374899
:1073F800374905F004FF0028F4D03448A0210022C2
:1074080005F01EFE4FF48053019304E0019B5A1EC1
:107418000192002B51D02D482E4905F0F0FE00288E
:10742800F4D0C4F30521294805F08DFE4FF48053AC
:10743800019304E0019B5A1E0192002B3FD0234880
:10744800254905F0DCFE0028F4D0E1B21F4805F01C
:107458007AFE4FF48053019304E0019B5A1E019277
:10746800002B2ED019481C4905F0C9FE0028F4D07D
:1074780000244FF4961710E0295D144805F063FEC8
:10748800019703E0019B5A1E0192E3B10F4813498B
:1074980005F0CAFE0028F5D00134E3B2B342EBD3BD
:1074A8000A48012105F0C0FD0D48FFF7DDFE002068
:1074B8000AE0012008E0022006E0032004E004209E
:1074C80002E0052000E00620FEBD00BF0054004099
:1074D800010003008200070080000700040000107C
:1074E800A086010013B50520012105F0F5FF184C11
:1074F8004FF4E053009302238DF804308DF80530E3
:107508002046002369468DF806308DF8073005F0CF
:107518003BFC20460A21062205F0B6FC20460C2139
:10752800062205F0B1FC062220460B21A4F50064D2
:1075380005F0AAFC4FF4004320466946009305F085
:1075480023FC20460F21062205F09EFC1CBD00BF2F
:10755800000802401FB50446FFF7CEF9FFF734FCD8
:10756800FFF7F6F9FFF7BEFF01214FF4004005F0E1
:10757800D7FF02940F4C1023ADF8023020460023A9
:107588006946ADF80430ADF80C30ADF80030ADF810
:10759800063006F0F4F869464FF0402006F0C3F9CB
:1075A8002046012106F073F94FF04020012106F032
:1075B8006EF91FBD003C0040014B1860704700BFCA
:1075C800CC0C0020704710B50A4A1379262B04D832
:1075D8000949C8540133137110BD074A0123591EC4
:1075E800D45C0133272B5454F9D1034B83F826007C
:1075F80010BD00BFCC0C0020903B0020704710B598
:1076080004462078FFF7DFFF14F8013F002BF8D17C
:1076180010BD38B504460D46013D14F8010BEDB216
:10762800FFF7D1FF002DF7D138BD00BF014B187807
:10763800704700BFD40C0020014B5878704700BF3A
:10764800D40C0020024B187880F00100704700BF6E
:10765800D40C0020024B00221A705A70704700BFE9
:10766800D40C0020014B01221A707047D40C002062
:10767800014B01225A707047D40C002082B00023BD
:1076880004E0019B01330193009B01330093009BAD
:107698008342F6D302B0704707B50420012105F0F4
:1076A8001BFF01214FF4804005F046FF4FF40073A3
:1076B800009300238DF804300348012369468DF8B0
:1076C800073005F061FB0EBD000802400D4B07B501
:1076D8001A680D484FF47A73B2FBF3F20B4B013A78
:1076E8005A600B4AF02182F8231000229A60072280
:1076F8001A60084B084A00930121084B04F072F8FD
:107708000EBD00BF9C0100205C3C002010E000E0A2
:1077180000ED00E0B80200209C02002004020020D6
:10772800054B1A6812B11A68013A1A60034B1A68B5
:1077380001321A60704700BF183C0020303C00201E
:1077480082B0044B0190019A1A601A68002AFCD191
:1077580002B07047183C0020704700BF40F0BE6080
:10776800024B40F42020D860704700BF00ED00E0D5
:10777800C37810B503B3164B4278DB688478DB43D3
:10778800C3F30223C3F10401C9B202FA01F10F22C3
:1077980042FA03F2C9B222400A430E4B01781201A1
:1077A800CB18D2B283F8002303780122590903F0D9
:1077B8001F0302FA03F307E003780122590903F0D3
:1077C8001F0302FA03F32031024A42F8213010BDA8
:1077D80000ED00E000E100E021F0604121F07F01D0
:1077E800014B08439860704700ED00E0044B1A69AC
:1077F80009B1104301E022EA00001861704700BF98
:1078080000ED00E0044B1A6804280CBF42F00402A3
:1078180022F004021A60704710E000E00000000047
:10782800034A044B1A60044A044B1A60704700BFAD
:107838000000FA4560180020DB0FC93F5C180020E3
:10784800034B00221A60034A034B1A60E8E700BFA3
:10785800804200200000FA455817002007EE100A61
:10786800024BF8EEC77AC3ED007A7047581700202C
:1078780038B510EE100A07F0E1F90DA3D3E900239B
:1078880007F030FA084B044618680D4607F0D6F999
:107898000B4602462946204607F04EFB07F004FD3A
:1078A800024B186038BD00BF601800205C1800202B
:1078B800182D4454FB2119402DE9F04F2DED068B6E
:1078C8006F4CDFF8F0A189B00027A34637F80A50BB
:1078D8006C4B2580FE5A6C4B6680186807F0AEF931
:1078E80065A3D3E9002307F0FDF907F095FC636869
:1078F800664AC018011101F580610905090D60602B
:10790800C0F30B100DF1200C32F8203032F8212092
:10791800616A238115FB02F0628115FB03F516FBF2
:1079280002F216FB03F60CEB4103E0602561C0F39D
:10793800CF30C5F3CF356261A661C2F3CF32C6F34B
:10794800CF3623F8200C23F8105C23F8182C23F8E2
:10795800086C4F4BA08301310B40002BE583228438
:10796800668403DA013B63F003030133CBF8243068
:10797800002B76D14748484A6946042308F0AAFCF8
:107988004648474A04A9042308F0A4FC4548464A47
:1079980002A9042308F09EFC444A454806A904238A
:1079A80008F098FCB4F9283007EE903AB4F92A3078
:1079B800B8EEE79A07EE903AB4F92C30B8EEE78AB9
:1079C80007EE903AB4F92E30F8EEE79A07EE903ABF
:1079D800F8EEE78A68EE087A49EE097A17EE900A17
:1079E80007F02CF941EC100B09F0D6FA51EC100B0A
:1079F80007F05AFC68EEA87A49EEA97A0AEE100A4E
:107A0800206317EE900A07F019F941EC100B09F002
:107A1800C3FA51EC100B07F047FC68EE897A58EE70
:107A2800297A28EE288A0AEE900A606309EE298AE4
:107A380017EE900A07F002F9804618EE100A8946F8
:107A480007F0FCF849EC108B41EC110B09F01CFA1B
:107A58008AEE2AAA51EC100B07F026FC84ED0FAA37
:107A6800A0630237B7F5007F7FF430AF09B0BDECF3
:107A7800068BBDE8F08F00BF39D6C56D305FC440B6
:107A8800E40C0020AC1900205C180020545A0408AB
:107A980003000080B40000200C0D0020A800002086
:107AA8000E0D00209C000020100D0020120D00205B
:107AB8009000002072210020014B93ED0F0A7047BF
:107AC800E40C0020014B93ED0E0A7047E40C0020F3
:107AD800014B93ED0C0A7047E40C0020014B93ED29
:107AE8000D0A7047E40C002010B5FEF725F90020B8
:107AF800012324210246FEF789F9114B1C78002046
:107B0800012C05D10146FEF75AFA2046002104E06F
:107B18000721FEF754FA01200721FEF750FA6322E5
:107B28001221C020FFF780F902200121FEF747FA51
:107B3800FEF724FB0120BDE81040FEF714BB00BF90
:107B4800280E00200D4B1B78012B05D10C4B0D4A3C
:107B5800196812688A181A600B4B1B78012B084B9E
:107B6800196805D1094A914207DD01321A60704748
:107B7800074A914201DD01321A607047F03B00204C
:107B880054420020EC3B0020280E00207FD1F00852
:107B9800FF1FA1070E4B1B78012B05D10D4B0E4A79
:107BA800196812688A1A1A600C4B1B78012B094B4A
:107BB80005D10B4A1968914208DC1A6070471A68A7
:107BC800B2F57A2FDCBF4FF47A221A60704700BFF3
:107BD800F03B002054420020EC3B0020280E0020FF
:107BE80040420F00024B1A68024B1A60704700BFF0
:107BF800503C0020544200202DE9F04F824658485E
:107C08008BB0B0FBF1F00C4606F0F6FF41EC100B20
:107C180009F036F851EC100B07F026FBC3070746AE
:107C280048BF471E04FB07F006F0E6FF46A3D3E96A
:107C3800002307F081F904460D4645EC104B09F086
:107C48001FF859EC108B204642464B46294606F051
:107C580095FECDE904014946404607F005FB3CA3E3
:107C6800D3E900230990DDE9040107F0B7FA0028F9
:107C78003DD1002401234FF015092246984620469D
:107C8800DFF8E4B003E0234642462C46B04600FB4A
:107C980004355D452ED800FB0826DDE904012EA336
:107CA800D3E9002307F09AFA30BBDDE9042300206A
:107CB8002C4907F041F941EC100B0390029108F0B0
:107CC800DFFF0398029953EC102B8DED060B06F09D
:107CD80055FE09F1FF39CDE904015FFA89F9DDE9BB
:107CE800060107F0C1FAB9F1000FCCD104E0012573
:107CF800002601E025464646099BD9B2BAF1000F95
:107D08000BD132462B465046FEF780F801230093EC
:107D1800504651463A46534609E032462B46012022
:107D2800FEF774F80120009001463A460023FEF75A
:107D380060F9FEF723FA01200BB0BDE8F04FFEF71B
:107D480012BA00BFAFF300800000000084D777416B
:107D5800956479E17FFDA53DBBBDD7D9DF7CDB3DCF
:107D680000E9A4350000F03FFFFF0F0038B52A4BAB
:107D78001B78022B294B03D1294A12681A6038BD97
:107D88001968284B284A1B68284CCB189342236053
:107D980018DC0020FFF730FF01202168FFF72CFFD7
:107DA800234B1C780020012C05D10146FEF707F96A
:107DB8002046002104E00721FEF701F901200721F0
:107DC800FEF7FDF81B4B1B78022B14D11A4B1B4DE9
:107DD8001A68124C2B68D31822689A420BDA184B8F
:107DE8001B78012B07D1174B186800F081F822681F
:107DF8002B68D3182360084B1A78012A0AD10E4A37
:107E080011680E4A12688A1804490968914201DB10
:107E180002221A7038BD00BFD4430020544200200B
:107E2800503C00206C42002080D1F00870420020B5
:107E3800280E0020F03B0020403C0020EC3B0020B6
:107E4800383C0020083C002008B5FEF707FD094B28
:107E58005A78187002435A701AB19A7801329A7097
:107E680030B99B78034A012B02D9002353709370D1
:107E780008BD00BF240D002007B50420012105F02E
:107E88002BFB4FF46043009301238DF80430022349
:107E98008DF805300448002369468DF806308DF8C2
:107EA800073004F071FF0EBD00080240084B1A6845
:107EB8004FF47A73B2FBF3F2064B013A5A60064A62
:107EC800F02182F8231000229A6007221A60704776
:107ED8009C01002010E000E000ED00E0034B5A6830
:107EE80012B15A68013A5A60704700BF240D002049
:107EF800024B58605A68002AFCD17047240D0020B4
:107F080030B585B004460D4601A85C490A220BF03D
:107F1800D3FA5B4B1B78032B10D8DFE803F002057C
:107F2800080B01A8574907E001A8574904E001A830
:107F3800564901E0564901A80BF0A8FB04AA1319F9
:107F480013F80C3C5D19EDB22F2D01D80A3502E06B
:107F5800392D01D90A3DEDB204AB1C194FF6FF705B
:107F680004F80C5CFCF754FE0020FCF747FF0DF109
:107F780003050F24204623345A21002315F8012F26
:107F8800A4B2FCF755FFB4F5A57FF3D164205A21BC
:107F98002C220023FCF74CFF0023CD205A212C2251
:107FA800FCF746FF0020FCF733FE354B1B78032B0C
:107FB80062D8DFE803F002284B5601A931480BF0DC
:107FC80065FB0A2200212F480BF004FD314A324B91
:107FD80012781860012A06D1304A904201DC013239
:107FE8001A602F4A06E0B0F5FA5FBCBF4FF4FA52A8
:107FF8001A602C4A1B689342C4BF274B1A602A4B4D
:108008001A682A4B20E001A91F480BF03FFB0A22FF
:1080180000211D480BF0DEFC1E4A254B1278186023
:10802800012A06D11D4A904201DC01321A601C4A1D
:1080380006E0B0F5FA5FBCBF4FF4FA521A60194A6D
:108048001B68934218DD1A4B1A6015E001A90F4806
:108058000BF01CFB0D4800210A220BF0BBFC154B52
:1080680009E001A90A480BF011FB094800210A227E
:108078000BF0B0FC104B186005B030BDB49D05087E
:108088004E3C00201C3C0020443C0020594200206B
:108098000C3C0020280E0020583C00203F420F00D6
:1080A80080D1F00840420F00503C0020544200208C
:1080B800744200204C420020083C002010B50D4BB3
:1080C8000D4C1A680D4821460BF0B8FA0C4B0D48B8
:1080D8001A6821460BF0B2FA0B4B0C481A68214675
:1080E8000BF0ACFA0A4B0B481A682146BDE8104061
:1080F8000BF0A4BA583C0020BE9D05081C3C00208B
:1081080074420020443C00204C4200205942002088
:10811800083C00200C3C00209FED010A704700BF7E
:10812800000000009FED010A704700BF000000003A
:108138009FED010A704700BF00000000054B83ED6A
:10814800000AC3ED010A83ED021AC3ED031A83ED99
:10815800042A7047B0450020054B83ED050AC3ED9E
:10816800060A83ED071AC3ED081A83ED092A70473A
:10817800B0450020044B18B1012801D1034A00E0A2
:10818800034A12681A60704754420020403C00209D
:10819800503C002010B9034B18687047024B186810
:1081A800704700BF583C0020503C002010B9034BDA
:1081B80018687047024B1868704700BF7442002067
:1081C800403C002008B54FF49570FEF77DFA40F268
:1081D8006523C31A584240EB030008BD08B5C62002
:1081E800FEF772FA40F28D13C21A504240EB0200B9
:1081F80008BD4FF4957040F26521FEF757BAC620C6
:1082080040F28D11FEF752BA08B50020F8F7E4FAEB
:10821800BCEEC00A4FF4967010EE101AFEF763FA1F
:108228000020F8F7E7FABCEEC00A4FF4987010EE99
:10823800101AFEF758FA0020F8F7EAFABCEEC00A5E
:108248004FF49A7010EE101AFEF74DFA0020F8F766
:10825800EDFABCEEC00A4FF49C7010EE101AFEF74F
:1082680042FA0020F8F7F0FABCEEC00A4FF49E700C
:1082780010EE101AFEF737FA0120F8F7ADFABCEE47
:10828800C00A4FF4A07010EE101AFEF72CFA012065
:10829800F8F7B0FABCEEC00A4FF4A27010EE101A4C
:1082A800FEF721FA0120F8F7B3FABCEEC00A4FF442
:1082B800A47010EE101AFEF716FA0120F8F7B6FAB5
:1082C800BCEEC00A4FF4A67010EE101AFEF70BFAB7
:1082D8000120F8F7B9FABCEEC00A4FF4A87010EE06
:1082E800101ABDE80840FEF7FEB92DE9F04F85B039
:1082F800FFF768FF002875D04FF49670FEF70CFA68
:10830800624ADFF8BCB110604FF498700192FEF732
:1083180003FA5F4BDFF8ACA118604FF49A70029330
:10832800FEF7FAF9CBF800004FF49C70FEF7F4F969
:10833800CAF800004FF49E70FEF7EEF9DFF8889156
:10834800DFF88881C9F800004FF4A070FEF7E4F95F
:10835800C8F800004FF4A270FEF7DEF94D4F4E4EFC
:1083680038604FF4A470FEF7D7F930604FF4A67068
:10837800FEF7D2F9494D4A4C28604FF4A870FEF731
:10838800CBF920604FF4AA70FEF7C6F9454908609A
:108398004FF4AC700391FEF7BFF984464248C0F829
:1083A80000C0029B41481B68019AC360DBF800309B
:1083B80003990361DAF8003012684361D9F8003094
:1083C80082608361D8F80030C0F834C0C3613B686C
:1083D8000362336843622B6883622368C3620B6855
:1083E80003630EE0314B324C324833499C60002223
:1083F800DA6018615A619961DC611A6258629A629E
:10840800D9622A4A2D4B116BD2ED023AD2ED034ABA
:10841800D2ED045AD2ED056AD2ED067A92ED073A0A
:1084280092ED084A92ED095A92ED0A6A92ED0B7A9A
:10843800C3ED003AC3ED014AC3ED025AC3ED036A26
:10844800C3ED047A73EE633A74EE644A75EE655AC6
:1084580076EE666A77EE677A526BD96383ED053AF2
:1084680083ED064A83ED075A83ED086A83ED097A9E
:10847800C3ED0A3AC3ED0B4AC3ED0C5AC3ED0D6ABE
:10848800C3ED0E7A1A6405B0BDE8F08F440E0020E3
:108498004C0E0020640E00205C0E00202C0E0020E4
:1084A800300E0020680E0020380E0020240D002019
:1084B8000000F04200008CC2CCBC8C2CB0450020DF
:1084C800600E0020480E0020580E0020540E002098
:1084D80060EEA00AB7EE007AF0EE606A70EE077AF6
:1084E80040EE006A47EEA70A36EEC77A08B5C7EE2F
:1084F800200A10EE900A06F0A1FB0022084B06F0B5
:10850800F1FB0022074B06F03BFA06F0CDFE07EE22
:10851800900AFDEEE77A17EE900A9F3008BD00BF7B
:10852800000059400000E03F38B52DED028BF7EE12
:10853800008AB0EE608A70EE288A10EE900A28EE63
:10854800088A06F07BFB08EEA88A00220F4B06F08B
:10855800C9FB044618EE100A0D4606F06FFB0246EA
:108568000B462046294606F0E7FC0022084B06F099
:1085780007FA06F099FE07EE900AFDEEE77A17EE85
:10858800900A7730BDEC028B38BD00BF000069400F
:108598000000E03FF0B56A4D2DED068B95E80F0021
:1085A8008DB008AE103586E80F000FCD01AC0FC4B2
:1085B80095E807004FF6FF7384E807009F207721AE
:1085C8006422FAF7B4F9A020772164224FF6FF73EA
:1085D800FAF7ADF99E20772164224FF6FF73FAF778
:1085E800A6F99F20762164224FF6FF73FAF79FF9C8
:1085F8004FF6FF73782164229F20FAF798F900203C
:10860800FCF762F99F2077216522FCF737FB9F2052
:1086180077216422FCF732FB07AD0C36F7EE009A9F
:108628000435F7EE008A95ED009A4FF49674B0EE93
:1086380068AA18EE900A06F001FB3FA3D3E90023CD
:1086480006F050FB06F030FE08EE900A38EEE98A94
:10865800B0EE490AF0EE480AFFF73AFFB0EE490AD1
:10866800F0EE480A0746FFF75FFFBFB281B20F225C
:108678003846FCF736F8013CDBD14FF49674F7EE38
:10868800008A18EE900A06F0D9FA2BA3D3E9002342
:1086980006F028FB06F008FE08EE900A39EEE88A94
:1086A800B0EE490AF0EE480AFFF712FFB0EE490AA9
:1086B800F0EE480A0746FFF737FFBFB281B20F2234
:1086C8003846FCF70EF8013CDBD1B542A8D16C4620
:1086D80007AE043494ED009A4FF4C875F7EE008A9B
:1086E80018EE900A06F0AAFA13A3D3E9002306F0BD
:1086F800F9FA06F0D9FD08EE900A38EECA8AF0EECB
:10870800490AB0EE480AFFF7E3FEB0EE480AF0EE79
:10871800490A0746FFF708FFBFB281B20022384670
:10872800FBF7DFFF013DDBD1B442D2D10DB0BDEC88
:10873800068BF0BDAFF30080295C8FC2F528F03FAF
:10874800549A0408121A06EE902A081AB8EEE67A25
:1087580006EE900AF8EEE67AC7EE277A9FED047ADD
:1087680067EE877AFDEEE77A17EE900A704700BF4A
:108778000000A0438A1A06EE902A081AB8EEE67A94
:1087880006EE900AF8EEE67AC7EE277A9FED047AAD
:1087980067EE877AFDEEE77A17EE900A704700BF1A
:1087A8000000484370B506460D460024610704D50D
:1087B800A0B231462A46FBF794FF0134B4F5A07FF6
:1087C800F4D170BD70B506460D460024600704D587
:1087D800A1B230462A46FBF784FF0134C82CF5D1F4
:1087E80070BD114B11481B781149124A0068012BC2
:1087F800114B09D1126808601A60104B1A68104BA7
:108808001A60104B1A680CE01268D2011A600B4B00
:108818001A680B4BD2011A600A4B1A68C00108602B
:10882800D201094B1A607047280E0020583C0020DE
:10883800503C002074420020403C00204C42002064
:10884800EC3B0020283C00206C420020024B1A68B8
:10885800024B1A60704700BF503C00205442002071
:1088680008B5FFF7BEFFBDE80840EFE770B5002187
:108878000A222748274D284E284C0BF0ABF8002138
:108888000A22286026480BF0A5F800210A22306049
:1088980024480BF09FF800210A22206022480BF0A0
:1088A80099F8224B326818602B68D31A06EE903A72
:1088B80023681F4AB8EEE67A06EE903AF8EEE67AB2
:1088C800C7EE277AFCEEE77A17EE903A01339BB2AF
:1088D80007EE903AB8EE677AF4EE007A67EE277AF8
:1088E8001380FCEEE76A134B16EE901A8AB206EE76
:1088F800902AB8EEE67A198077EEC77AF5EEC07A54
:10890800F1EE10FA01DD01321A80BDE87040A7E7E8
:108918001C3C0020583C0020744200204C4200209F
:10892800443C0020594200200C3C0020083C002018
:1089380080450020F84500200022F0B51346202687
:1089480003254FF02C0C00E02646303EF6B21746C1
:108958000132092E10F8014B0AD897FBF5F605FBF2
:1089680016772FB9CE1801F803C07470023301E0EE
:10897800CC540133092AE7D12022CA54CB18482203
:108988005A707A229A700022DA70F0BD70B58CB0F5
:1089980005460C4608A80E491E460AF04FFE08A8D0
:1089A8006946FFF7C9FF6A460A4904A80AF046FE65
:1089B800BDF84000FCF72CF93046FCF73FF9284693
:1089C800214604AA0023FCF751FA0CB070BD00BF81
:1089D80046950508979B05082DE9F04F084B2DEDA6
:1089E8000A8B1B78022BCBB0064B0FD1064A1268B4
:1089F80042F210701A60FEF737FC00F0A3BD00BF0A
:108A0800D443002054420020503C0020D44A1E6821
:108A1800127812B9802396FBF3F6D24CD24FE36B4F
:108A2800F21A07EE102A226CD31AB8EEC79A07EE8C
:108A3800103AF8EEC77A9FEDCDCA89EE279AFFF76C
:108A48003BF887ED0E0AFFF73DF8D4ED0A7A94ED6E
:108A5800008AD4ED018A09EE278AD4ED0B7A87EDD6
:108A68000F0AB86B49EE278A10EE105A06F0E6F89E
:108A780080462846894606F0E1F841EC100B41ECA7
:108A88001B0B08F0A5F8404653EC102B494606F09E
:108A980029F906F009FCB0EE4B0AF0EE6B0A0AEE73
:108AA800100A08F095F9404653EC102B494606F099
:108AB80019F906F0F9FB07EE100AD4ED0C6AD4EDAB
:108AC800027A68EE879A58EE0A9A49EE267A68EE94
:108AD8008A8A79EEA79A48EE078AD4ED037A94ED4C
:108AE8000D7A49EE077ADFEDA2BA78EEA78AF4EE9E
:108AF800EB8A68EEA87A49EEA97AF1EE10FAB1EE9F
:108B080068AAC8BFF0EE6B8AF4EE4C8AF1EE10FA50
:108B180048BFF0EE4C8A89EEA7BA8AEE27AAFDEE86
:108B2800007AF4EEE78AF1EE10FA08DDF5EE408AF5
:108B3800DFED907AF1EE10FA48BFF0EE678A8E4BBF
:108B480019EE900AC3ED009AC3ED018A06F076F893
:108B580000228A4BCDE9040105F010FF68EEA87ADF
:108B6800044617EE900A0D4606F068F8224680463D
:108B780089462B462046294606F0B4F842464B461D
:108B880005F0FEFE41EC100B08F006FA0022DDE9C4
:108B980004017A4B5BEC10AB05F0F2FE02460B4683
:108BA80006F0A0F842464B4605F0EAFE41EC100BF1
:108BB80008F0F2F95946504655EC104B06F074FB94
:108BC800294608EE100A204606F06EFB07EE900ACA
:108BD80088EE278A6A4C6B4DF7EE00AA18EE100A49
:108BE80006F02CF858A3D3E9002306F0EDFADFEDE0
:108BF800667A002818BFB0EE678AB4EE6A8ADFED9D
:108C0800637AF1EE10FAC8BFB0EE678ADFED607ADA
:108C18006AEE277A84ED008A17EE900A06F00EF8BD
:108C2800DFED5C7A4BEE4B7A4AEE4A7A894680460B
:108C3800C5E9028917EE900A06F000F849EC108B96
:108C480041EC110BC5E9000108F01EF951EC100BBD
:108C580006F02AFB38EE2A9A7AEEC87A4E4B89EE4D
:108C6800279A1B78DFED427AB4EE6B9AF1EE10FA90
:108C7800C8BFB0EE679AB4EE4C9ADFED3C7AF1EEDD
:108C880010FA80F0004948BFB0EE679A022BC4F88A
:108C9800049040F0A980414B1B78002B00F0A48081
:108CA8003F4B404C1B681C40002C03DA013C64F02D
:108CB80007040134082718EE100A93FBF7F705F0AC
:108CC800BDFF0022384B06F00DF806F0CDFA054638
:108CD800484605F0B3FF1EA3D3E9002306F002F8C7
:108CE8001DA3D3E9002305F04BFE06F0BDFA2F4B78
:108CF8001D491E6001EBC403C6F3072283F8412017
:108D0800C6F30742BF0183F8422083F84450320E6D
:108D1800C5F3072583F84600072CC0F30720BFB228
:108D280083F8406083F8432083F8455083F8470070
:108D38003ED107F5806080B240314022FEF736FB15
:108D4800B0B3FEE7AFF300802D431CEBE2361A3FC9
:108D5800CDCCCCCC0C5FC44000000000C0FFDF408D
:108D6800280E0020B0450020240D0020003C1CC621
:108D7800003C1C46CDCC4C3DCC4300200000494073
:108D8800B44200208845002017B7D13872F97F3FD8
:108D98000AD7233D17B7D139F03B00209C45002066
:108DA800B0420020070000800000F040C4430020CB
:108DB8009B4B1B689E4213DB07F58067B8B2994945
:108DC8004022FEF7F3FA044600B1FEE7964D4FF451
:108DD8007F70B5F90010FDF769FC944B2C601C708E
:108DE800914B1A6801321A60FEF772FE904C84EDBE
:108DF800200AFEF773FE84ED210AFDF723FC3246B4
:108E0800C4F888008B4936A80AF018FCD4F880000A
:108E180005F014FF02460B4626A887490AF00EFC07
:108E2800D4F8840005F00AFF02460B462AA88349B5
:108E38000AF004FC1BEE100A05F000FFCDE906015C
:108E4800DDE906237E492EA80AF0F8FB1AEE100A7F
:108E580005F0F4FE82468B4652467A495B4632A8B4
:108E68000AF0ECFBDDE90423774912A80AF0E6FBD7
:108E780018EE900A05F0E2FECDE90A01DDE90A23C1
:108E8800724916A80AF0DAFB18EE100A05F0D6FEA9
:108E9800CDE90C01DDE90C236D491AA80AF0CEFBD7
:108EA800484605F0CBFECDE90801DDE9082369490C
:108EB8001EA80AF0C3FB19EE100A05F0BFFE804693
:108EC8008946424664494B4622A80AF0B7FB0EA8D9
:108ED8006249D4F888200AF0B1FBF5EEC08AF1EEB9
:108EE80010FA9FED5FAA37D5304605F095FE46A3E8
:108EF800D3E9002305F0F6FEF1EE687A044617EE92
:108F0800900A0D4605F09AFE02460B462046294671
:108F180005F0E8FE02460B463DA1D1E9000106F046
:108F28000BF806F0C1F99FED4F7A07EE900AF4EEC0
:108F3800C77AF1EE10FAC6BFC7EE8A7A4A4C4B4C94
:108F4800F4EECA7AF1EE10FA36DD9FED457A484D17
:108F5800484CC7EE877A32E02FA3D3E90023DDE936
:108F68000A0105F0BFFE044630460D4605F054FEE2
:108F780025A3D3E9002305F0B5FE02460B4620469B
:108F8800294605F0D9FF06F08FF907EE900AF4EEAE
:108F9800EA7AF1EE10FA46BF67EE8A7A364C374C19
:108FA800F4EECA7AF1EE10FA08DD9FED2D7A344D11
:108FB800344CC7EE877A02E02D4D00E0304D17EEB5
:108FC800900A05F03BFE2A46CDE900013AA82E4951
:108FD80002940AF033FB2D4B1B78013BDBB2012BCB
:108FE80000F2A2822A4B1B78072B00F29D82DFE851
:108FF80013F051009B02DF006601CB011B027102D6
:109008003D0200BFAFF300801F85EB51B81E194029
:10901800000000A2941A6D420000000080842E41D6
:1090280074420020640D0020B04200209C450020BE
:10903800240D0020D59D0508DF9D0508EA9D05083B
:10904800F59D0508FF9D0508099E0508149E05085D
:109058001F9E05082A9E0508359E0508419E05089D
:1090680000007A4400247449C49D05083F9505080A
:10907800629F0508CD9D0508CA9D0508C79D05087E
:10908800D09D0508D29D05084E9E0508F03B00209E
:10909800684200200220FBF7B1FE4FF6FF70FBF795
:1090A800CDFD1F20FBF7B4FD19210023A64A2D2072
:1090B800FBF7DCFE4FF6FF70FBF7C0FD0020002435
:1090C800FBF7A6FD0F20B42132464FF6FF7300943C
:1090D800FFF75CFC0F206E2126AA2346FBF7C6FE8D
:1090E800A0206E212AAA2346FBF7C0FE0F203821B4
:1090F8001AAA2346FBF7BAFEA02038211EAA234647
:10910800FBF7B4FE0F205C212EAA2346FBF7AEFE28
:10911800A0205C2132AA2346FBF7A8FE0F204A2193
:1091280012AA2346FBF7A2FEA0204A2116AA23462C
:10913800FBF79CFE0F209B21234622AAFBF796FEF5
:10914800824B1B78012B05D10F2084213AAA234694
:10915800FBF78CFE7E4BD3F88830B3F57A7FCCBF13
:109168004FF4FC604FF47840FBF768FD0023A02023
:109178009B210EAAFBF77AFE764B1B78012B08D1B0
:109188004FF4FC60FBF75AFD4FF48C700221724AD1
:1091980007E04FF6E070FBF751FD704A4FF48C7012
:1091A80002210023FBF762FE1F20FBF747FDBBE10E
:1091B800DDE9062344A86A490AF040FA52465B46AC
:1091C80047A868490AF03AFADDE904233EA8664947
:1091D8000AF034FADDE90A2341A864490AF02EFAB4
:1091E800E620022144AA0023FBF740FEE6201621D0
:1091F80047AA0023FBF73AFE0220C8213EAA002313
:10920800FBF734FE41AA00230220DC21FBF72EFEE7
:10921800DFED577A28EE278A4FF6E07518EE100A28
:1092280005F00CFD9DED080B8B46824607F0D0FC3F
:1092380059EC108B9DED080B07F0CAFD00208DED51
:10924800040BFBF7FBFC0A2132460023052000959E
:10925800FFF79CFB4FF47840FBF7DAFC42464B469D
:109268005046594605F03EFD33A3D3E9002305F0E7
:1092780087FB05F0D1FFDDE9042384B25946504647
:1092880005F030FD02460B462DA1D1E9000105F09D
:1092980075FB05F0C1FF81B22046F9F778FB9D20E8
:1092A800772105220023FBF7E3FC9F207521052287
:1092B8000123FBF7DDFC2846FBF7AAFC34E12D4B24
:1092C80018682D4B324619689FED2C8AFFF73AFA39
:1092D800F4EEC89AF1EE10FA044614D5F5EEC09AE9
:1092E800F1EE10FA0FDDFDEEE99A4FF4FA7119EE7E
:1092F800902A0020FFF73EFAA3B281B24FF6FF7220
:109308001846FBF7EEF9F4EEC88AF1EE10FA40F1D0
:109318000B81DFED1B7AF4EEE78AF1EE10FA40F3E9
:109328000381FDEEE88A174818EE902A4FF4FA7187
:10933800FFF720FAA4B2C8E00000000000E0634094
:109348000000000000C05D405B9E0508F03B002067
:10935800240D0020280E00207A9E05087E9E050810
:10936800829E05088C9E0508969E0508A09E050805
:109378000000C842583C0020744200200000FA4314
:109388000000FAC30CFEFFFF7F4B18687F4B324684
:109398001968FFF7D7F9B5EEC0BAF1EE10FA04462E
:1093A8001DDDDDE906016AA3D3E9002305F00CFF02
:1093B800A8B169A3D3E90023DDE9060105F092FC11
:1093C80002460B460020724905F0D8FA05F024FF42
:1093D800A5B281B24FF6FF722846FBF782F95046D4
:1093E80059465FA3D3E9002305F00CFF002800F0DD
:1093F8009B805046594656A3D3E9002305F0E4FE66
:10940800002800F0918058A3D3E90023504659461C
:1094180005F068FC02460B4600205E49A4B205F040
:10942800ADFA05F0F9FE50E0574B1868574B324635
:109438001968FFF787F94EA3D3E900230446DDE94D
:109448000C0105F0DFFE68B19DED0C0B07F01EFD69
:10945800002251EC100B504B05F044FC05F0DCFEEB
:10946800014600E0C821A0B289B259E0464B18680D
:10947800464B32461968FFF765F9DFED487A48EE42
:10948800677A84B2FDEEE77A204617EE901A4FF617
:10949800FF7289B2FBF725F937A3D3E90023DDE989
:1094A800080105F01FFC36A3D3E9002305F044FDAD
:1094B80005F0FAFE07EE900AFDEEE77A6FF0B300CA
:1094C80017EE902AB421FFF755F981B24FF4FC62E8
:1094D800204627E0DFED327AB4EEE79AF1EE10FA93
:1094E80022D5294B1868294B32461968FFF72AF903
:1094F80049EC108B044607F0C9FC53EC102B1046BE
:1095080019460022234B05F0EDFB02460B460020CE
:109518001F4905F033FA05F07FFEA4B281B2204658
:109528004FF6FF72FBF7DDF81E4B1B78022B09D0B4
:1095380043B14FF6FF7300930520DC213246002328
:10954800FFF724FA4BB0BDEC0A8BBDE8F08F00BFE3
:109558009A9999999999B93F0000000000409F4055
:109568009A9999999999B9BF0000000000408F40D5
:1095780089B5F81400E3693F0000000000807640D8
:109588001F85EB51B81E1940583C0020744200203A
:109598000000694000005940000054C000004843E2
:1095A8000000C842684200202DE9F04F764B2DEDAF
:1095B800048B93ED008A78EE087A83B017EE900A50
:1095C80005F03CFB714B064618680F4605F036FB64
:1095D80068EE088A82468B46F7EE009A4BEC10AB91
:1095E80007F0F6FA78EEA97A55EC104B17EE900AC8
:1095F80005F024FB22462B468046894630463946EC
:1096080005F070FB02460B464046494605F0B6F9A0
:1096180005F04AFE79EEE88A09EE100AC8EE898A52
:10962800DFED5B7A4BEC10AB68EEA78A07F0D0FB56
:10963800304653EC102B394605F054FB044619EE1E
:10964800100A0D4605F0FAFA02460B46204629464E
:1096580005F072FC4F4B002205F044FB05F024FE98
:109668004D4B1B78033B09EE100A042B78D8DFE832
:1096780003F003122F58460018EE900A05F0DEFAA0
:10968800044619EE100A0D4605F0D8FACDE9000196
:109698004248434917E029EE098A08EEA88AB1EE44
:1096A800499AC8EE888A89EE088A18EE900A05F069
:1096B800C5FA044618EE100A0D4605F0BFFACDE9C2
:1096C80000013648374922462B4609F0B7FF47E0E4
:1096D80018EE100A05F0B2FA41EC100B07F0D6FBB1
:1096E8000022314B51EC100B05F0FCFA05F0DCFDC3
:1096F80005F0A4FA02460B4628482C492EE018EE3D
:10970800100A05F09BFA1CA3D3E9002304460D4672
:109718005046594605F0E6FACDE900011F482449AC
:10972800D1E718EE100A05F089FA15A3D3E900234A
:1097380005F068FDDFED1F7A002818BFB0EE678AD4
:1097480078EE297A79EEC89AC7EEA99A19EE900AA6
:1097580005F074FA02460B461048174909F06EFFE7
:109768000E4A0220CA21002303B0BDEC048BBDE8D9
:10977800F04FFBF77BBB00BFF6285C8FC2A54C40BF
:10978800AE47E17A14AEEF3FBC420020C042002051
:109798000000484200004940684200208A420020F8
:1097A800AA9E0508BA9E0508000034C0CA9E05088E
:1097B800DC9E0508A4707D3FF89E050873B5044635
:1097C800002800F0B1805C4B18880419A4B222B2BA
:1097D800002A05DB40F23F139A42C8BF1C4600E04E
:1097E80000240121FAF7DCFE0120FAF72DFD534E83
:1097F8000025A85B0235FAF775FDB5F5C67FF8D1E7
:10980800A0B20121C7224EF29C73FBF7DFF84C4D42
:10981800494B4C4A1C8012682B6824B206EE904AC9
:10982800D21AB8EEE67A06EE902AF8EEE67ADC214D
:1098380067EE277A9FED447AC7EE877A05200026DF
:10984800FDEEE77A17EE904A1C194FF6FF73224691
:1098580000930023FFF79AF82B68E41A3B4B1B6828
:1098680094FBF3F407EE104AF8EEC77A384CFCEE96
:10987800E77A17EE905AED00ADB205F58065A8B20B
:10988800FDF714FC2070681C80B2FDF70FFC6070B7
:10989800A81C80B2FDF70AFCA070E81C80B2FDF796
:1098A80005FCE070281D80B2FDF700FC60F3070698
:1098B800681D80B2FDF7FAFB60F30F26B6B207EE1B
:1098C800906AB8EE677ADFED237A234C67EE277A41
:1098D800A81DC4ED007A80B2FDF7E8FB0735002625
:1098E80060F30706A8B2FDF7E1FB60F30F26B6B2F6
:1098F800A6F5FE46FF3E06EE906AF8EEE67A174DAC
:1099080017EE900A05F09AF909A3D3E9002305F0A8
:1099180013FB05F0C9FC124B28601A78204629462B
:1099280002B0BDE870403FE602B070BDAFF3008002
:10993800CDCCCCCC0C5FC44088420020D64300205C
:10994800583C00207442002000809F434C42002075
:10995800C443002000008037BC420020C0420020E1
:1099680068420020124B1B78022B13B51FD0114CF4
:10997800B4F88C30ADF80630BDF806309BB25BB158
:10998800BDF806004EF29C7380B20121C722FBF796
:109998001DF80023A4F88C30074B1B78022B06D146
:1099A800064C94F90000FFF709FF002323701CBD43
:1099B80068420020240D0020D44300208C2B002076
:1099C8002DE9F0434FF47F708DB0FCF77DFE002742
:1099D8001FFA80F86BE04FEAC7091FFA89F909F501
:1099E80080691FFA89F0FDF761FB60F3070409F14C
:1099F800010080B2FDF75AFB60F30F2409F1020061
:109A080080B2FDF753FB60F3174409F1030080B2FD
:109A1800FDF74CFB60F31F6409F1040080B2FDF709
:109A280045FB60F3070609F1050080B2FDF73EFB30
:109A380060F30F2609F1060080B2FDF737FB09F144
:109A4800070960F307051FFA89F0FDF72FFB60F39C
:109A58000F25B0B205F0E0F800221B4B05F042F9E3
:109A680005F022FC05F0EAF8CDE90001A8B205F0FE
:109A7800D3F811A3D3E9002304F080FF10A3D3E99E
:109A8800002305F059FA05F00FFC05F0D7F8224637
:109A9800CDE902010D4905A809F0D0FDC1B205A81C
:109AA80001F04AFD0120FEF723FA0137BFB2B8459D
:109AB80091DA0DB0BDE8F08300000000C0FFDF4080
:109AC800E17A14AE47C166400000F03E039F0508E6
:109AD80008B50021C620FCF7E9FD4FF49570002178
:109AE800BDE80840FCF7E2BD024B4FF6FF721A8052
:109AF800704700BF8842002000200146C82240F27B
:109B08003F13FAF748BF07B50DF1070001F015FD3F
:109B18009DF807000EBD08B5FFF7F5FF0028FBD13B
:109B280008BD30B5044687B010EE100A0D4605F0A2
:109B380085F802460B4601A8054909F07FFD204635
:109B4800294601AA0023FBF791F907B030BD00BFF1
:109B5800169F050808B5084802F078FB0648022158
:109B680002F045FC0028F9D0034802F09BFB07EE01
:109B7800900AB8EE670A08BD0020014010B50C4CE9
:109B880000232DED028B23809FED0A8A06E0FFF764
:109B9800E1FF238838EE008A013323802388182BBD
:109BA800F5D99FED050A28EE000ABDEC028B10BD21
:109BB800BC3B002000000000ACC8683910B54FF469
:109BC800C770FCF781FDDB2805D14FF4C870FCF79E
:109BD8007BFD84B219E041F2E104214644F2010020
:109BE800FCF764FD44F20100FCF76EFDA04214BFCF
:109BF80080244FF4007421B24FF4C870FCF756FD6E
:109C08004FF4C770DB21FCF751FD204610BD024B15
:109C180000221A70704700BF9C450020014B0122AA
:109C28001A7070479C450020014B00221A6070474B
:109C3800B0420020014B1878704700BF9C450020B7
:109C48000030024B18BF0120187070479D45002056
:109C58000C4B1A680C4B1A600C4A002313700C4A00
:109C680013700C4A012111700B4A4FF6FF701080D7
:109C78000A4A13700A4B04224FF080401A7004F00D
:109C88008CB800BF503C002054420020383C0020D3
:109C98009C450020D80C002088420020D443002096
:109CA800E00C0020AFF300807047FEE7FEE7FEE718
:109CB800FEE7704770477047FEF710B910B5094CBA
:109CC800A37A4BB1084B1A6822F006021A6000F01A
:109CD80013F8204600F063FE4FF48020BDE81040E2
:109CE80002F0AEBD5C3C002010ED00E0014801F040
:109CF80025B800BF5C3C0020364BD3F8882042F4DE
:109D08007002C3F88820344B1A6842F001021A60C6
:109D180000229A60196821F0847121F48031196059
:109D28002E495960196882B021F480211960DA60DF
:109D3800009201921A6842F480321A601A6802F49A
:109D480000320192009A01320092019A1AB9009ADF
:109D5800B2F5A06FF2D1204B1B6813F4003318BF83
:109D680001230193019B012B2ED11B4B1A6C42F04E
:109D780080521A641A4A116841F4804111609A6845
:109D88009A609A6842F400429A609A6842F4A05233
:109D98009A60144A5A601A6842F080721A60196808
:109DA8000D4A8901FBD5104B40F205611960936893
:109DB80023F003039360936843F00203936093686E
:109DC80003F00C03082BFAD1024B4FF000629A60A3
:109DD80002B0704700ED00E0003802401030002467
:109DE8000070004008544007003C0240184B194AD4
:109DF800996801F00C01042903D0082903D0164BF7
:109E080019E0164B17E059685A6811F4800F596821
:109E180014BF124B104B02F03F02B3FBF2F30C4A93
:109E28005268C2F30142C1F38811013252004B4318
:109E3800B3FBF2F3074A1360054B9A68054BC2F36C
:109E480003129A181968127921FA02F21A607047F7
:109E5800003802409C0100200024F40000127A001F
:109E680037B51C230124002501A88DF804308DF88E
:109E780005508DF806408DF80740FDF779FC20461F
:109E8800214603F04DFB09494CF24F334B60A723A1
:109E98000B800D814D804FF0804003F0E9FE4FF0BC
:109EA80080402146224604F0A8FA3EBDFC45002029
:109EB80010B54FF08040012104F0B4FA00282CD0EE
:109EC8004FF080400121154C04F0B7FA4FF0804064
:109ED800002103F062FF2378013B032B1DD8DFE844
:109EE80003F002060A0FBDE81040F6F709BDBDE809
:109EF8001040F6F7DFBCF7F759F90023237010BDBF
:109F0800074A002323701370064B01241C70FFF7C7
:109F180085FEFFF789FE044B1C7010BDE00C002085
:109F2800D80C0020D4430020383C002008B540203D
:109F380002F078FC30B1FBF7F7F84020BDE80840A4
:109F480002F07EBC08BD0000014608B5044804F0D4
:109F580033FC0348402104F0DCFC0028F9D008BD9C
:109F680000440040F0B589B04FF4E133012001937B
:109F780000232B4CADF808301E460146ADF80A30D8
:109F8800ADF80C30ADF810300C23ADF80E3003F0FE
:109F9800A3FA4FF40030012103F0C2FA206802212D
:109FA800072202F071FF07226068032102F06CFFAC
:109FB8000125022704232068059305A98DF81A6056
:109FC8008DF81B508DF818708DF8197002F0DCFEB2
:109FD80008236068059305A98DF8187002F0D4FE6F
:109FE800A06801A904F03EFB2A4640F225510D481D
:109FF80004F076FC262307A88DF81C308DF81D6028
:10A008008DF81E608DF81F50FDF7B2FBA068294639
:10A0180004F0A5FB044A054B1A6009B0F0BD00BF67
:10A02800B001002000440040519F0008684F002004
:10A03800024B9868002104F092BB00BFB0010020D9
:10A0480010B5094C40F22551204604F06CFC50B183
:10A05800A288D2B2112A02D1044B01211970044BF3
:10A0680019884A401A8010BD00440040DA0C0020CC
:10A07800B40D00207047704773B50120014603F006
:10A088002BFA264C4FF4D8530093022303268DF85D
:10A0980004302046002369468DF806308DF80730D5
:10A0A8008DF8056002F070FE204608210A2202F0B1
:10A0B800EBFE204609210A2202F0E6FE20460B218B
:10A0C8000A2202F0E1FE0A2220460C2102F0DCFE00
:10A0D80001254FF480632046694600938DF80650A9
:10A0E8008DF807508DF8056002F04EFE0A210A46E9
:10A0F800204602F0C9FE29464FF4804003F01CFABE
:10A108008020294603F0F4F94FF08050294603F0E7
:10A1180043FA284602F094FB7CBD00BF00000240D1
:10A1280007B54FF4C060FDF719FB43238DF80430E1
:10A138000322012301A88DF805308DF806208DF83B
:10A148000730FDF715FB0EBD782358430723B0FBF6
:10A15800F3F0002301338342FCD970474FF47A733C
:10A168005843F1E737B50023104C01930546032007
:10A17800FFF7EAFFEB681A69013C019213D0019AD4
:10A18800002AF4DA019A42F001020192019A1A6156
:10A19800064A1969013A019102D00199C907F8D410
:10A1A8000320FFF7D1FF00203EBD00BF410D030093
:10A1B80010B5C47874B900EB820003339B10D0F853
:10A1C800D000224603E051F8044C01320460043107
:10A1D8009A42F8D1002010BD033230B59210D0F861
:10A1E800D0400B46002003E02568013043F8045CAA
:10A1F80004339042F8D101EB800030BD0122F0B564
:10A208000023827040220129C37082800CD1082368
:10A218000370042343704FF4A073C38002230372B6
:10A22800C1724FF0A04309E041B90C230370062323
:10A2380043704FF4A063C3801F4BC17203F50062E3
:10A248000261C3604678044601461A46002508E0C4
:10A2580002F5106C02F530620A65C1F814C00135C8
:10A268003A460431B54202F12007F1D303F5806282
:10A27800426103F58862C0F8CC20067803F5A06532
:10A288000146002203E0C1F88C5001322035043128
:10A29800B242F8D31946002202E0C4F8CC100132C9
:10A2A8000434B24201F58051F7D303F56063C0F876
:10A2B8000C310020F0BD00BF0000044038B5037A1F
:10A2C800C2680025012B044625D1936B417A65F3BA
:10A2D800104309B143F480139363D36823F48003D4
:10A2E80023F0500343F010036FF3C3036FF3C71356
:10A2F8006FF351436FF3D343D3602046FFF732FF28
:10A30800E378012B3ED1052363F34405E36845F068
:10A3180020059D6036E0D36843F04003D360FFF723
:10A3280021FF237A627A032B14BF4FF434134FF4BE
:10A338003C130AB143F48013E26814209363FFF7D7
:10A348000DFFE268217AD368032908BF43F48033FC
:10A35800D360237A032B15D1156B012363F39B6517
:10A368006FF3D7552D2345F0805563F316451563D4
:10A37800C820FFF7F3FEE36845F400051D63C82015
:10A38800FFF7ECFEE378012B07D1E3689D6805220F
:10A3980062F3440545F020059D60002038BDC36880
:10A3A8009A6842F001029A6000207047C3689A6870
:10A3B80022F001029A600020704707B5002301933C
:10A3C800019B43F020030193019B61F38A130193DE
:10A3D800019BC2681361064B1169013B019102D0D0
:10A3E80001998806F8D40320FFF7AEFE00200EBDC1
:10A3F800410D030007B500230193019B43F01003AF
:10A408000193019BC2681361064B1169013B0191DD
:10A4180002D00199C906F8D40320FFF795FE002061
:10A428000EBD00BF410D030008B5C268D3680129FD
:10A438006FF35D736FF39E7302D143F0005302E034
:10A4480009B943F080433220D360FFF787FE00202C
:10A4580008BDC368586900F001007047C3685B69AC
:10A4680013F0010F14BF002001207047C36858691A
:10A4780000F001007047C3685A6998691040704736
:10A48800C3685868704703691A6861F301021A6063
:10A498007047C268002393614FF0FF3353615360E4
:10A4A80053610B4B9361C3789169002B14BF4FF430
:10A4B80000634FF4016343F4701343F4405343F0D3
:10A4C800080321EA03010B4393610020704700BF92
:10A4D80000080080F8B5D0F80C3100221A60036932
:10A4E80015461A6865F3CC221A60C37A012B044614
:10A4F8001BD10321FFF7C7FFE36880214FF48002D7
:10A5080061F30F0259629A62C02262F30F0561F388
:10A518001F454FF4A072C3F8045162F30F056FF39F
:10A528001F45C3F80851C3F80C5110212046FFF706
:10A5380044FF2046FFF75EFF226900234FF0FF31FA
:10A548001361204653611E469161FF25D361214660
:10A5580010E082691768C7F3076707F08007FFB242
:10A56800002F14BF4FF09047002717600133166182
:10A578000430956062789342EBD300231D46FF2098
:10A5880010E04A6D1668C6F3076606F08006F6B254
:10A59800002E14BF4FF09046002616600133156157
:10A5A8000431906062789342EBD323691A6942F4CC
:10A5B80080721A61E278012A04D1054A402161F3C8
:10A5C80059421A632046FFF764FF0020F8BD00BF18
:10A5D8000301010003699B68C3F34103013B022B9C
:10A5E8009ABF024AD05C0320704700BF9C9A0408B7
:10A5F80010B5036981699C680A68C4F341000228A0
:10A6080002D06FF30A0202E0032060F30A020A6034
:10A618005A6842F480725A60002010BD30B54D78F7
:10A628000B780022012D00EB830405D105FA03F312
:10A63800A46963F30F0205E0012505FA03F3646DCD
:10A6480063F31F422368C3F3072505F08005EDB2C5
:10A658006DB98D6865F30A03CD78C98865F39343AE
:10A6680061F3995343F0805343F400432360036933
:10A67800D9690A43DA61002030BD30B54D780B78CE
:10A688000024012D224600EB830105D105FA03F3CE
:10A69800896963F30F0205E0012505FA03F3496DA3
:10A6A80063F31F4203696FF3CF340C60D96921EA61
:10A6B8000202DA61002030BDF8B54F780B78012F1F
:10A6C80000EB830349D19E694C69356833692A4692
:10A6D80064F3120314B967F3DC430BE08F68E419E1
:10A6E800013CB4FBF7F7CC7867F3DC43012C08BFD7
:10A6F80064F35E733361C378012B06D10B780C6960
:10A7080000EB83039B695C610CE0CB78012B09D0DB
:10A718004B693BB103690C785E6B012707FA04F4B7
:10A7280034435C63CB78012B07D103699B68DB0555
:10A7380054BF45F0005245F080520B7800EB83037C
:10A7480042F004429B691A60CB78012B38D10A7811
:10A758008B8AC968FFF72CFD32E05E6D4F6935685A
:10A768008C6833692A462FB964F31203012464F311
:10A77800DC430AE03F19013FB7FBF4F7BF05BF0D03
:10A7880067F3DC437C4364F312033361C378012B22
:10A7980005D10B780C6900EB83035B6D5C61CB78AA
:10A7A800012B06D14B7913B145F0005201E045F079
:10A7B80080520B7800EB830042F00442436D1A602C
:10A7C8000020F8BD73B54D78012D3DD183694A69E4
:10A7D8001E681C690094E4B242B962F306048DF85D
:10A7E80000409DF8024065F3C4040EE08D68AA425B
:10A7F80086BF4D6165F3060462F306048DF80040D8
:10A808009DF80240012262F3C4048DF80240009AC8
:10A818001A61C278012A05D10A780C6900EB820214
:10A828009269546146F004421A60C378002B34D10F
:10A838004B69002B31D003690A78586B012101FA62
:10A8480002F202435A6328E00B784E698C6800EBE9
:10A8580083035B6D1A681D690095EDB206B14C6102
:10A8680064F306059DF802408DF80050012565F354
:10A87800C4048DF80240009C1C61C378012B05D1EB
:10A888000B780C6900EB83035B6D5C610B7800EB64
:10A89800830042F00442436D1A6000207CBD4B786F
:10A8A800012B0B7800EB83000AD182691368C3F38C
:10A8B800076101F08001C9B221B143F0804301E092
:10A8C800426D136843F400131360002070474B78FF
:10A8D800012B0B78C97800EB83000CBF8269426DAD
:10A8E80002391368C9B26FF35553012998BF43F071
:10A8F800805313600020704703699A69D869104033
:10A90800000C704700EB810102694B6D9B68506930
:10A918001840704703699869DB69184080B270472E
:10A9280082B000230093C0238DF803300122002356
:10A9380062F3C4038DF8023018238DF80030009AB2
:10A94800436D1A61C278012A06D100F5B9605861D1
:10A958001A684FF080221A6002B07047D0F814319C
:10A9680010B50446D3B103699A68D20716D5827A1E
:10A9780042B1D0F80C21D0F80C116FF341026FF3FB
:10A9880000020A605A6842F001025A600520FFF787
:10A99800E5FB23695A6822F001025A6010BD837AE8
:10A9A80063B103699B68D90708D5D0F80C31D0F892
:10A9B8000C216FF341036FF3000313607047012309
:10A9C80010B5002280F8123104460346FF2104E046
:10A9D80058698160186D0132816060780433824261
:10A9E800F6D3236900221A615A61DA614FF0FF3207
:10A9F8009A612046FFF7FEFC20461021BDE8104072
:10AA0800DBE44B78012B0B7800EB83000FD18369D3
:10AA18001868C0F3074000F02003DBB2CBB900F0A0
:10AA28000200C0B200280CBF302020207047436DC0
:10AA38001868C0F3074000F02003DBB25BB900F0F0
:10AA48000200C0B200280CBF4FF440504FF4005031
:10AA58007047102070474FF4805070474B78012B97
:10AA68000B7810B500EB83030AD19C69102A236880
:10AA780002D1BDE8104012E7202A0CD0302A0FE09E
:10AA88005C6DB2F5805F236802D143F400131BE0CC
:10AA9800B2F5005F02D143F0006315E0B2F5405F04
:10AAA8000FD1C3F3074202F02002D2B222B1002331
:10AAB8004B71BDE810400AE743F0806343F0802300
:10AAC80002E00AB962F3CF33236010BDF8B504463B
:10AAD800FFF794FB0122002384F8122184F8133134
:10AAE80028271646194640250CE007FB03F000F519
:10AAF8008C7022182354D3805670D1709560D16021
:10AB08005161013362789342EFD300232826194616
:10AB180040250CE006FB03F000F55C702218235476
:10AB2800D3805170D1709560D160516101336278E2
:10AB38009342EFD32046FFF739FC2046FFF7BEFBD0
:10AB480000212046FFF770FC2046FFF7C3FC204693
:10AB5800BDE8F840FFF723BC70B5CDB20C464FF006
:10AB6800280601F07F0106FB010115F0800F14BFD4
:10AB780001F58C7101F55C7104F07F04ED090C702E
:10AB88004D708A60CB7005B1CC80022B01D10023B7
:10AB98000B71FFF743FD002070BD10B5CAB201F07C
:10ABA8007F034FF0280404FB030312F0800F14BF47
:10ABB80003F58C7303F55C7301F07F01D2091970FA
:10ABC8005A701946FFF759FD002010BD38B501F03D
:10ABD8007F0528246C4304F55C7401194B6100233C
:10ABE8008B614B70EBB20355CA60C478012C08BF67
:10ABF8000A6113B9FFF7E6FD01E0FFF75DFD0020EC
:10AC080038BD70B501F07F042825654305F58C75BE
:10AC180041190126E4B2CA600A6100224E70445507
:10AC28008A614B6114B9FFF7CDFD01E0FFF744FDE0
:10AC3800002070BDCAB212F0800F10B54FF0280383
:10AC480006D001F07F0403FB040303F58C7303E0D3
:10AC580003FB010303F55C73D209012401F07F01B2
:10AC680019709C705A701946FFF719FE002010BD24
:10AC7800CAB212F0800F10B54FF0280306D001F0C9
:10AC88007F0403FB040303F58C7303E003FB010358
:10AC980003F55C730024D20901F07F0119709C70E0
:10ACA8005A701946FFF713FE204610BD08B50B066B
:10ACB80004D501F07F01FFF780FB01E0FFF79AFB65
:10ACC800002008BD0369002261F30A1219680A43CB
:10ACD8001A60704703695A6803206FF341025A608B
:10ACE800FFF73CBA03695A68032042F002025A602F
:10ACF800FFF734BA11F0800F4FF0280306D001F0A7
:10AD08007F0103FB010101F58C7103E003FB0101E5
:10AD180001F55C71FFF775BE11F0800F4FF0280345
:10AD280006D001F07F0103FB010101F58C7103E0FE
:10AD380003FB010101F55C71FFF790BE2DE9F74FA8
:10AD48000446FFF78BFB002800F03F822046FFF700
:10AD580092FB0546002800F03882C0F3074000F057
:10AD68000800C0B2002861D02046FFF7C5FDA14603
:10AD7800824627464FF00008DFF86CB32E4650E0B5
:10AD88001AF0010F46D05FFA88F211462046009269
:10AD9800FFF7B8FD10F0010F0546009A20D07B6D33
:10ADA80001259D60E178A94207D11B69D9F878137C
:10ADB800C3F31203CB1AC9F88833DBF800302046F6
:10ADC8001B6811469847E378012B09D1B8F1000FA9
:10ADD80006D194F81131052B02D12046FFF7A0FDCA
:10ADE80005F00203DBB213B17B6D02259D6005F00F
:10ADF8000403DBB213B17B6D04259D6005F00805E3
:10AE0800EDB23DB1DBF8003020469B6898477B6D7A
:10AE18000820986008F101084FEA5A0A043709F136
:10AE28002809BAF1000FABD135460120C5F3074315
:10AE380003F00403DBB2002B00F0AF802046FFF7DD
:10AE480069FD264683464FF0000801959FE01BF0F8
:10AE5800010F00F0978023695FFA88F919695D6B23
:10AE680004EB890225FA09F59269ED019268EDB2C1
:10AE78000D431540EA071CD55A6B012000FA08F16A
:10AE880022EA01025A63B369974A98601368054633
:10AE98005B68204649469847E378AB4209D1B8F148
:10AEA800000F06D194F81131042B02D12046FFF788
:10AEB80037FD05F00403DBB213B1B36904259D60C7
:10AEC80005F00803DBB213B1B36908259D6005F0EE
:10AED8001003DBB213B1B36910259D6005F02003A0
:10AEE800DBB213B1B36920259D6005F04003DBB2E6
:10AEF80013B1B36940259D6005F00203DBB213B1BD
:10AF0800B36902259D6025F07F0515F0FF0F39D044
:10AF1800282505FB084505F58C75C246AB696A69A5
:10AF2800C3EB020CAB689C4528BF9C460CF1030C94
:10AF3800B3694FEA9C0C9B696746A04614E0AA686F
:10AF4800E9681C1B944228BF1446A3B240464A46EF
:10AF5800FFF72EF9EB681B19EB60AB69E71C1C19AE
:10AF6800AC61B3699B69BF089BB2BB4205D9AC69A8
:10AF78006B699C4201D2002BE1D1B369802544461C
:10AF88009D60D04608F101084FEA5B0B0436BBF11F
:10AF9800000F7FF45CAF019D012005F00203DBB2D6
:10AFA80013B1E36802225A61C5F3076303F0800313
:10AFB800DBB2CBB1A37A43B1D4F80C31D4F80C216D
:10AFC8006FF341036FF30003136023695A6822F09B
:10AFD80001025A60444B1B6820469B699847E36806
:10AFE8004FF000425A610120C5F3072303F008031C
:10AFF800DBB2F3B13C4B1B6820465B699847236979
:10B00800E2689B684FF400615161A27A82B1DB0764
:10B018000ED5D4F80C311A6842F001021A601A6889
:10B0280042F003021A60314B1A6942F006021A61B3
:10B03800012005F00803DBB243B12B4B1B68204607
:10B04800DB689847E36808225A61012005F010037D
:10B05800DBB2002B33D0E3689A6922F010029A61C0
:10B068001F6A282607F00F0306FB0346C7F343436E
:10B07800022B06F55C7602D0062B1AD10EE047F6B5
:10B08800F0733B40ABB1C7F30A172046F1683A4664
:10B09800FFF7A2F8F368DB19F36007E004F5B9617C
:10B0A80020460822FFF798F8C7F30A17B369DF1993
:10B0B800B761E3689A6942F010029A610120C5F30A
:10B0C800072303F01003DBB2002B39D023695A6839
:10B0D800002622F001025A6031462046FFF76DF93A
:10B0E80023463246FF2108E04C02002000ED00E034
:10B0F80058698160186D013281606078043382423A
:10B10800F6D3236901274FF0FF3267F30F069A61E0
:10B1180067F31F460F22DE615A612F221A611A68EF
:10B128006FF30A121A602046FFF7FAFBE3684FF440
:10B1380080525A61264B1B6820461B69984738463F
:10B14800C5F3072303F02003DBB2EBB12046FFF77A
:10B158004FFAE3682046DE68FFF73CFA032806D179
:10B168000023A3704FF40073A380092304E0012394
:10B17800A3704023A380052363F38D26E3684FF46F
:10B188000052DE6001205A61C5F3074303F0100343
:10B19800DBB24BB10E4B1B682046DB699847E3686E
:10B1A8004FF480125A610120C5F3074505F02005C8
:10B1B800EDB255B1064B1B6820461B6A9847E368F9
:10B1C8004FF400125A610120FFE7BDE8FE8F00BF6F
:10B1D8004C02002043230B8000487047BC0100202C
:10B1E80038B51F4B1A68511C052A196035D11979D1
:10B1F800002201291A6030D09968B1F5006F08BFA4
:10B208009A60174B9968DC68A1421A4602D100225D
:10B218001A7122E086BFC1F500631361C1EB040413
:10B22800D0F8EC3598BF14611569B3F839300C4C77
:10B238009D428AB204D95918ED1AA160256104E02B
:10B248006918A1600021ABB22161054901240C7184
:10B2580004498A188121FFF7D4FC002038BD00BFBB
:10B26800B80D00209B46002038B528230A4D03FB63
:10B2780001010A4BB1F888131B6904462846984710
:10B28800D4F8EC352046B3F8403001212A46FFF7C0
:10B298009DFC002038BD00BF534600203802002026
:10B2A80070B50B7813F0600506460C4625D0202DA6
:10B2B8001FD1CD88B5B113F0800F487808D0214B45
:10B2C80021499B682A469847E2881F49304625E06D
:10B2D8001E4B1D4958641E4B30465D612A4600F0DE
:10B2E80022FB1DE0174B48789B6829462A46984759
:10B2F80025E000F077FB022521E04B780A2B11D0DE
:10B308000B2B14D0062B1AD14B881B0A212B03D1E7
:10B31800CA883A2A28BF3A220E49304600F0EAFA8B
:10B3280000250CE00C49012200F0E4FA07E08B78D4
:10B338001BB9074A1D46936101E000F053FB2846FC
:10B3480070BD00BF3802002093460020BC010020D9
:10B35800B80D0020CE010020D00D002010B58121AD
:10B368000446FFF71AFC01212046FFF716FC82214C
:10B378002046FFF712FC024B5B689847002010BD7F
:10B388003802002038B5D0F8EC350446B3F8392037
:10B3980081210223FFF7E0FBD4F8EC350121B3F853
:10B3A800402020460223FFF7D7FB822108220323EF
:10B3B8002046FFF7D1FB094B022200251A715D7167
:10B3C800074B1B689847D4F8EC35064AB3F8403069
:10B3D80020460121FFF7FAFB284638BD7C020020F1
:10B3E800380200205346002010B5074C606CFF2837
:10B3F80007D0064B064A9B68064952699847FF23BF
:10B408006364002010BD00BFBC010020380200208A
:10B41800B80D00209346002038B510490B79012B50
:10B4280019D10C690CB90C7115E0D0F8EC358D68A0
:10B43800B3F839309C42AAB203D95D198D60E41A79
:10B4480003E0A3B22C198C6000240C610449521843
:10B458008121FFF7D6FB002038BD00BFB80D0020C2
:10B468009B46002000207047002070470023F0B55D
:10B47800084A094E1D4609E01468C75C375501346F
:10B488000133B4F5006F146008BF15608B42F3D127
:10B498000020F0BDC40D00209B460020104B114A2F
:10B4A800D3F800C000232DE9F0410F4F16461D4682
:10B4B8000DE0146810F8038007F804800134802C2C
:10B4C80008BF2C4614603468644505D001338B42AC
:10B4D800EFD10020BDE8F0810220BDE8F08100BF77
:10B4E8001C4F0020304F00209C4E002021280FD1F7
:10B4F800084B1A680A701A68120A4A705A888A70C1
:10B50800DA78CA701A790A715A794A719B798B71FB
:10B51800002070473002002007B502AB012103F874
:10B52800010D1846FFF7A2FF0EBD002100E0013112
:10B53800435C002BFBD199E798E70B4B0B491A6842
:10B54800096891420BD00A498A5C02701A68013274
:10B55800802A1A6005D100221A6001207047002055
:10B5680070470120704700BF1C4F0020304F00205B
:10B578009C4E0020204B1A68204B1B689A42F0B55D
:10B5880009D135E00133802B08BF00239A4203D14B
:10B598001A4B1A602CE01A4CE15C0029F2D00A29F7
:10B5A800F0D00D29EED0154C1549134D23600E46E9
:10B5B8000023CF182268BA5CC254226801339F184E
:10B5C800802F08BF53422F689A18974210D0B25C58
:10B5D8001AB10A2A01D00D2AEBD10022C254074A17
:10B5E800116859187F29116003D98039116000E06A
:10B5F80000231846F0BD00BF304F00201C4F00202C
:10B608009C4E0020704700BFD0F8E43510B51B6988
:10B6180004469847032384F81231002010BD08B56A
:10B62800042380F81231D0F8E435DB68984700200D
:10B6380008BD08B5D0F8E035DB6903B198470020AC
:10B6480008BD08B5D0F8E0351B6A9847002008BD4A
:10B6580008B5D0F8E0355B6A9847002008BD00219E
:10B6680010B5402204460B46FFF776FA80214022A7
:10B6780000232046FFF770FA012384F81231D4F82A
:10B68800E435A0785B689847002010BD13B569467B
:10B69800044600F085F99DF8001001F01F03012B06
:10B6A80007D0022B0AD073B92046694600F026FA63
:10B6B8000FE02046694600F007FA0AE0204669468E
:10B6C80000F0A2F905E021F07F01C9B22046FFF79A
:10B6D800B1FA00201CBD38B5044600293DD190F8C8
:10B6E8001131022B42D1D0F83421D0F820319A42BE
:10B6F80011D9C178D21A0129C0F8342104D1D0F85F
:10B708002411CB18C0F8243192B22046D4F8241161
:10B7180000F000F92AE0D0F83821B2FBF3F503FB7A
:10B72800152565B99A420AD3D0F83C319A4206D217
:10B7380029462A4600F0EEF8C4F83C5116E0D4F841
:10B74800E035DB682BB194F81221032A01D1204699
:10B758009847204600F00FF908E0D0F8E0355B691B
:10B7680023B190F81221032A00D19847002038BD50
:10B7780010B5044659BB90F81131032B30D1D0F8DD
:10B788008C23D0F878339A4214D9C178D21A012977
:10B79800C0F88C2304D1D0F87C13C918C0F87C13E6
:10B7A8009A4228BF1A4692B22046D4F87C1300F079
:10B7B800CAF815E0D0F8E0351B6923B190F81221DA
:10B7C800032A00D19847204600F0C6F808E0D0F8D0
:10B7D800E0359B6923B190F81221032A00D19847DC
:10B7E800002010BD2DE9F041069F044616469846F4
:10B7F8000D46FEF741FC20462946C4F8E085C4F80A
:10B80800E475C4F8E865FFF761F9D4F8E4351B6816
:10B8180098472046BDE8F041FEF782BC00207047FB
:10B82800D0F8E03510B504461B689847D4F8E435DD
:10B838009B689847002010BD08B5D0F8E0355B68D4
:10B848009847002008BD000012230B80004870476D
:10B858007C02002004230B80004870478E020020E1
:10B8680010B5044C04480A46214600F075FA2046F3
:10B8780010BD00BF344F00201E9F05080A4608B5BA
:10B888000248034900F068FA014808BD319F0508DD
:10B89800344F00200A4608B50248034900F05CFA14
:10B8A800014808BD3F9F0508344F002008B50A46E7
:10B8B80008B9044800E00448044900F04DFA034878
:10B8C80008BD00BF4A9F0508579F0508344F002050
:10B8D80008B50A4608B9044800E00448044900F0DD
:10B8E8003BFA034808BD00BF649F0508859F05080B
:10B8F800344F002010B513460C46C0F83821C0F864
:10B908003421022280F8112100212246FFF779F91B
:10B91800002010BD10B50C46134600212246FFF743
:10B9280070F9002010BD10B513460C46C0F89023DE
:10B93800C0F88C23032280F8112100212246FFF74A
:10B9480045F9002010BD10B50C46134600212246CB
:10B95800FFF73CF9002010BD0021042310B50A466A
:10B96800044680F811310B46FFF74BF92046FEF7E5
:10B97800D7FF002010BD0021052310B50A46044654
:10B9880080F811310B46FFF721F92046FEF7C8FF72
:10B99800002010BD282303FB0100B0F8880370477E
:10B9A80090F8C8350B7090F8C9354B7090F8CB25D6
:10B9B80090F8CA3503EB02234B8090F8CD2590F818
:10B9C800CC3503EB02238B8090F8CF2590F8CE3549
:10B9D80003EB02239BB2CB80C0F83C31012380F8F3
:10B9E8001131704710B591F90030002B044601DB86
:10B9F800CB880BB9802100E00021FFF71BF9204616
:10BA0800BDE81040FEF78CBF38B50D4604466B788C
:10BA18000979012B10D027D3032B51D190F812317B
:10BA2800022B28D0032B47D16B889BB991B1802971
:10BA380010D0FFF7FFF80DE090F81231022B1AD062
:10BA4800032B39D16B88002B3AD149B1802907D013
:10BA5800FFF70EF9D4F8E03520469B682946984749
:10BA68002046FFF779FF2BE090F81231022B02D025
:10BA7800032B21D106E019B3802921D02046FFF7F6
:10BA8800D9F81DE011F0800F4FF0280306D001F01F
:10BA98007F0103FB010393F81A2103E003FB010173
:10BAA80091F87223074B02B101221A60204605491A
:10BAB8000222FFF71FFF03E020462946FFF792FF07
:10BAC800002038BDD40D002038B590F81231032B72
:10BAD80004460D460CD10B79012B09D8D0F8E03576
:10BAE8009B689847EB883BB92046FFF735FF03E092
:10BAF80020462946FFF776FF002038BD73B54B78FE
:10BB080004460D46092B00F21C81DFE813F0D10032
:10BB180008011A01E4001A0172000A001A01C000A3
:10BB280092004B881A0A013A062A00F20A81DFE8D5
:10BB380012F007001A00270008010801080108018F
:10BB4800D4F8E835A0781B680DF106019847EB8812
:10BB5800402B014603D094F81231012B3AD1082327
:10BB6800ADF8063036E0D4F8E035A0789B6A0DF1E0
:10BB780006019847022343700146C4F8EC0529E002
:10BB8800DBB2052B00F2DD80DFE803F003080D12BD
:10BB9800171CD4F8E835A0785B6817E0D4F8E835C6
:10BBA800A0789B6812E0D4F8E835A078DB680DE04F
:10BBB800D4F8E835A0781B6908E0D4F8E835A0780F
:10BBC8005B6903E0D4F8E835A0789B690DF10601BC
:10BBD80098470146BDF80630002B00F0B680EA8889
:10BBE800002A00F0B2809A4228BF1A46ADF8062013
:10BBF8005CE08B88002B40F0A480CB88002B40F0C1
:10BC0800A08094F812214B88032A00F09A8003F050
:10BC18007F05204684F813512946FFF753F820463C
:10BC2800FFF79AFE0DB1022300E0012384F81231D8
:10BC38008BE08978464E0129317100F2828094F8B0
:10BC48001231022B02D0032B7BD108E0002962D0ED
:10BC58000121032384F8101184F8123113E041B94B
:10BC6800022384F8123184F810112046FFF7E4FD0E
:10BC780051E094F81011012920464DD0FFF7DCFD62
:10BC8800317984F810112046FFF7CAFD43E0CA88CD
:10BC9800012A56D194F81231022B02D0032B50D12D
:10BCA80002E020462B4913E004F5887120460FE096
:10BCB80094F81231023B012B43D8D4F814312449AB
:10BCC800002B0CBF0123032341F80C3F204601221F
:10BCD800FFF710FE39E04B88012B29D0022B34D115
:10BCE8008B8813F0FF0F30D121691B0A013B4A688A
:10BCF800042B0FD8DFE803F0030507090B00012325
:10BD080006E0022304E0032302E0042300E0052305
:10BD180063F306124A602046FFF71EFE15E094F80A
:10BD28001231023B012B0CD84B88012B0DD100237B
:10BD3800C4F81431D4F8E03520469B682946984762
:10BD4800E9E720462946FFF74DFE00207CBD00BFED
:10BD5800D40D0020DC0D002030B5C8B10023DDB2C1
:10BD68000133C41814F8014C002CF8D16B1C5B008B
:10BD780013800B7003234B70022305E0CA545A1C2E
:10BD8800D2B202338C54DBB210F8012B002AF5D161
:10BD980030BD00BF704770477047704770477047A5
:10BDA800704700000EB403B070470A2810B5044667
:10BDB80002D10D20FFF7F9FF064A13681BB103F8FB
:10BDC800014B136010BD044B1B680BB1204698470C
:10BDD80010BD00BFE40D0020684F002010B50446D8
:10BDE80001E0FFF7E2FF14F8010B0028F9D110BDBC
:10BDF8002DE9F04F044685B00D464FF00A0A00E0E1
:10BE080035462078002800F0C480252801D0013468
:10BE180067E06078302803D1A0780123033407E075
:10BE28002D2802D00234002302E0A0780223033434
:10BE38004FF0000805E00AFB080814F8010BA8F108
:10BE48003008A0F13002D2B2092AF4D96C2801D006
:10BE58004C2803D114F8010B43F00403002800F028
:10BE68009880602886BFA0F12002D2B202464F2AED
:10BE78003DD006D8432A2DD0442A09D0422A30D1B1
:10BE880033E0552A04D0582A29D0532A29D101E071
:10BE98000A272DE02E1D2F68002500E001357A5D68
:10BEA800002AFBD104E02020FFF77FFF4D4601E088
:10BEB800980704D4454505F10109F4D34D463846A1
:10BEC800FFF78CFF03E02020FFF76FFF01354545A2
:10BED800F9D395E728782E1DFFF767FF90E710271D
:10BEE80006E0FFF762FF2E468AE7022700E00827F0
:10BEF8002E1D442A296804D1002902DA494243F058
:10BF08000803002200E02A46B1FBF7FE07FB1E11DA
:10BF1800CDB2092D714607D9782814BF4FF0070C08
:10BF28004FF0270C6544EDB230350DF80250551C22
:10BF3800BEF1000F02D0102DE5D10F22190705D54B
:10BF480004A94D192D2105F8101C951C13F0010F9B
:10BF58000CBF4FF0200B4FF0300B9B072F4604D53A
:10BF680008E05846FFF721FF4F46474507F101090A
:10BF7800F7D34F46013D1DF80500FFF716FF002DCA
:10BF8800F8D103E02020FFF710FF01374745F9D328
:10BF980036E705B0BDE8F08F70B5064D0C462E6843
:10BFA800286001E0FFF701FF14F8010B0028F9D120
:10BFB8002E6070BD684F00200FB407B504A951F872
:10BFC800040B0191FFF714FFBDE80E4004B0704761
:10BFD8000EB417B505A9084C51F8043B2060184663
:10BFE8000191FFF705FF2268002313702360BDE865
:10BFF8001E4003B0704700BFE40D00200EB433B5F7
:10C0080005A9074C51F8043B2568206018460191A2
:10C01800FFF7EEFE2560BDE83C4003B0704700BF67
:10C02800684F002070B51E4604461C481546FFF7A9
:10C03800C3FF022E1FD0042E25D0012E2AD105E0E1
:10C04800A15D1748FFF7B8FF013600E00026AE42B1
:10C05800F6DB2020FFF7A9FE002609E0A05DA0F18D
:10C068002003DBB25E2B88BF2E20FFF79EFE013631
:10C07800AE42F3DB0EE034F8021B0A48FFF79CFFE0
:10C08800013DF8D106E054F8041B0748FFF794FF78
:10C09800013DF8D10A20BDE8704086E6A69F050854
:10C0A800AD9F0508B39F0508B99F050808B501218C
:10C0B8004FF4807001F07CFA4FF480700021BDE8E5
:10C0C800084001F075BA43680A6823F0407323F406
:10C0D800807313430A7943EA02234360CA680B69F1
:10C0E80030B51A4384688D68084B2A4323401343AC
:10C0F8004A7943EA420383600B7DC26A013B22F41A
:10C108007002DBB242EA0353C36230BDFDF7FFC0E1
:10C1180000230360037143718360C36003610123DB
:10C1280003757047074A084B516810B50B4090E8F3
:10C13800120021438468C068214301430B435360C4
:10C1480010BD00BF00230140E030FCFF0023036066
:10C1580043608360C3607047836811B143F0010393
:10C1680001E023F0010383607047436823F4400330
:10C1780023F400730B434360704741628262704747
:10C18800436823F01F030B4343607047044B5A680E
:10C1980010B142F4000201E022F400025A60704734
:10C1A80000230140044B5A6810B142F4800201E0B8
:10C1B80022F480025A60704700230140092970B5B3
:10C1C8000CB20CD904EB44041E3CC6680725A540F4
:10C1D80026EA0505A34045EA0304C4600AE00669A7
:10C1E80004EB44040725A54026EA050513FA04F4E0
:10C1F8002C430461062A0CD80523013A5A43446BA0
:10C208001F23934024EA0303914043EA0102426357
:10C2180070BD0C2A12B20CD802EB8202233A046BCE
:10C228001F23934024EA0303914043EA0102026377
:10C2380070BD02EB8202413AC46A1F23934024EA8C
:10C248000303914043EA0102C26270BD836843F070
:10C258008043836070478068C0F38050704783686C
:10C2680011B143F4806301E023F480638360704775
:10C27800836811B143F0020301E023F002038360F5
:10C2880070474368013923F4604343EA413343600C
:10C298007047436811B143F4006301E023F400637D
:10C2A80043607047C06C80B27047014B1868704794
:10C2B80008230140836811B143F4807301E023F43B
:10C2C800807383607047836811B143F4007301E0A1
:10C2D80023F4007383607047044B5A6810B142F42A
:10C2E800005201E022F400525A60704700230140D6
:10C2F800092970B50CB20CD904EB44041E3CC6687D
:10C308000725A54026EA0505A34045EA0304C460BD
:10C318000AE0066904EB44040725A54026EA05055A
:10C3280013FA04F42C430461836BC3F30154121B06
:10C338000232D2B202EB82021F24944023EA0403A1
:10C3480091400B43836370BD836B013923F4401321
:10C3580043EA01538363704782B00023019301903D
:10C36800019BCB180193019B1A6002B07047836848
:10C3780023F470230B4383607047836823F44013CE
:10C388000B4383607047836843F48003836070477E
:10C398008068C0F380507047436811B143F48063EC
:10C3A80001E023F4806343607047436811B143F4AC
:10C3B800805301E023F480534360704782B0002328
:10C3C80001930190019B28335B180193019B186826
:10C3D80080B202B070470123C9B213FA01F1436871
:10C3E8000AB1194301E023EA01014160704703687B
:10C3F80019420CBF002001207047C94301607047F3
:10C408004368006810EA112007D00122C9B212FA65
:10C4180001F119420CBF0020012070476FEA112179
:10C4280001607047036823F0010303600023036081
:10C4380043608360C3600361212343612C4B9842AE
:10C448001CD02C4B984220D02B4B984225D02B4BFC
:10C4580098422AD02A4B98422FD02A4B984233D060
:10C46800294B984237D0294B984204D14FF03D527E
:10C4780043F8AC2C7047264B984203D13D2243F831
:10C48800082C7047234B984204D14FF4746243F848
:10C49800202C7047204B984204D14FF4741243F873
:10C4A800382C70471D4B984204D14FF0746243F802
:10C4B800502C70471A4B984203D11A4A43F8642CFF
:10C4C8007047194B984203D1184A43F87C2C70479F
:10C4D800174B984203D1174A43F8942C7047164BD0
:10C4E800984204BF4FF03D5243F8AC2C704700BF50
:10C4F80010600240286002404060024058600240DC
:10C508007060024088600240A0600240B86002404B
:10C5180010640240286402404064024058640240AB
:10C52800706402403D00002088640240400F0020F3
:10C53800A064024000003D20B86402400268134B2A
:10C5480010B51340CC680A6822434C6922438C69B1
:10C558002243CC6922430C6A22434C6A22438C6AE8
:10C5680022434C6B22438C6B224313430360426982
:10C578000C6BCB6A22F007022343134343610B6918
:10C5880043604B6883608B68C36010BD3F801CF0BC
:10C598000023036043608360C36003614361836178
:10C5A800C361036243628362C36203634363836359
:10C5B8007047036811B143F0010301E023F0010360
:10C5C80003607047036811B143F4004301E023F4AA
:10C5D800004303607047036811B143F0200301E092
:10C5E80023F020030360704741607047406880B2C1
:10C5F8007047036812B143F4002301E023F40023D9
:10C60800036001617047036811B143F4802301E0BE
:10C6180023F48023036070470AB101617047C16049
:10C6280070470068C0F3C0407047006800F0010020
:10C638007047406900F0380070470A4A0A4B10B545
:10C648000A4CA04288BF13468A004CBF5B681B682F
:10C6580021F0F02121F0821119420CBF00200120A5
:10C6680010BD00BF00640240006002400F64024039
:10C6780010B5084B084A094CA04288BF134611F070
:10C68800005F21F0F02121F0821114BFD960996078
:10C6980010BD00BF00600240006402400F64024009
:10C6A8000B0607D5436912B143F0800301E023F07C
:10C6B80080034361802909D001F01E01036812B18B
:10C6C80019430160704723EA010101607047124B6A
:10C6D800124A10B5124CA0428CBF14461C4621F0D9
:10C6E800F02323F0C3132BB1026802F01E0202EA02
:10C6F800D12202E0426902F0800288004CBF6368E0
:10C70800236821F0F02121F08210184002D0101C7B
:10C7180018BF012010BD00BF006002400064024045
:10C728000F64024010B5084B084A094CA04288BF64
:10C73800134611F0005F21F0F02121F0821114BF9F
:10C74800D960996010BD00BF0060024000640240DB
:10C758000F640240044B00221A605A609A60DA6043
:10C76800024A5A61704700BF003C0140FFFF7F004A
:10C77800837910B5002B29D01A4B01681C68CA436D
:10C7880014401C605C6822405A60027902F18042C1
:10C7980002F59E3214682143116002689C68D143F7
:10C7A8000C409C60DC682140D9604179102906D191
:10C7B800996811439960D9680A43DA6010BD01F19C
:10C7C800804303F59E3319680A4308E0037901683A
:10C7D80003F1804303F59E331A6822EA01021A60C6
:10C7E80010BD00BF003C014000230C220360037110
:10C7F800427183717047024B1A6902431A6170478C
:10C80800003C0140034B5B6918420CBF002001202B
:10C81800704700BF003C0140014B5861704700BFA2
:10C82800003C0140054B1A685B69034004D0104284
:10C838000CBF00200120704718467047003C01409B
:10C84800014B5861704700BF003C01404FF0204346
:10C8580018B943F2DB021A6003E043F2D20243F84C
:10C8680020204FF02042411C6FF0704342F82130E5
:10C8780002F5827242F82030704770B584684568C6
:10C88800C368C16A026825431D4303691D434369A0
:10C898001D4383691D43C3691D43036A1D43436ADE
:10C8A8001D43836A1D43036B0D431D434FF0204313
:10C8B800082C43F8225005D153F8224044F0400494
:10C8C80043F82240436B9E691D6835435E6845EA1C
:10C8D80006159E6845EA0625DE6845EA06451E698E
:10C8E8005B6945EA0655541C45EA03654FF0204349
:10C8F800B1F5804F43F8245010D1836B98691968BB
:10C908000143586841EA0011986841EA0021186912
:10C918005B6941EA005141EA036101E06FF070414F
:10C92800014B43F8221070BD040100A002224260AE
:10C938004FF480524262416B4FF4005210B582624C
:10C9480000230F22FF2403608360C36003614361F7
:10C958008361C3610362C36203630A604A608C60D7
:10C96800CA600A614A618B61816B0A604A608C60A7
:10C97800CA600A614A618B6110BD4FF0204321B142
:10C9880053F8202042F0010203E053F82010024A35
:10C998000A4043F820207047FEFF0F0010280CBF04
:10C9A800064B074B4FF040024FF0180119605A60D0
:10C9B8004FF0FC329A60DA60704700BF600000A058
:10C9C800800000A030B5836844681C43C36844F005
:10C9D80008041C4303691C43436944EA43248369EC
:10C9E80044EA4334C36999685A68090441EA022150
:10C9F8001A68DB68114341EA0361036A9A685D6853
:10CA0800120442EA05221D68DB682A4342EA0362EF
:10CA18000368102B0CBF034B034B1C609960DA6052
:10CA280030BD00BF600000A0800000A0102303609C
:10CA3800C269002343608360C3600361436183610B
:10CA4800FC23136053609360D360026A13605360E1
:10CA58009360D360704741B110280CBF074B084B57
:10CA68001A6842F004021A60704710280CBF034A83
:10CA7800034A044B11680B4013607047600000A024
:10CA8800800000A0FBFF0F0041B110280CBF084B2D
:10CA9800084B1A6842F040021A60704710280CBF11
:10CAA800034A044A044B11680B401360704700BFE7
:10CAB800600000A0800000A0BFFF0F00102802D176
:10CAC800024B58697047024B58697047600000A0D4
:10CAD800800000A0054B18221A6000225A604FF00F
:10CAE800FC329A60DA601A61704700BFA00000A0AB
:10CAF8000268436842F0100242EA4322836842EA2D
:10CB08004332144B10B51A60C2689168546809041E
:10CB180041EA04211468D268214341EA02629A601A
:10CB2800026991685468090441EA04211468D268CA
:10CB3800214341EA0262DA60426991685068090457
:10CB480041EA00211068D268014341EA02621A6191
:10CB580010BD00BFA00000A0C268002303604360AE
:10CB68008360FC23136053609360D3600269136091
:10CB780053609360D3604269136053609360D360DD
:10CB88007047054B18B11A6842F0040202E01968B0
:10CB9800024A0A401A607047A00000A0FBFF0F007D
:10CBA80062B1102801D10E4B03E0B0F5807F03D1AC
:10CBB8000C4B5A68114311E00B4BFAE7102804D1CB
:10CBC800074B5A6822EA010108E0B0F5807F0CBFE4
:10CBD800044B054B5A686FEA0101114059607047D0
:10CBE800600000A0800000A0A00000A0102801D1D3
:10CBF800064B04E0B0F5807F0CBF054B054B5B6826
:10CC08000B420CBF00200120704700BF600000A04D
:10CC1800800000A0A00000A0102804D1074B5A688B
:10CC280022EA010108E0B0F5807F0CBF044B054BF8
:10CC38005A686FEA0101114059607047600000A00E
:10CC4800800000A0A00000A0102801D1084B04E03B
:10CC5800B0F5807F0CBF074B074B5B6813EA0100F8
:10CC680004D013EAD1010CBF00200120704700BF97
:10CC7800600000A0800000A0A00000A0102804D13F
:10CC8800084B5A6822EAD10109E0B0F5807F0CBF51
:10CC9800054B064B5A684FEAD10122EA0101596057
:10CCA800704700BF600000A0800000A0A00000A0A6
:10CCB80008B52C4B984205D10120014600F048FCEC
:10CCC800012048E0284B984205D10220012100F0BC
:10CCD8003FFC02203FE0254B984205D1042001216A
:10CCE80000F036FC042036E0214B984205D108209C
:10CCF800012100F02DFC08202DE01E4B984205D1A3
:10CD08001020012100F024FC102024E01A4B984246
:10CD180005D12020012100F01BFC20201BE0174B2F
:10CD2800984205D14020012100F012FC402012E079
:10CD3800134B984205D18020012100F009FC802086
:10CD480009E0104B98420BD14FF48070012100F09C
:10CD5800FFFB4FF480700021BDE8084000F0F8BBED
:10CD680008BD00BF00000240000402400008024065
:10CD7800000C02400010024000140240001802405B
:10CD8800001C0240002002402DE9F0470023D1F8A2
:10CD980000801A464FF0010C03270CFA02F404EA4B
:10CDA8000805A5422ED1066817FA03F4E443264085
:10CDB80006600E79D0F8009006FA03FA013E4AEAB6
:10CDC8000909012EC0F8009014D8866891F80590DA
:10CDD80026408660866809FA03F949EA06068660ED
:10CDE800466826EA050545608D7946689540ADB2E6
:10CDF80035434560C5682C40C460CC79C5689C4003
:10CE08002C43C46001320233102AC6D1BDE8F08732
:10CE18004FF6FF7303600023037143718371C3717D
:10CE2800704782B04FF480330193019B0B43019309
:10CE3800019BC361C161019BC361C3690193C3695C
:10CE4800019302B07047036919420CBF002001200A
:10CE58007047006980B27047436919420CBF0020CF
:10CE680001207047406980B2704701837047418351
:10CE780070470AB101837047418370474161704729
:10CE880043694B404361704701F00703C908083103
:10CE980030B59B0050F821500F249C4025EA04042B
:10CEA80040F8214050F8214012FA03F31C4340F89F
:10CEB800214030BD08B5134B984207D14FF40010FC
:10CEC800012100F069FB4FF4001014E00E4B98426A
:10CED80007D14FF48000012100F05EFB4FF4800081
:10CEE80009E00A4B98420BD14FF40000012100F0F1
:10CEF80053FB4FF400000021BDE8084000F04CBB94
:10CF080008BD00BF0054004000580040005C0040CD
:10CF18007FB50446868868460D4600F06DFA02998A
:10CF28002C482B6826F03F063604B1FBF0F0360C8F
:10CF380080B20643A680228822F001021204120C55
:10CF48002280254A93420AD85B00B1FBF3F30130F3
:10CF58009BB280B22084032B98BF042321E0EE8883
:10CF68004BF6FF72964205D103225343B1FBF3F30C
:10CF78009BB206E019225343B1FBF3F39BB243F48F
:10CF880080431A054FF4967208BF43F001035043DB
:10CF98004FF47A7290FBF2F0013080B243F4004310
:10CFA8002084A38323886989AA889BB243F001035C
:10CFB8002380238823F4816323F002031B040A439C
:10CFC8001B0C13439BB223802A89AB8913439BB262
:10CFD80023817FBD40420F00A086010041F28833C3
:10CFE8000360002383804BF6FF72038143814FF473
:10CFF8008043C28083817047038819B19BB243F094
:10D00800010303E023F001031B041B0C038070479A
:10D01800038819B19BB243F4807303E023F480734F
:10D028001B041B0C03807047038819B19BB243F49F
:10D03800007303E023F400731B041B0C0380704788
:10D0480012B141F0010101E001F0FE0101827047D7
:10D05800038819B19BB243F4806303E023F480632F
:10D068001B041B0C0380704783899BB201F0FE01EF
:10D0780023F0FE030B4383817047838919B19BB268
:10D0880043F0010303E023F001031B041B0C83811D
:10D098007047038819B19BB243F0400303E023F0C3
:10D0A80040031B041B0C03807047038829B16FEAF7
:10D0B80043436FEA53439BB201E05B045B0C03807C
:10D0C8007047038819B99BB243F0800303E023F04B
:10D0D80080031B041B0C03807047B1F5804F838BC2
:10D0E80004D023F480431B041B0C02E09BB243F4DE
:10D0F800804383837047B1F5006F038803D19BB2E7
:10D1080043F4006303E023F400631B041B0C038057
:10D118007047B1F5005F038803D19BB243F4005315
:10D1280003E023F400531B041B0C0380704703889F
:10D1380019B19BB243F0100303E023F010031B0462
:10D148001B0C0380704701827047008AC0B2704789
:10D15800038819B19BB243F4805303E023F480534E
:10D168001B041B0C03807047B1F5006F038803D1C3
:10D178009BB243F4006303E023F400631B041B0C1D
:10D1880003807047038819B19BB243F0200303E082
:10D1980023F020031B041B0C03807047008BC0F393
:10D1A80007207047838819B19BB243F4006303E0FA
:10D1B80023F400631B041B0C83807047838819B118
:10D1C8009BB243F4805303E023F480531B041B0CED
:10D1D8008380704782B0002301930190019BCB1894
:10D1E8000193019B188880B202B0704783889BB274
:10D1F8000AB1194301E023EA010181807047838A5B
:10D20800008B9BB243EA0040084020F07F40431A5D
:10D21800584240EB03007047838A008B9BB243EA75
:10D22800004020F07F40704782B0002300930193B4
:10D238000B0F01900093009B21F07F4113B1019BDC
:10D24800143302E0019B090C18330193019B1B68FE
:10D2580019420CBF0020012002B07047C94389B2AF
:10D26800818270478388808A80B208409BB206D04A
:10D2780001F0E06113EA11410CBF00200120704762
:10D28800C94389B2818270470A4B1A6842F0010289
:10D298001A6000229A60196821F0847121F48031A3
:10D2A800196005495960196821F480211960DA600C
:10D2B800704700BF0038024010300024024B0022A3
:10D2C8001A701870704700BF02380240034B1A6882
:10D2D80022F0F80242EAC0021A60704700380240A1
:10D2E800014B1860704700BF00004742064B002200
:10D2F80001281A701A7002D0042804D101E01870AD
:10D30800704705221A70704770380240014B186048
:10D31800704700BF800E4742014341EA82120099DC
:10D328005B08013B42EA016141EA0341014B596054
:10D33800704700BF00380240014B1860704700BFBB
:10D34800600047428001034B40EA0171C3F8841032
:10D35800704700BF00380240014B1860704700BF9B
:10D3680068004742014B1860704700BF4C004742B5
:10D37800034B9A6822F0EC6202430A439A607047B2
:10D3880000380240034B9A6822F0784202430A436D
:10D398009A60704700380240034B9A6822F00302F3
:10D3A80002439A60704700BF00380240024B9868F9
:10D3B80000F00C00704700BF00380240034B9A6829
:10D3C80022F0F00202439A60704700BF0038024022
:10D3D800034B9A6822F4E05202439A60704700BFF8
:10D3E80000380240034B9A6822F4604242EAC002C5
:10D3F8009A607047003802401E4B9A6802F00C028F
:10D40800042A10B503D0082A03D01B4B18E01B4B85
:10D4180016E059685A6811F4800F596814BF174B01
:10D42800154B02F03F02B3FBF2F3124A5268C2F303
:10D438000142C1F3881101324B435200B3FBF2F3AE
:10D448000C4903608B680E4A0468C3F30313D35C6A
:10D4580034FA03F343608C68C4F38224145D33FA0E
:10D4680004F484608968C1F34231525CD340C360DC
:10D4780010BD00BF003802400024F40000127A00FA
:10D48800D402002000F44073B3F5407F084B08D164
:10D49800996820F0704221F4F81122F440720A438E
:10D4A8009A601A6F000542EA10501867704700BF6B
:10D4B80000380240014B1860704700BF3C0E4742DD
:10D4C800014B1860704700BF400E4742014B18607F
:10D4D800704700BF5C014742044B1A6B09B1104307
:10D4E80001E022EA00001863704700BF00380240DC
:10D4F800044B5A6B09B1104301E022EA000058635B
:10D50800704700BF00380240044B9A6B09B11043C2
:10D5180001E022EA00009863704700BF003802402B
:10D52800044B1A6C09B1104301E022EA00001864A8
:10D53800704700BF00380240044B5A6C09B11043D1
:10D5480001E022EA00005864704700BF003802403A
:10D55800044B1A6909B1104301E022EA000018617E
:10D56800704700BF00380240044B5A6909B11043A4
:10D5780001E022EA00005861704700BF003802400D
:10D58800044B9A6909B1104301E022EA000098614E
:10D59800704700BF00380240044B1A6A09B11043B3
:10D5A80001E022EA00001862704700BF003802401C
:10D5B800044B5A6A09B1104301E022EA000058629C
:10D5C800704700BF00380240044B1A6D09B1104380
:10D5D80001E022EA00001865704700BF00380240E9
:10D5E800044B5A6D09B1104301E022EA0000586566
:10D5F800704700BF00380240044B9A6D09B11043D0
:10D6080001E022EA00009865704700BF0038024038
:10D61800044B1A6E09B1104301E022EA00001866B3
:10D62800704700BF00380240044B5A6E09B11043DE
:10D6380001E022EA00005866704700BF0038024047
:10D64800044B1A7809B1104301E022EA000018706F
:10D65800704700BF0D3802404309012B074A01D12A
:10D66800136803E0022B0CBF136F536F00F01F0009
:10D6780033FA00F000F00100704700BF00380240A4
:10D6880007B5002301933120FFF7E6FF019B013323
:10D698000193019BB3F5A06F01D00028F3D031208E
:10D6A800FFF7DAFF003018BF01200EBD024B5A6F9A
:10D6B80042F080725A67704700380240034BDB68BB
:10D6C80018420CBF00200120704700BF00380240FC
:10D6D800014B1870704700BF0E38024008B5154B53
:10D6E80098420BD101214FF48050FFF761FF4FF4AE
:10D6F80080500021BDE80840FFF75ABF0E4B984202
:10D7080007D14FF480400121FFF746FF4FF48040D6
:10D7180009E00A4B98420BD14FF400400121FFF772
:10D728003BFF4FF400400021BDE80840FFF734BF3D
:10D7380008BD00BF0030014000380040003C0040F8
:10D748000B88028810B54C8823438C882343CC88E7
:10D7580023430C8923434C8923438C892343CC8955
:10D7680002F44152234313439BB20380838B23F477
:10D7780000631B041B0C83830B8A038210BD838BFD
:10D7880023F47B6323F00F031B041B0C8383022306
:10D7980003848B68F0B5858B022BADB238D0294A4B
:10D7A8008E889468002E14BF02260126240203D511
:10D7B800946824F400049460D2F88440D2F8847009
:10D7C8005268DFF884C002F03F02BCFBF2F2C4F3F7
:10D7D80088145443C7F30272B4FBF2F4CA88B2F552
:10D7E800007F4FF00A0201D1240A02E07601B4FB5F
:10D7F800F6F46243B2FBF3F305330A229BB2B3FBA0
:10D80800F2F303F001021202C3F34F0392B200E0F5
:10D8180000229C1EA4B2FE2C28BF0022CC8828BF60
:10D828000223134323439BB203840B884A882B4368
:10D8380043F4006313438A8813438A8913439BB2D2
:10D848008383F0BD0038024000127A000023038071
:10D8580043808380C380038143818381C3810723FD
:10D868000382704700230222038043808380C380A1
:10D87800826083817047038819B19BB243F04003EB
:10D8880003E023F040031B041B0C03807047838BC9
:10D8980019B19BB243F4806303E023F480631B0453
:10D8A8001B0C83837047038823F400631B041B0C41
:10D8B800038003889BB20B4303807047B1F5804F08
:10D8C800038803D19BB243F4804303E023F48043ED
:10D8D8001B041B0C038070474FF6FF6399420388B3
:10D8E80003D09BB243F4807303E023F480731B04DA
:10D8F8001B0C03807047838819B19BB243F0040363
:10D9080003E023F004031B041B0C83807047838807
:10D9180019B19BB243F0100303E023F010031B047A
:10D928001B0C83807047838B23F47B6323F00F03E6
:10D938001B041B0C8383022303840B88828BB3F59F
:10D94800007F10B592B205D0002B0CBF4FF4807346
:10D95800002301E04FF480734C8822438C88898926
:10D9680042F4006222430A4392B21343838310BDF8
:10D97800808980B2704781817047038819B19BB252
:10D9880043F4005303E023F400531B041B0C0380EF
:10D99800704703889BB243F4805303807047012982
:10D9A80002D0008B80B27047808A80B27047008AAC
:10D9B80080B2704783889BB20AB1194301E023EA19
:10D9C800010181807047090901238B409BB21AB17C
:10D9D800828892B2134303E0828892B222EA030358
:10D9E80083807047038919420CBF002001207047CB
:10D9F800C94389B20181704710B584880089012321
:10DA080001F00F0280B213FA02F21040A4B205D05E
:10DA180009098B401C420CBF0020012010BD01F0F9
:10DA28000F0101238B40DB439BB20381704700BF8A
:10DA380008B501214FF48040FFF7BAFD4FF480404C
:10DA48000021BDE80840FFF7B3BD014B18607047DF
:10DA58000038014001F0030289080A4B023130B551
:10DA6800920053F821500F24944025EA040443F807
:10DA7800214053F8214010FA02F2144343F82140A0
:10DA880030BD00BF00380140014B1860704700BF2F
:10DA9800DC002742014B1860704700BF0004274292
:10DAA800024B186AC0F30020704700BF00380140DD
:10DAB80030B5048C24F001042404240C0484058B60
:10DAC800048CADB2A4B225F0F305154324F00A0482
:10DAD80045EA031544F00104ADB20C430583048400
:10DAE80030BD30B5048C24F010042404240C0484C4
:10DAF800048B058C24F44074ADB22405240D25F064
:10DB0800A00544EA022445F0100544EA033445EA36
:10DB18000115A4B2ADB20483058430BD08B5474BE6
:10DB2800984205D101200146FFF742FD01203DE062
:10DB3800B0F1804F05D101200146FFF72DFD0120EE
:10DB480076E03F4B984205D102200121FFF724FDE2
:10DB580002206DE03B4B984205D104200121FFF7DC
:10DB68001BFD042064E0384B984205D108200121B0
:10DB7800FFF712FD08205BE0344B984205D11020D6
:10DB88000121FFF709FD102052E0314B984205D1E1
:10DB980020200121FFF700FD202049E02D4B98426D
:10DBA80009D102200121FFF703FD02200021BDE871
:10DBB8000840FFF7FDBC284B984207D14FF480304E
:10DBC8000121FFF7F5FC4FF48030EFE7234B984233
:10DBD80007D14FF400300121FFF7EAFC4FF4003081
:10DBE800E4E71F4B984207D14FF480200121FFF74B
:10DBF800DFFC4FF48020D9E71A4B984205D140202A
:10DC08000121FFF7C9FC402012E0174B984205D1CB
:10DC180080200121FFF7C0FC802009E0134B9842C7
:10DC28000BD14FF480700121FFF7B6FC4FF48070E0
:10DC38000021BDE80840FFF7AFBC08BD0000014067
:10DC48000004004000080040000C004000100040A4
:10DC5800001400400004014000400140004401401D
:10DC68000048014000180040001C0040002000400F
:10DC78001C4A038890429BB212D002F580629042FF
:10DC88000ED0B0F1804F0BD0A2F58032904207D071
:10DC980002F58062904203D002F58062904203D17F
:10DCA8004A8823F0700313430F4A904208D002F5C4
:10DCB8008062904204D023F440730A899BB21343D4
:10DCC80003804B68C3620B880385064B984203D0D8
:10DCD80003F58063984201D18B7A038601238382FE
:10DCE800704700BF00000140001000404FF0FF33B4
:10DCF800436000230380038143808372704701855A
:10DD080082827047038823F070031B041B0C0B43AB
:10DD18000380704741627047C1627047406A70472C
:10DD2800008D80B27047038819B19BB243F002039B
:10DD380003E023F002031B041B0C038070470388D5
:10DD480019B19BB243F0040303E023F004031B045E
:10DD58001B0C03807047038819B19BB243F0800302
:10DD680003E023F080031B041B0C03807047038827
:10DD780023F008031B041B0C038003889BB20B438E
:10DD880003807047038823F440731B041B0C038033
:10DD980003889BB20B4303807047038819B19BB279
:10DDA80043F0010303E023F001031B041B0C038071
:10DDB8007047038C23F001031B041B0C038470B50C
:10DDC800038C8488028B0D884E8822F0730212041B
:10DDD800120C2A438D8923F002031B0435431B0CC4
:10DDE800ADB22B430E4DA842A4B203D005F5806511
:10DDF800A8420ED1CD894E8A23F008032B438D8883
:10DE080023F004032B430D8A354324F44074ADB248
:10DE18002C43848002838A684263038470BD00BFF8
:10DE280000000140038C23F010031B041B0C038427
:10DE3800038C828830B5048B0D8824F4E6442404CE
:10DE4800240C23F0200344EA05241B048D891B0CB1
:10DE580043EA05134D8843EA0513134DA84292B2CD
:10DE6800A4B29BB203D005F58065A84215D1CD892F
:10DE780023F080039BB243EA05134FF6BF751D409C
:10DE88008B8845EA03130D8A22F4406242EA850230
:10DE98004D8A42EA85029BB292B282808A680483E4
:10DEA8008263038430BD00BF00000140038C23F46B
:10DEB80080731B041B0C0384038C828830B5848B0D
:10DEC8000D8824F073042404240C23F400731B0429
:10DED8002C438D891B0C43EA05234D8843EA05230F
:10DEE800124DA84292B29BB203D005F58065A842B4
:10DEF80015D1CD8923F400639BB243EA05234FF67D
:10DF0800FF351D408B8845EA03230D8A22F44052D1
:10DF180042EA05124D8A42EA05129BB292B2828009
:10DF28008A688483C263038430BD00BF0000014057
:10DF3800038C23F480531B041B0C0384038C30B51F
:10DF48008488828B0D8822F4E6421204120C23F492
:10DF5800005342EA05221B048D891B0C43EA053352
:10DF68004D8843EA05330B4DA842A4B292B29BB246
:10DF780003D005F58065A84205D10D8A24F48044B4
:10DF880044EA8514A4B2848082838A680264038484
:10DF980030BD00BF00000140002303804380838020
:10DFA80083608381C38103824382704730B5058CC7
:10DFB8000124ADB28C4025EA040400F1180304845E
:10DFC80009B1082907D149084FF68F70CC5820406D
:10DFD800C850C8580AE00439C1F34E0148F6FF702A
:10DFE800CC582040C8501202C85892B20243CA50B6
:10DFF80030BD4163704781637047C16370470164F6
:10E008007047038B23F070031B041B0C0B43038323
:10E018007047038B23F4E0431B041B0C43EA0123E2
:10E028009BB203837047838B23F070031B041B0C84
:10E038000B4383837047838B23F4E0431B041B0C3F
:10E0480043EA01239BB283837047038B23F00803C1
:10E058001B041B0C0B4303837047038B23F40063DF
:10E068001B041B0C43EA01239BB203837047838B79
:10E0780023F008031B041B0C0B4383837047838B1B
:10E0880023F400631B041B0C43EA01239BB2838324
:10E098007047038B23F004031B041B0C0B430383FF
:10E0A8007047038B23F480631B041B0C43EA012392
:10E0B8009BB203837047838B23F004031B041B0C60
:10E0C8000B4383837047838B23F480631B041B0CEF
:10E0D80043EA01239BB283837047038B23F08003B9
:10E0E8001B041B0C0B4303837047038B09025B045F
:10E0F80041EA53439BB203837047838B23F0800329
:10E108001B041B0C0B4383837047838B09025B043E
:10E1180041EA53439BB283837047038C23F0020385
:10E128001B041B0C0B4303847047038C23F0080368
:10E138001B041B0C0B4303847047038C23F0200340
:10E148001B041B0C43EA01139BB203847047038C26
:10E1580023F080031B041B0C43EA01139BB20384C6
:10E168007047038C23F400731B041B0C43EA012340
:10E178009BB203847047038C23F400631B041B0CBD
:10E1880043EA01239BB203847047038C23F40053B2
:10E198001B041B0C43EA01339BB20384704710B580
:10E1A800048C01238B40A4B224EA03030384038C68
:10E1B80012FA01F10B439BB2038410BD10B5048C15
:10E1C80004238B40A4B224EA03030384038C12FAC9
:10E1D80001F10B439BB2038410BD0023012203808D
:10E1E80043808280C38003817047406B7047806B97
:10E1F8007047C06B7047006C7047038B23F00C03AB
:10E208001B041B0C0383038B9BB20B4303837047D4
:10E21800038B23F440631B041B0C0383038B9BB207
:10E2280043EA01239BB203837047F8B50C4649883B
:10E23800A288B4F800E02389054600290CBF02270C
:10E248000027012A14BF01260226BEF1000F10D1B3
:10E25800FFF72EFC2846E188FFF7CFFF284639460E
:10E2680032462389FFF73DFCE1882846BDE8F8409F
:10E27800CEE7FFF736FC2846E188FFF7C9FF2846B6
:10E28800394632462389FFF713FCE1882846BDE862
:10E29800F840B2E7838B23F00C031B041B0C838329
:10E2A800838B9BB20B4383837047838B23F4406338
:10E2B8001B041B0C8383838B9BB243EA01239BB211
:10E2C80083837047F8B50D460B88AA8849880446A9
:10E2D8003BB92B89FFF7ECFBE9882046BDE8F840FD
:10E2E8008BE7042B07D12B89FFF7FBFBE988204636
:10E2F800BDE8F8408CE7082BB5F808C0078C1DD19D
:10E3080027F480773F043F0C0784868B038CB6B2D2
:10E318009BB226F0F30623F4206346EA0C1C43EA7A
:10E3280001211FFA8CFC89B24CEA020241F4807187
:10E3380082830184E988BDE8F840ABE727F4805779
:10E348003F043F0C0784868B038C26F4407623F425
:10E35800005336055B04360D5B0C46EA022243EA9D
:10E36800013342EA0C329BB2E98892B243F48053FB
:10E3780082830384BDE8F84097E74A880B881343F3
:10E388008A881343CA8813430A8913434A89134363
:10E398008A8913439BB2A0F8443070470023038056
:10E3A80043808380C3800381438183817047B0F8B1
:10E3B800443029B16FEA43436FEA53439BB201E00B
:10E3C8005B045B0CA0F844307047838819B19BB29A
:10E3D80043F0040303E023F004031B041B0C8380B5
:10E3E8007047838819B19BB243F0010303E023F01F
:10E3F80001031B041B0C8380704783899BB20AB1FD
:10E40800194301E023EA0101818170478182704745
:10E41800038A19420CBF002001207047C94389B202
:10E4280001827047038A828911EA030092B203D0FD
:10E4380011420CBF002001207047C94389B20182F4
:10E4480070470A43A0F84820704783899BB20AB1F5
:10E45800194301E023EA010181817047838819B1DA
:10E468009BB243F0080303E023F008031B041B0CD2
:10E4780083807047038923F007031B041B0C038167
:10E488007047038923F070031B041B0C0B430381A3
:10E4980003899BB243F007030381704738B50D46E3
:10E4A80011460122602D044602D1FFF71AFB01E054
:10E4B800FFF7FEFA238923F070031B041B0C1D438E
:10E4C800258123899BB243F00703238138BD038943
:10E4D80023F070031B041B0C0B43038170478388D4
:10E4E80023F070031B041B0C838083889BB20B43AF
:10E4F80083807047038923F007031B041B0C0381E7
:10E5080003899BB20B4303817047038923F080037F
:10E518001B041B0C038103899BB20B4303817047C7
:10E5280010B50489E4B20C43144344EA0324A4B2AA
:10E53800048110BD10B50446FFF7F2FF23899BB292
:10E5480043F48043238110BD10B50446FFF7E8FF6C
:10E55800238923F077031B041B0C43F077032381E3
:10E5680010BD70B50489068B058C26F44076ADB2D3
:10E5780026F0030624F00704360425F022052404B7
:10E58800360C1543240C46F4807645EA03152143DE
:10E5980046F00106ADB201810683058470BD83880B
:10E5A80019B19BB243F0800303E023F080031B04FE
:10E5B8001B0C83807047A0F85010704708B5234B98
:10E5C800984205D110200121FEF7F2FF102037E014
:10E5D8001F4B984207D14FF400300121FEF7DCFFB2
:10E5E8004FF4003009E01B4B98420BD14FF48020C8
:10E5F8000121FEF7D1FF4FF480200021BDE808403B
:10E60800FEF7CABF144B984207D14FF400200121EE
:10E61800FEF7C2FF4FF40020EFE7104B984207D1F6
:10E628004FF480100121FEF7B7FF4FF48010E4E7A4
:10E638000B4B984209D120200121FEF7B9FF202079
:10E648000021BDE80840FEF7B3BF08BD0010014037
:10E658000044004000480040004C0040005000408A
:10E6680000140140038ACA889BB223F4405330B592
:10E6780013430D46038283890989AA8823F4B0537A
:10E688000A43698923F00C031B040A431B0C92B24A
:10E6980013438381838AAA899BB223F4407313436B
:10E6A80085B0838204466846FEF7A6FE1A4B9C4254
:10E6B80003D003F580639C4201D1039B00E0029BD9
:10E6C800A28912B2002A4FF019012A6801FB03F14E
:10E6D80001DA520000E092006423B1FBF2F1B1FBD1
:10E6E800F3F21201100903FB1011A08900B20028EF
:10E6F80006DAC9003231B1FBF3F303F0070305E092
:10E7080009013231B1FBF3F303F00F031A4392B25C
:10E71800228105B030BD00BF001001404FF41653F0
:10E7280003600C2200238380C3800381428183819C
:10E7380070470B88028A10B54C8823438C88C98897
:10E74800234392B20B4322F470629BB213430382B9
:10E7580010BD0023038043808380C3807047838972
:10E7680019B19BB243F4005303E023F400531B0494
:10E778001B0C83817047038B03F47F430383038B54
:10E788009BB20B4303837047838929B16FEA4343E4
:10E798006FEA53439BB201E05B045B0C83817047D3
:10E7A800838A19B19BB243F4006303E023F4006346
:10E7B8001B041B0C83827047C905C90D81807047F3
:10E7C8008088C005C00D7047038A23F00F031B041F
:10E7D8001B0C0382038A9BB20B4303827047838915
:10E7E80019B19BB243F0020303E023F002031B04B8
:10E7F8001B0C83817047838923F400631B041B0C63
:10E80800838183899BB20B4383817047038A23F0FA
:10E8180020031B041B0C0382038A9BB20B43038255
:10E828007047038A19B19BB243F4804303E023F491
:10E8380080431B041B0C0382704783899BB243F0FF
:10E84800010383817047838A19B19BB243F008039F
:10E8580003E023F008031B041B0C83827047038B1F
:10E86800DBB20383038B9BB243EA01230383704724
:10E87800838A19B19BB243F0200303E023F02003FD
:10E888001B041B0C83827047838A19B19BB243F027
:10E89800100303E023F010031B041B0C8382704752
:10E8A800838A23F004031B041B0C8382838A9BB294
:10E8B8000B4383827047838A19B19BB243F00203EA
:10E8C80003E023F002031B041B0C83827047838A36
:10E8D8009BB20AB1194301E023EA01018182704722
:10E8E800C1F3421310B501F01F01012414FA01F11C
:10E8F800A34201D10C3004E0022B01D1103000E01A
:10E90800143003680AB1194301E023EA01010160E8
:10E9180010BD038819420CBF002001207047C9436D
:10E9280089B201807047012210B501F01F03C1F3BD
:10E9380042149A40012C01D1838903E0022C0CBFB8
:10E94800038A838A9BB21340028892B243B1090AB0
:10E95800012313FA01F111420CBF0020012010BD60
:10E96800184610BD090A01238B40DB439BB2038084
:10E97800704700BF81F0004102E000BF83F0004310
:10E9880030B54FEA41044FEA430594EA050F08BF42
:10E9980090EA020F1FBF54EA000C55EA020C7FEA06
:10E9A800645C7FEA655C00F0E2804FEA5454D4EB83
:10E9B8005555B8BF6D420CDD2C4480EA020281EA4D
:10E9C800030382EA000083EA010180EA020281EA85
:10E9D8000303362D88BF30BD11F0004F4FEA0131D7
:10E9E8004FF4801C4CEA113102D0404261EB4101E6
:10E9F80013F0004F4FEA03334CEA133302D052426C
:10EA080063EB430394EA050F00F0A780A4F1010427
:10EA1800D5F1200E0DDB02FA0EFC22FA05F2801861
:10EA280041F1000103FA0EF2801843FA05F3594147
:10EA38000EE0A5F120050EF1200E012A03FA0EFCC6
:10EA480028BF4CF0020C43FA05F3C01851EBE371F0
:10EA580001F0004507D54FF0000EDCF1000C7EEB0D
:10EA680000006EEB0101B1F5801F1BD3B1F5001F4B
:10EA78000CD349085FEA30004FEA3C0C04F101046A
:10EA88004FEA445212F5800F80F09A80BCF1004F93
:10EA980008BF5FEA500C50F1000041EB045141EA15
:10EAA800050130BD5FEA4C0C404141EB010111F416
:10EAB800801FA4F10104E9D191F0000F04BF0146C1
:10EAC8000020B1FA81F308BF2033A3F10B03B3F19F
:10EAD80020020CDA0C3208DD02F1140CC2F10C022F
:10EAE80001FA0CF021FA02F10CE002F11402D8BF8D
:10EAF800C2F1200C01FA02F120FA0CFCDCBF41EA59
:10EB08000C019040E41AA2BF01EB0451294330BD27
:10EB18006FEA04041F3C1CDA0C340EDC04F1140404
:10EB2800C4F1200220FA04F001FA02F340EA0300DB
:10EB380021FA04F345EA030130BDC4F10C04C4F121
:10EB4800200220FA02F001FA04F340EA0300294601
:10EB580030BD21FA04F0294630BD94F0000F83F44B
:10EB6800801306BF81F480110134013D4EE77FEA2E
:10EB7800645C18BF7FEA655C29D094EA050F08BF7A
:10EB880090EA020F05D054EA000C04BF194610465B
:10EB980030BD91EA030F1EBF0021002030BD5FEA9F
:10EBA800545C05D14000494128BF41F0004130BDC7
:10EBB80014F580043CBF01F5801130BD01F000451B
:10EBC80045F0FE4141F470014FF0000030BD7FEA8E
:10EBD800645C1ABF194610467FEA655C1CBF0B4689
:10EBE800024650EA013406BF52EA033591EA030FA0
:10EBF80041F4002130BD00BF90F0000F04BF002198
:10EC0800704730B54FF4806404F132044FF00005CA
:10EC18004FF0000150E700BF90F0000F04BF002143
:10EC2800704730B54FF4806404F1320410F00045A9
:10EC380048BF40424FF000013EE700BF42004FEAA4
:10EC4800E2014FEA31014FEA02701FBF12F07F4321
:10EC580093F07F4F81F06051704792F0000F14BF1E
:10EC680093F07F4F704730B54FF4607401F0004562
:10EC780021F0004120E700BF50EA010208BF7047B9
:10EC880030B54FF000050AE050EA010208BF7047AE
:10EC980030B511F0004502D5404261EB41014FF417
:10ECA800806404F132045FEA915C3FF4DCAE4FF01B
:10ECB80003025FEADC0C18BF03325FEADC0C18BF02
:10ECC800033202EBDC02C2F1200300FA03FC20FA53
:10ECD80002F001FA03FE40EA0E0021FA02F11444A0
:10ECE800C1E600BF70B54FF0FF0C4CF4E06C1CEAB5
:10ECF80011541DBF1CEA135594EA0C0F95EA0C0F2A
:10ED080000F0DEF82C4481EA030621EA4C5123EA9C
:10ED18004C5350EA013518BF52EA033541F48011CB
:10ED280043F4801338D0A0FB02CE4FF00005E1FB7E
:10ED380002E506F00042E0FB03E54FF00006E1FBC8
:10ED480003569CF0000F18BF4EF0010EA4F1FF040B
:10ED5800B6F5007F64F5407404D25FEA4E0E6D414B
:10ED680046EB060642EAC62141EA55514FEAC5205C
:10ED780040EA5E504FEACE2EB4F1FD0C88BFBCF5D8
:10ED8800E06F1ED8BEF1004F08BF5FEA500E50F189
:10ED9800000041EB045170BD06F0004646EA01014F
:10EDA80040EA020081EA0301B4EB5C04C2BFD4EB81
:10EDB8000C0541EA045170BD41F480114FF0000E7A
:10EDC800013C00F3AB8014F1360FDEBF002001F0E8
:10EDD800004170BDC4F10004203C35DA0C341BDC62
:10EDE80004F11404C4F1200500FA05F320FA04F034
:10EDF80001FA05F240EA020001F0004221F0004168
:10EE080010EBD37021FA04F642EB06015EEA430EDA
:10EE180008BF20EAD37070BDC4F10C04C4F120050A
:10EE280000FA04F320FA05F001FA04F240EA0200BD
:10EE380001F0004110EBD37041F100015EEA430E8E
:10EE480008BF20EAD37070BDC4F1200500FA05F2AE
:10EE58004EEA020E20FA04F301FA05F243EA02032D
:10EE680021FA04F001F0004121FA04F220EA02003C
:10EE780000EBD3705EEA430E08BF20EAD37070BD82
:10EE880094F0000F0FD101F00046400041EB010162
:10EE980011F4801F08BF013CF7D041EA060195F044
:10EEA800000F18BF704703F00046520043EB0303FE
:10EEB80013F4801F08BF013DF7D043EA06037047EB
:10EEC80094EA0C0F0CEA135518BF95EA0C0F0CD0F6
:10EED80050EA410618BF52EA4306D1D181EA03013C
:10EEE80001F000414FF0000070BD50EA410606BF36
:10EEF8001046194652EA430619D094EA0C0F02D17B
:10EF080050EA013613D195EA0C0F05D152EA0336BF
:10EF18001CBF104619460AD181EA030101F00041DD
:10EF280041F0FE4141F470014FF0000070BD41F026
:10EF3800FE4141F4780170BD70B54FF0FF0C4CF400
:10EF4800E06C1CEA11541DBF1CEA135594EA0C0F1F
:10EF580095EA0C0F00F0A7F8A4EB050481EA030E6C
:10EF680052EA03354FEA013100F088804FEA033353
:10EF78004FF0805545EA131343EA12634FEA022221
:10EF880045EA111545EA10654FEA00260EF00041E2
:10EF98009D4208BF964244F1FD0404F5407402D234
:10EFA8005B084FEA3202B61A65EB03055B084FEAC5
:10EFB80032024FF480104FF4002CB6EB020E75EBC2
:10EFC800030E22BFB61A754640EA0C005B084FEAEA
:10EFD8003202B6EB020E75EB030E22BFB61A754667
:10EFE80040EA5C005B084FEA3202B6EB020E75EBB2
:10EFF800030E22BFB61A754640EA9C005B084FEA2A
:10F008003202B6EB020E75EB030E22BFB61A754636
:10F0180040EADC0055EA060E18D04FEA051545EA25
:10F0280016754FEA06164FEAC30343EA52734FEACE
:10F03800C2025FEA1C1CC0D111F4801F0BD141EA47
:10F0480000014FF000004FF0004CB6E711F4801FAC
:10F0580004BF01430020B4F1FD0C88BFBCF5E06F8C
:10F068003FF6AFAEB5EB030C04BFB6EB020C5FEA9C
:10F07800500C50F1000041EB045170BD0EF0004EF1
:10F088004EEA113114EB5C04C2BFD4EB0C0541EA23
:10F09800045170BD41F480114FF0000E013C90E620
:10F0A80045EA060E8DE60CEA135594EA0C0F08BFE4
:10F0B80095EA0C0F3FF43BAF94EA0C0F0AD150EAE3
:10F0C80001347FF434AF95EA0C0F7FF425AF104676
:10F0D80019462CE795EA0C0F06D152EA03353FF49E
:10F0E800FDAE1046194622E750EA410618BF52EA1B
:10F0F80043067FF4C5AE50EA41047FF40DAF52EAEF
:10F1080043057FF4EBAE12E74FF0FF3C06E000BF8B
:10F118004FF0010C02E000BF4FF0010C4DF804CD98
:10F128004FEA410C7FEA6C5C4FEA430C18BF7FEA58
:10F138006C5C1BD001B050EA410C0CBF52EA430C86
:10F1480091EA030F02BF90EA020F0020704710F106
:10F15800000F91EA030F58BF994208BF90422CBF95
:10F16800D8176FEAE37040F0010070474FEA410C8E
:10F178007FEA6C5C02D150EA013C07D14FEA430CAC
:10F188007FEA6C5CD6D152EA033CD3D05DF8040B1D
:10F19800704700BF8446104662468C46194663464F
:10F1A80000E000BF01B5FFF7B7FF002848BF10F126
:10F1B800000F01BD4DF808EDFFF7F4FF0CBF01206B
:10F1C80000205DF808FB00BF4DF808EDFFF7EAFFE7
:10F1D80034BF012000205DF808FB00BF4DF808EDA2
:10F1E800FFF7E0FF94BF012000205DF808FB00BF97
:10F1F8004DF808EDFFF7CEFF94BF012000205DF821
:10F2080008FB00BF4DF808EDFFF7C4FF34BF01202D
:10F2180000205DF808FB00BF4FEA410212F500121A
:10F2280015D211D56FF47873B3EB625212D94FEA45
:10F23800C12343F0004343EA505311F0004F23FA2F
:10F2480002F018BF404270474FF00000704750EA84
:10F25800013005D111F0004008BF6FF00040704741
:10F268004FF00000704700BF4A0011D212F500129B
:10F2780011D20DD56FF47873B3EB62520ED44FEA06
:10F28800C12343F0004343EA505323FA02F0704786
:10F298004FF00000704750EA013002D14FF0FF30C4
:10F2A80070474FF0000070474FEA4102B2F1E04367
:10F2B80024BFB3F5001CDCF1FE5C0DD901F0004C55
:10F2C8004FEAC0024CEA5070B2F1004F40EB8300A5
:10F2D80008BF20F00100704711F0804F21D113F1D1
:10F2E8003872BCBF01F00040704741F480114FEA0A
:10F2F8005252C2F11802C2F1200C10FA0CF320FA93
:10F3080002F018BF40F001004FEAC1234FEAD323AF
:10F3180003FA0CFC40EA0C0023FA02F34FEA430319
:10F32800CCE77FEA625307D150EA01331EBF4FF0A2
:10F33800FE4040F44000704701F0004040F0FE40BD
:10F3480040F40000704700BF4BB942B9002908BF1C
:10F35800002802D04FF0FF31084600F037B882B0DD
:10F36800EC462DE9005000F01BF8DDF804E002B08F
:10F378000CBC7047F8B5144606460F461D4600F00B
:10F3880027F804FB01F300FB0535A4FB0023EB1869
:10F39800069CB21A67EB0303C4E90023F8BD00BF5B
:10F3A800F8B5144606460F461D4600F075F900FBF1
:10F3B80005F5A0FB042304FB0155EB18069CB21AC3
:10F3C80067EB0303C4E90023F8BD00BF704700BF23
:10F3D80000292DE9F0071D46C0F29E800024002D6B
:10F3E800C0F2958007460D4616469C46002B3ED136
:10F3F8008A4254D9B2FA82F343B1C3F1200620FA03
:10F4080006F501FA03F19A4029439840160CB1FB1E
:10F41800F6F597B206FB15114FEA104C07FB05F3FA
:10F428004CEA01418B4209D9891805F1FF3C80F06B
:10F4380015818B4240F21281023D8918C3EB010C01
:10F44800BCFBF6F306FB13C180B207FB03F740EAE7
:10F458000140874207D9591E821880F005819742DA
:10F4680040F20281023B43EA0542002303E08B425B
:10F478000AD900231A461046194614B1404261EBD6
:10F488004101BDE8F0077047B3FA83F3002B40F061
:10F4980087808C4501D38242ECD80122EBE712B970
:10F4A8000123B3FBF2F2B2FA82F6002E3AD1891A9E
:10F4B800150C1FFA82FC0123B1FBF5F705FB1711A8
:10F4C8004FEA10480CFB07F648EA01418E4207D97B
:10F4D800891807F1FF3802D28E4200F2DA804746D7
:10F4E800891BB1FBF5F605FB161180B20CFB06FC77
:10F4F80040EA0140844507D9711E821880F0B08027
:10F50800944540F2AD80023E46EA0742B3E7E44341
:10F51800524263EB430365E7404261EB41014FF020
:10F52800FF345CE7B240C6F1200521FA05F320FA62
:10F5380005F701FA06F9150CB3FBF5F847EA0909CE
:10F548001FFA82FC05FB18374FEA19410CFB08F338
:10F5580041EA0747B040BB420AD9BF1808F1FF315A
:10F5680080F09580BB4240F29280A8F10208BF1853
:10F57800FE1AB6FBF5F305FB13611FFA89F90CFBBC
:10F5880003F649EA01418E4206D95F1E891878D2EE
:10F598008E4276D9023B8918891B43EA08438BE7D8
:10F5A800C3F1200726FA07F80CFA03F248EA020C1E
:10F5B80021FA07F105FA03FA4FEA1C4920FA07F580
:10F5C800B1FBF9F845EA0A0509FB18172A0C1FFAD6
:10F5D8008CFA0AFB08F142EA0747B94206FA03F631
:10F5E80009D917EB0C0708F1FF324ED2B9424CD9B2
:10F5F800A8F1020867447F1AB7FBF9F209FB1271F8
:10F60800ADB20AFB02FA45EA01418A4507D9551EFF
:10F6180011EB0C0137D28A4535D9023A614442EAE6
:10F6280008424FEA124C1FFA86F808FB0CF7360C12
:10F6380095B208FB05F806FB057505EB184506FBB2
:10F648000CFCAF4288BF0CF5803CCAEB01010CEB07
:10F658001546B14212D309D000230CE76546EDE602
:10F668000E4646EA074206E70B46FCE61FFA88F80C
:10F6780000FA03F308EB0545AB42EDD2013A00234B
:10F68800F9E63B4688E72A46C9E79046B3E7884645
:10F698006EE7023F891823E72DE9F00F1446054667
:10F6A8000E46002B3FD18A424AD9B2FA82F343B1BF
:10F6B800C3F1200025FA00F201FA03F69C40164334
:10F6C8009D40210CB6FBF1F22F0CA0B201FB126C8D
:10F6D80000FB02F347EA0C46B34208D9571E361915
:10F6E80080F0FF80B34240F2FC80023A3619F61AE5
:10F6F800B6FBF1F301FB1361ADB200FB03F045EA81
:10F708000141884207D95E1E091980F0EC808842C1
:10F7180040F2E980023B43EA0242002310461946C0
:10F72800BDE8F00F70478B4243D8B3FA83F4002C3E
:10F7380042D18B42234601D382423BD80122EDE7D6
:10F7480012B90123B3FBF2F4B4FA84F2002A40F0B0
:10F758008A80091B260CA7B20123B1FBF6F006FB31
:10F7680010114FEA154C07FB00F24CEA01418A429E
:10F7780007D9091900F1FF3C02D28A4200F2D3806E
:10F788006046C2EB010CBCFBF6F206FB12C1ADB23F
:10F7980007FB02F745EA0145AF4207D9511E2C196C
:10F7A80080F0A380A74240F2A080023A42EA0042D9
:10F7B800B4E700231A46B1E7C4F1200722FA07F696
:10F7C80003FA04F3334321FA07FA4FEA134C01FA18
:10F7D80004FB20FA07F141EA0B0BBAFBFCF70CFB20
:10F7E80017A61FFA83F84FEA1B4508FB07F945EAF5
:10F7F8000645A94502FA04FA04D97A1EED18C0F0A4
:10F8080088801746C9EB0505B5FBFCF60CFB1652BC
:10F818001FFA8BFB08FB06F84BEA0241884503D91F
:10F82800721EC91870D3164646EA0742170C1FFA0B
:10F838008AFC0CFB07F695B24FEA1A430CFB05FC51
:10F8480003FB056505EB1C4503FB07F3AE4288BFC8
:10F8580003F58033C8EB010103EB1543994250D3FC
:10F8680047D000235AE79440C2F12008260C20FA1A
:10F8780008F721FA08F501FA02F9B5FBF6F847EAA4
:10F88800090906FB1855A7B24FEA194C4CEA054C72
:10F8980007FB08F3634500FA02F509D91CEB040CD1
:10F8A80008F1FF323DD263453BD9A8F10208A444D0
:10F8B800C3EB0C02B2FBF6F306FB13201FFA89F91F
:10F8C80007FB03F249EA00418A4206D9581E091982
:10F8D80025D28A4223D9023B0919891A43EA0843E7
:10F8E8003BE73A4603E7334615E70A4642EA004251
:10F8F80014E71FFA8CF100FA04F001EB0545A84261
:10F90800AFD2013A002309E788458CD9023EC918CD
:10F918008AE7A9457FF675AF023FED1872E70346FF
:10F92800DBE79046C4E7023809192AE7002103E01B
:10F938000A4B5B584350043109480A4B42189A4213
:10F94800F6D3094A02E0002342F8043B074B9A42E7
:10F95800F9D3FAF7D1F900F00DF87047BCA40508FF
:10F9680000000020A40B0020A80B0020704F0020EE
:10F97800FEE700009D4BF7B54FF4FA661E609C4AFF
:10F988009C4B9D4F1A609D4A9D4B1A609D4B42F2BD
:10F9980010721A609C4B64241C6001233B70FAF7B8
:10F9A80036F99A4B00251D70F8F780FAF6F7EEFB4A
:10F9B800F6F7F8FBF6F706FCF7F7E0F92046F7F755
:10F9C8005DFEF7F701FA2046F7F758FEF8F754FA04
:10F9D800F8F78AF8F7F760FE2046F7F74FFEFAF7D0
:10F9E800C1FA2046F7F74AFE4FF4FA50F7F7B2FD8E
:10F9F8002046F7F743FEF7F719F92046F7F73EFEDA
:10FA08002846F7F71DFF8248F7F738FEF4F77AFC27
:10FA18002046F7F733FE7F4B03F1100229468DE8A5
:10FA2800240028465A681B68F4F772FE3046F7F738
:10FA380025FE2846F5F7ECF84FF6FF70F5F7FEF8C7
:10FA480003213220744A2B46F5F710FA9620734AA0
:10FA58008C212B46F5F70AFA9620A021704A2B46EE
:10FA6800F5F704FA6F4A2B469620B421F5F7FEF90C
:10FA7800FAF784F85021DC20FAF753F83046F7F704
:10FA8800FDFD694A2B46DC212846F5F7EFF9674862
:10FA9800F7F7F4FD2046F7F7F1FDF6F78FFE20465D
:10FAA800F7F7ECFD9FED620AF7F7E2FE2046F7F75D
:10FAB800E5FDF7F70BFEF5F7A1FC2046F7F7DEFDAD
:10FAC80014200146F6F7EAFB2846F6F73DFC2046E7
:10FAD800F7F7D4FDF6F7BCFD2046F7F7CFFDF7F7AB
:10FAE80045F92046F7F7CAFDF6F7B8FE00B13D70B4
:10FAF800F6F7C0FE08B1F9F7EBFF4E4B00241C7077
:10FB0800F2F756F8F5F730FC08B94B4802E04B4BD2
:10FB18004B481C70F2F763F8F6F79AF8F8F761FEAD
:10FB2800F8F794FEF8F7E1FBF8F7C8FAF9F7F3FFEE
:10FB3800FAF796F9FAF742F8424B434D434C8028BE
:10FB480014BF4FF480504FF4806018802C4B1A6813
:10FB5800284B1B68D21A2B4B1B6892FBF3F23C4BC9
:10FB68002E461A80F6F79CFE2B7833B1012B02D172
:10FB7800F7F7E8FF01E0F8F70DF800233370F8F71E
:10FB880063F9F3F741FEF9F7EDFE228812B2012A74
:10FB980013D130484FF40051FDF76BF92E4B1B7809
:10FBA8000BB9F8F719FFF8F7E1F82A484FF40051B4
:10FBB8000022FDF75EF900232380274B5B7843B1D1
:10FBC800F9F7DCFFF0209621F9F7ABFF2348F7F7A8
:10FBD8004BFB234F3846FBF7B0FC0028C2D03B78DC
:10FBE800112BBFD1F9F7ECFEBCE700BF283C002081
:10FBF800E0673500583C0020280E002080C3C9016A
:10FC0800744200204C420020083C0020D4430020CD
:10FC180000127A00F87C0108119D05082B9D050843
:10FC2800389D0508449D05084D9D0508002D3101A6
:10FC38000000FA44383C0020100F0020F03B002060
:10FC4800FC100020543C002050420020BC0C002036
:10FC58008045002000080240D80C002040420F00D8
:10FC6800F13B002010B4314C0180B1F5807F446035
:10FC78008270C37052D00DD9B1F5806F39D017D9C1
:10FC8800B1F5006F2ED0B1F5805F24D0FF2040B2CF
:10FC980010BC704720293AD014D9402930D0802987
:10FCA800F4D123494FF02012C26081600020EEE7B2
:10FCB800B1F5007FEAD11F4B4FF00811C160836096
:10FCC8000020E4E71029E1D11B494FF00122C2606E
:10FCD80081600020DBE7194B4FF00111C1608360A0
:10FCE8000020D4E7164A4FF00213C3608260002058
:10FCF800CDE714494FF00412C26081600020C6E7C6
:10FD0800114B4FF04011C16083600020BFE70F4ADC
:10FD18004FF08013C36082600020B8E70C4A4FF0B0
:10FD28001013C36082600020B1E700BF209C040864
:10FD38005E8C05082E8C05081E8E0508208C05088B
:10FD4800228C0508268C05089E8C05081E8D050842
:10FD58003E8C05082DE9F00FB2B02E9030932E9B03
:10FD680000882E9C5B68309FA4682D90451E03EB8D
:10FD78004506BF08209328942C952F911F921E9614
:10FD8800319700F03A814FEA900A4FEACA0B00F027
:10FD980003002F99299003F1080504EB0B00CDF817
:10FDA80084A0CDF8A8B019951A921B9718961791A8
:10FDB8002B90179A189E13883380B2F802C0A6F8C1
:10FDC80002C09488B480D788F78008361896219F97
:10FDD800199E0832179256F8041C56F8082C4FF052
:10FDE800000A4FF0000B002F00F06982CDE904AB48
:10FDF800CDE906ABCDE902ABCDE900AB289CBC460A
:10FE0800029BDDF80C902568C2FBC5394FF000084D
:10FE180048EA030ACB46CDE902AB049BDDF814B0EF
:10FE2800C1FBC53BCDF824B0CDF82080DDE908AB97
:10FE3800C1EA02004AEA030ACDE904AB069BDDF8F1
:10FE48001CB03268C0FBD53BCDF82CB0CDF828806B
:10FE5800DDE90AABC2EA01074AEA030ACDE906ABC3
:10FE68009DE80108C7FBD50BCDF834B0CDF830803C
:10FE7800DDE90CAB4AEA000A63680298CDE900ABF9
:10FE88000834DDF80CB0C1FBC30BCDF83CB0CDF89D
:10FE98003880DDE90EAB4AEA000ACDE902AB7168A9
:10FEA8000498DDF814B0C2FBC30BCDF844B0CDF80C
:10FEB8004080DDE910AB4AEA000ACDE904AB0698B8
:10FEC800DDF81CB0C7FBD30BCDF84CB0CDF848809B
:10FED800DDE912ABC1EA02054AEA000ACDE906AB40
:10FEE8009DE80108C5FBD30BCDF854B0CDF8508080
:10FEF800DDE914AB08364AEA000ABCF1010CCDE989
:10FF080000AB7FF47DAF2A9D19982B9B2E18299F53
:10FF1800002F35D01868039F029BC2FBC03700240E
:10FF28001D971C94DDE91C4544EA0304CDE902450C
:10FF3800049B059DC1FBC035002723952297DDE969
:10FF4800224544EA0304CDE90445C1EA0203079DBA
:10FF5800069AC3FBD02525952497DDE9244544EA74
:10FF680002043368C3EA0101CDE9064553465D46FC
:10FF7800C1FBD03527952697DDE926AB4AEA030A67
:10FF8800069A029C0499039D079FD30B059AE60BDA
:10FF9800C90B46EA454043EA474441EA424604F36E
:10FFA8000F0500F30F0C199BCCEA054706F30F0069
:10FFB8001A9D1B9E2F604FEADA3A08334AEA4B4BE8
:10FFC8000BF30F04C0EA04426A600835711E1993E6
:10FFD8001A951B917FF4EDAE319A2F9E1E991F9BA7
:10FFE800DDF880B0D00037180D182F970BEB000AFA
:08FFF8001F181E951F97CDF89C
:020000040801F1
:1000000080A0DDF8C0C01CF0030BCDF820B000F0DC
:1000100086802D9BDDF8BC80CDF808B05808DDF84F
:1000200080A0DDF8A0B00690CDF81080049A1E9E46
:1000300032F8025B069826F8025B0492BAF8027066
:10004000BBF80230BAF80020BBF800401E9617FB40
:1000500003F112FB04F6451E4FEAE17711EB0608A7
:100060002B4605F0010047EBE6790AF104020BF19B
:100070000401002D3BD0A8B1B2F800C0BBF8047059
:10008000548848881CFB07F518EB050749EBE57613
:1000900014FB00F917EB090846EBE9790432043147
:1000A000013B24D00F88B2F800C0568848888C885D
:1000B00095881CFB07FC18EB0C0816FB00F7D08892
:1000C000CE8849EBEC7C15FB04F518EB07084CEBEC
:1000D000E77918EB050710FB06FC49EBE57417EB15
:1000E0000C0844EBEC7908320831023BDAD11F9A54
:1000F00002994FEAD83545EA494404F30F0322F840
:10010000023B4F1E0AF1020A1F9202978ED1DDF8C0
:1001100080A0DDF820B00AEB4B0ACDF880A02C9E21
:100120002E98B50840683FD0209F47EA000212F0A1
:10013000030F00F1080307F1080214BF0021012199
:100140009F4298BF904294BF00260126314277D04B
:1001500097E84200016001216C1EA942466004EA52
:10016000010419D044B192E81200196002215C60C8
:1001700008320833A9420FD092E850001C605E603C
:10018000966802F1080BD2689E600231DA60103383
:10019000A9420BF10802EFD1DDF880C0ED000CEBB5
:1001A000050B4019CDF880B02C9C14F0030343D00C
:1001B0005A085400002A00F08E80209D40EA05076E
:1001C00017F0030F209F14BF00250125011D3E1DC0
:1001D000012B94BF002505F001058F4298BFB04266
:1001E00094BF002101210D4275D039689200BF18DB
:1001F000A342016020971044C4EB03011CD0209B54
:10020000013933F8024B0A4620F8024B01F0010194
:1002100092B129B133F8021B013A20F8021B0BD02E
:100220001C46014634F802CB21F802CB5D88A31CA2
:100230004580881C023AF3D132B0BDE8F00F704718
:10024000B7F800C0A0F800C07C884480BE888680D3
:10025000691EFE880C46BA4601F00101C680002CDA
:100260009AD089B1B2F800B0A3F800B05188598093
:10027000B2F804C0A3F804C0B2F806B00832A3F87C
:1002800006B00833013C87D016881E8051885980FB
:10029000B2F804B0A3F804B0B2F806C0A3F806C0E0
:1002A00016891E8103F1080B5189ABF8021093895E
:1002B000ABF80430D6891032023C0BF10803ABF8DE
:1002C0000660E1D168E7289BCDE904ABCDE906AB38
:1002D000CDE902AB1FE6194691E700BF2DE9F00F0B
:1002E0009CB006780F900F9C40880F9DA4686D68A5
:1002F0001990B3FBF6FA471E4FEA5A0804EB470978
:10030000AAEB480340460A940D951A97CDF86C80E5
:100310000C911492CDF82C901193002800F0B58127
:100320001746199A199CCDF848809108CA00159172
:1003300004F00303A91817921693109718917600EA
:1003400075084FEA450C002D00F03B840B9FDDF84B
:10035000308047EA080010F0030F14BF002101218C
:1003600008F10404381D012E94BF002101F00101A1
:10037000804598BFA74294BF4FF000094FF0010994
:1003800011EA090F00F01D84BB46D8F800200123B4
:100390006F1EAB42CBF8002007EA03072146024656
:1003A00014D237B1246802230431021DAB42046029
:1003B0000CD20C46104654F8047B40F8047B496884
:1003C00002335160211D021DAB42F2D3DDF83080B3
:1003D000DDF82CB04FEA4C05664508EB05020BEB47
:1003E0000503CCEB06001DD0013832F802CB0146E4
:1003F00023F802CB00F00100A1B128B132F8029B32
:10040000013923F8029B0DD014461F4634F8029B95
:1004100027F8029BB2F802A0A21CA3F802A0BB1C02
:100420000239F1D10C9ADDF83CC00B989CF80080A1
:10043000710053180A9E0C93159BCDF84C804518FB
:1004400006EB48020B950E92002B00F0B1830024BE
:100450000025CDE90445CDE9024507930D991346E2
:100460000A9AB3F804A0B2F806B0CDF804A0B3F825
:1004700006A00E881588CDF820B0CDF824A0DDE9BF
:1004800002AB15FB06F51AEB050A4BEBE57BCDE954
:1004900002AB1F884888B2F802C0B3F80290B2F8E5
:1004A00004808C88CDF81880DDE904AB16FB07F6D4
:1004B0001AEB060A4BEBE67BDDE902671CFB00F555
:1004C000761910FB09F047EBE5771AEB000A4BEBC6
:1004D000E07BCDE902ABDDF818B0DDF804C0B1F87F
:1004E0000680099D1BFB04F016EB000A47EBE07B3E
:1004F000DDE9026714FB0CF4361947EBE477089C3E
:1005000014FB08F00831083208331AEB000418FB1A
:1005100005F84BEBE075079816EB080A47EBE87B0C
:100520000138CDE90245CDE904AB079099D1179E7A
:100530000E9C0A9B1899A7199A190E97169F002FBF
:1005400073D00E9B31F8020B32F8024B33F8026B7A
:10055000DDE90289DDE904AB14FB00F47D1E10FB2C
:1005600006F618EB040849EBE4791AEB060A4BEBA4
:10057000E67B2F4605F00100CDE90289CDE904AB09
:10058000002D52D0002873D031F8024B32F8020B04
:1005900033F8025B10FB04F614FB05F0DDE90245BD
:1005A000DDE90489A41945EBE67518EB000849EB71
:1005B000E079013FCDE90245CDE9048935D0C24655
:1005C000CB46DDE902890D461446049721462846AC
:1005D0001A4630F8026B31F8027B32F802CB6D8894
:1005E00064885B8817FB06F718EB070816FB0CF608
:1005F00049EBE7791AEB060714FB05FA4BEBE67BB0
:1006000015FB03FC8C1C931C0499851C18EB0A0831
:1006100049EBEA7917EB0C0A4BEBEC7B8A1ECDE930
:1006200002890492D2D1CDE904AB029D03990498CA
:10063000DDF828A0059BEA0B109D42EA414812997B
:1006400008F30F09A5F80090DDF84C90C70B0AEBF2
:100650008908281D4A1E47EA4346CDF8288006F33C
:100660000F0410906C8012920AD00F9C267866E6D8
:10067000DDE904AB0D4614460497DDE90289A5E7E0
:10068000149F1B9B07EB83061496119F002F00F00D
:10069000A681DDF864B0DDF86480DDF834C04FEA8F
:1006A0009B09CDF81C904FEAC90908F0030A0CEB2E
:1006B000090BCDF82090CDF810A0CDF824B0DDF8CE
:1006C0003CC09CF8006075084FEA450C002D00F016
:1006D0007E820C990B980B9F40EA010414F0030FE3
:1006E00014BF002201220C1D0430012E94BF0022F1
:1006F00002F00102814298BFA74294BF0023012368
:100700001A4200F06482BA4601230F68691EAB42A8
:10071000CAF80070024601EA0307214614D237B135
:1007200027680223211D021DAB4207600CD20C4634
:10073000104654F8047B40F8047B4968023351604A
:10074000211D021DAB42F2D3DDF83090DDF82C8084
:100750004FEA4C05664509EB050208EB0503CCEBB7
:1007600006001DD0013832F802BB014623F802BB57
:1007700000F00100A1B128B132F8025B013923F881
:10078000025B0DD014461F4634F802AB27F802ABCB
:10079000B2F802C0A21CA3F802C0BB1C0239F1D1FE
:1007A000DDF82CA0DDF830B0079876000AEB060CD7
:1007B0000BEB0608CDF82CC0CDF83080002800F0F7
:1007C000F0810A9ADDF834805788B2F800A0DDF88D
:1007D00028909488B9F80690B8F8062084460D98B9
:1007E00041880588B8F8040017FB01F61AFB05F3E9
:1007F000B3461BEB03014FEAE67714FB00F047EB2F
:10080000E3750F180A9B19FB02F145EBE0750CF13B
:10081000FF3617EB010AB14606F0010008F10802A5
:1008200003F1080345EBE17B002E00F0858048B31F
:10083000DDF834C01E88BCF8084058885188978875
:100840009D88B2F80680B3F806C016FB04F41AEBD4
:10085000040A10FB01F14BEBE4761AEB010415FBE3
:1008600007FB46EBE17014EB0B011CFB08F640EBB9
:10087000EB740832083311EB060A44EBE67BB9F15E
:10088000010959D0CDE902ABCB46B3F80080B3F8EB
:1008900008901688CDF8389018FB06F6DDE9028935
:1008A0005D88548898889188B2F806C0DF88B2F8CD
:1008B00008A015FB04F418EB060810FB01F149EB46
:1008C000E67918EB040817FB0CF749EBE47918EB11
:1008D000010849EBE17918EB070849EBE779CDE925
:1008E0000289DDF838905D89548998899189B2F838
:1008F0000EC0DE8919FB0AF7DDE9028915FB04F455
:1009000018EB070810FB01F149EBE77918EB040835
:1009100049EBE47916FB0CF618EB010449EBE175A1
:1009200010321033A01945EBE671BBF1020BCDE993
:100930000201AAD182468B460DF1200898E81600E4
:100940006318049D9DB332F802CB33F8026B16FB9B
:100950000CF4013D1AEB040A294605F001004BEBAB
:10096000E47B25B358B132F8028B33F8020B10FB4D
:1009700008F71AEB070A4BEBE77B691E17D0144602
:10098000184634F8025B30F8027B52885B8817FB0C
:1009900005F81AEB08064BEBE87713FB02FBA21CE9
:1009A000831C16EB0B0A47EBEB7B0239E7D10F9D5B
:1009B000DDF8508095F800C00A9A119E4FEADA33AC
:1009C00043EA4B4404F30F0028F8020B02EB4C07F8
:1009D000711E0A97CDF8508011917FF470AE1A9E67
:1009E0000F9CB508A06842D00A9F47EA000616F09F
:1009F000030F07F1080200F1080314BF00210121D1
:100A00009F4298BF904294BF4FF0000A4FF0010AF6
:100A100011EA0A0F7FD097E84200016001216C1EA5
:100A2000A942466004EA010419D044B192E81200D8
:100A3000196002215C6008320833A9420FD092E8A5
:100A400050001C605E60966802F10804D2689E60E7
:100A50000231DA601033A94204F10802EFD1DDF867
:100A600028A0ED000AEB05094019CDF82890DDF823
:100A700068A01AF003034AD05A085400002A00F074
:100A8000A480DDF828B040EA0B0515F0030F14BF71
:100A9000002501250BF10406011D012B94BF002543
:100AA00005F001058B4598BFB04294BF4FF0000C94
:100AB0004FF0010C15EA0C0F00F08780DBF80010F6
:100AC00092009344A3420160CDF828B01044C4EBD7
:100AD00003011CD00A9B013933F8024B0A4620F867
:100AE000024B01F0010192B129B133F8021B013A26
:100AF00020F8021B0BD01C46014634F802CB21F82B
:100B000002CB5D88A31C4580881C023AF3D11CB03F
:100B1000BDE8F00F7047B7F80090A0F800907C880F
:100B20004480BE888680691EFE880C46B84601F067
:100B30000101C680002C92D091B111881980B2F8C1
:100B400002C0A3F802C0B2F804A0A3F804A0B2F84F
:100B500006900832A3F806900833013C3FF47FAFBB
:100B600011881980B2F802C0A3F802C0B2F804904C
:100B7000A3F80490B2F806A0A3F806A016891E8177
:100B800003F1080C5189ACF802109389ACF80430D9
:100B9000D6891032023C0CF10803ACF80660DFD1B4
:100BA0005DE70D9A0A9B4FF0000A4FF0000BC8E674
:100BB00000260027CDE904670A9A0D99CDE902675E
:100BC000BCE430460B9B0C9A0EE4194682E7304693
:100BD0000B9B0C9AC6E500BF00B553EC102B42F2FC
:100BE000FB1223F00043C3F6E972934285B026DD81
:100BF0004FF6FF72C7F6EF7293420BDD51EC100B0C
:100C000002460B46FDF7BEFE02460B4643EC102B98
:100C100005B000BD684600F0BFFB00F003000128EE
:100C20009DED000B9DED021B1AD0022810D0F8B9E3
:100C300000F0D2FE53EC102B10461946E4E79FED6E
:100C4000101B00F0C9FE53EC102B10461946DBE7D1
:100C500000F0C2FE53EC102B104603F10041D3E725
:100C600001F0F6FB53EC102B104603F10041CBE7EB
:100C7000012001F0EDFB53EC102B10461946C3E7A1
:100C800000000000000000002DE9F04759EC108B37
:100C9000C9F30A56A6F57E74073C132C4D46CA4686
:100CA000474626DC002C4FDB4FF6FF76C0F20F06DE
:100CB00046FA04F606EA090555EA080517D044A3E2
:100CC000D3E9002351EC100BFDF75EFE0022002358
:100CD000FEF79CFA00284AD0B9F1000F6EDB2AEA31
:100CE000060A4FF000085346424643EC102BBDE87D
:100CF000F087332C0CDDB4F5806FF8D151EC100B7C
:100D00003A460B46FDF740FE41EC100BBDE8F0877C
:100D1000A6F58265033D4FF0FF3323FA05F515EA8A
:100D2000080FE4D02AA3D3E9002351EC100BFDF700
:100D30002BFE00220023FEF769FAC0B1B9F1000FC3
:100D40001CDB28EA050813E021A3D3E9002351ECBA
:100D5000100BFDF719FE00220023FEF757FA38B1F9
:100D6000B9F1000F1BDB4FF00008C24600E0CA4695
:100D70005346424643EC102BBDE8F087142C09D0B3
:100D8000C6F5866303334FF0010808FA03F818EB41
:100D90000708D6D30AF1010A28EA0508E8E729F08E
:100DA000004848EA07084FF0000AD045CBF6F07A31
:100DB00008BFCA4618BF4FF00008D9E74FF48013A8
:100DC00043FA04F409EB040A89E700BFAFF300809B
:100DD0009C7500883CE4377E00B553EC102B42F242
:100DE000FB1223F00043C3F6E972934285B027DD7E
:100DF0004FF6FF72C7F6EF7293420BDD51EC100B0A
:100E000002460B46FDF7BEFD02460B4643EC102B97
:100E100005B000BD684600F0BFFA00F003000128ED
:100E20009DED000B9DED021B1DD0022812D008BBCA
:100E3000012001F00DFB53EC102B10461946E3E79F
:100E400000209FED111B01F003FB53EC102B10460B
:100E50001946D9E7012001F0FBFA53EC102B10469C
:100E600003F10041D0E700F0B7FD53EC102B104622
:100E70001946C9E700F0B0FD53EC102B104603F102
:100E80000041C1E7AFF30080000000000000000057
:100E900000F0E6B8D0B52DED048BB0EE408AF0EE50
:100EA000608A3C4C8AB000F0DBF994F90030B0EE77
:100EB000409AF0EE609A013335D0B0EE480AF0EE79
:100EC000680A01F04FFD00282DD051EC180B0022CC
:100ED0000023FEF787F930B32F4B247801930023CA
:100EE00008938DED028B8DED048B002C23D0002711
:100EF0000026CFF6F07751EC180B00220023CDE945
:100F00000667FEF75BF9002825D002239C42009378
:100F100036D0684601F05EFD002831D0089B002BDA
:100F200027D19DED069BB0EE490AF0EE690A0AB0A2
:100F3000BDEC048BD0BD4FF6FF774FF06046CCF28E
:100F4000EF7751EC180B00220023CDE90667FEF77E
:100F500035F90028D9D10123022C009315D0684619
:100F600001F038FD88B10D4801F036FD8DED060B1E
:100F7000D4E701F0EFFF089B9DED069B0360D2E7ED
:100F800001F0E8FF22230360C8E701F0E3FF21231B
:100F90000360E8E7E4020020C09F050820A20508DE
:100FA00010B52DED048BB0EE408AF0EE608A294C2E
:100FB0008AB000F02DFC94F90030B0EE409AF0EECB
:100FC000609A01332BD0B0EE480AF0EE680A01F0C7
:100FD000C9FC20B351EC180B00220023FEF7F8F8EF
:100FE000E8B11D4B2478019301230093002308935B
:100FF0008DED048B8DED028BCCB1002000210246DB
:101000000B46FDF79DFF022CCDE9060115D101F03D
:10101000A1FF21230360089BABB99DED069BB0EEB9
:10102000490AF0EE690A0AB0BDEC048B10BD00223B
:10103000002343EC172B8DED067B684601F0CAFCBC
:101040000028E8D1E3E701F085FF089B9DED069BB2
:101050000360E4E7E4020020C89F050800000000E8
:10106000F8B5B0EE407AF0EE607A53EC112B5442B2
:1010700010461D46002125F00047044353EC102B79
:1010800047EAD474C7F6F0718C4216463DD85442F4
:10109000344323F0004242EAD4748C4235D805F13F
:1010A000404101F5801101434FD0AC1704F0020418
:1010B000164344EAD37435D0384341D00021C7F6F3
:1010C000F0718F424FD00021C7F6F0718A4237D0BD
:1010D000D21B12153C2A42DC002D7DDB53EC112B78
:1010E00051EC170BFDF72CFF41EC100B01F030FC1D
:1010F00001F06AFA51EC100B012C68D0022C57D089
:10110000002C48D141EC170B07E051EC170B53ECC6
:10111000112BFDF739FC41EC170BB0EE470AF0EE4E
:10112000670AF8BD032CC7D801A151F824F000BF0D
:101130001B1101081B110108591101085311010865
:10114000002B25DB9FED307BE7E7BDE8F84001F0A1
:101150003BBA9FED2F7BE0E79FED2F7BDDE72AA1D8
:10116000D1E90001C8E7BA423CD0032CABD801A1B9
:1011700051F824F08B11010885110108591101085B
:10118000531101089FED267BC7E79FED277BC4E73E
:101190009FED277BC1E730A3D3E90023FDF7F2FBE6
:1011A0001DA3D3E90023FDF7EDFB41EC170BB4E7DA
:1011B00029A3D3E90023FDF7E5FB02460B4616A160
:1011C000D1E90001FDF7DEFB41EC170BA5E701F1CA
:1011D000004141EC170BA0E73C32BFF67FAF002087
:1011E000002189E7032CABD8DFE804F00B080502E7
:1011F0009FED117B91E79FED127B8EE79FED127BB8
:101200008BE79FED137B88E7182D4454FB21F93FB2
:10121000182D4454FB2109C0182D4454FB210940CA
:10122000000000000000008000000000000000003E
:10123000182D4454FB21F9BFD221337F7CD902C041
:10124000D221337F7CD90240182D4454FB21E9BFC1
:10125000182D4454FB21E93F075C143326A6A13C1A
:101260002DE9F84F55EC104BB5F5801F2F4622DACB
:1012700025F00043234368D0002D2046294670DB2B
:1012800000230022C4F25033FDF730FD4FF6FF7308
:101290000F46C7F6EF739F4204460D466FF03502C6
:1012A00010DD2046294622462B46FDF76DFB41EC1A
:1012B000100BBDE8F88F4FF6FF73C7F6EF730022EF
:1012C0009F42EEDC3B15A3F57E73073B9A18D60FC1
:1012D000901927F07F47C6F57E76FDF7A1FC07360B
:1012E00027F4700747EA065545EC104B80468946BF
:1012F00001F00AFC4046494621A3D3E9002355ECFE
:10130000104BFDF7F3FC20A3D3E9002382468B4664
:1013100040464946FDF7EAFC1DA3D3E900230646F3
:101320000F4620462946FDF7E1FC02460B463046B3
:101330003946FDF729FB02460B4650465946FDF754
:1013400023FB41EC100BBDE8F88F00210020CCF20C
:10135000503100220023FDF7F3FD41EC100BBDE8F6
:10136000F88F22462B46FDF70DFB00220023FDF7E8
:10137000E7FD41EC100BBDE8F88F00BFAFF3008034
:1013800000609F501344D33F362BF111F3FE593DBB
:101390000EE526157BCBDB3F2DE9F04F53EC102BF0
:1013A00042F2FB1223F00044C3F6E97294428FB07C
:1013B0001E46074640F3AA804DF67B13C4F2020393
:1013C0009C422ADC002E51EC100BDDA3D3E9002354
:1013D00040F3CA81FDF7D6FA42F2FB13C3F6F97364
:1013E0009C428046894600F0AA80D7A3D3E9002317
:1013F000FDF7C8FA0D4604462B462246C7E90045CC
:1014000040464946FDF7BEFACFA3D3E90023FDF7D6
:10141000B9FA0125C7E9020181E042F2FB13C4F2E7
:1014200039139C4240F3AA804FF6FF73C7F6EF735F
:101430009C4278DC4FEA245AAAF5826AAAF1060A8D
:1014400051EC100BA4EB0A5319461D460446FDF758
:10145000E7FEFDF7E5FB8046894642464B462046BF
:101460002946CDE90889FDF78DFA00230022C4F250
:101470007013FDF73BFC0D460446FDF7D1FEFDF76A
:10148000CFFB804689462046294642464B46CDE959
:101490000A89FDF777FA00230022C4F27013FDF7E2
:1014A00025FC002204460D460023CDE90C45FDF73E
:1014B00085FE002800F07B8140464946002200233B
:1014C000FDF77CFE03240AAD013C40B175E9020141
:1014D00000220023FDF772FE013C0028F6D12346CE
:1014E000022400949E4C08A839465246019400F00C
:1014F000ABFB002E054612DA7A68FB6802F1004267
:1015000003F100437A60FB60454208E000220023BB
:1015100043EC172B87ED000B80ED027B002528465E
:101520000FB0BDE8F08F51EC100B02460B46FDF7F3
:1015300029FA0025C7E90201C7E90001EFE77AA30C
:10154000D3E90023FDF71EFA79A3D3E900238046EF
:101550008946FDF717FA0D4604462B462246C7E991
:10156000004540464946FDF70DFA71A3D3E9002333
:10157000FDF708FA0125C7E90201D0E701F0E8F913
:1015800059EC108B6CA3D3E9002340464946FDF784
:10159000ADFB00230022C3F6E073FDF7F5F9FDF77C
:1015A0003FFE0546FDF73CFB65A3D3E90023CDE9EB
:1015B0000201FDF79BFB02460B4640464946FDF7FC
:1015C000E1F961A3D3E9002382468B46DDE90201FC
:1015D000FDF78CFB1F2DCDE90401504659462BDC4D
:1015E0006A1E604B53F82230A34225D0DDE9042364
:1015F000FDF7C8F902460B46C7E900238146884635
:101600004A46434650465946FDF7BCF9DDE90423F6
:10161000FDF7B8F9002E02460B46C7E90223BFF6D4
:101620007EAF08F1004301F10041C7F800907B60F4
:10163000B860F9606D4272E7DDE90423FDF7A2F9B5
:1016400088462415C8F30A53E31A102B8146C7E9CC
:101650000001D5DD34A3D3E90023DDE90201FDF764
:1016600045FB8046894642464B4650465946FDF763
:1016700089F9CDE90601DDE9062350465946FDF713
:1016800081F942464B46FDF77DF929A3D3E90023B2
:1016900080468946DDE90201FDF728FB42464B46BC
:1016A000FDF770F9CDE90401DDE90423DDE9060168
:1016B000FDF768F98846C8F30A53E41A312C8146CD
:1016C000C7E9000140F3958021A3D3E90023DDE9B8
:1016D0000201FDF70BFB8046894642464B46DDE999
:1016E0000601FDF74FF982468B4652465B46DDE91F
:1016F0000601FDF747F942464B46FDF743F916A3AD
:10170000D3E9002380468946DDE90201FDF7EEFAC0
:1017100042464B46FDF736F9CDE90401504659469D
:1017200064E700BFAFF300800000601A61B4D03DF1
:101730007370032E8A19A33B83C8C96D305FE43FE1
:1017400000004054FB21F93F3163621A61B4D03D7F
:101750000000002E8A19A33BC14920259A837B39BA
:1017600050A00508D09F0508FDF70EF942F2FB13C3
:10177000C3F6F9739C42804689461AD01EA3D3E96A
:101780000023FDF701F90D4604462B462246C7E922
:10179000004540464946FDF7F5F817A3D3E9002375
:1017A000FDF7F2F84FF0FF35C7E90201B7E6032471
:1017B00095E613A3D3E90023FDF7E6F812A3D3E9D6
:1017C000002380468946FDF7DFF80D4604462B4688
:1017D0002246C7E9004540464946FDF7D3F80AA32B
:1017E000D3E90023FDF7D0F84FF0FF35C7E9020138
:1017F00095E6DDE906AB03E73163621A61B4D03DDB
:101800000000601A61B4D03D7370032E8A19A33BA7
:101810002DE9F84353EC102B00242546C7F6F0744D
:10182000C7F6F0751C40AC422DED028BB0EE408A3D
:10183000F0EE608A1946104600F0AB80002B7FDD89
:101840001A1500F08980A2F57E7721F07F4323F4FA
:101850007003073FD20743F4801366D5C20F4FF0E1
:10186000000C02EB43037F104200654616204FF444
:1018700000116C18D60F9C424FEA420202DC651838
:101880001B1B8C444908013806EB4303F1D1202689
:1018900080464FF0004107E043D0D40F4908520082
:1018A000013E04EB43031BD0AB4208EB0104F3DD24
:1018B00004F00049B9F1004F04EB01082BD0A94610
:1018C0009442C5EB0303C4EB020288BF013B4018FE
:1018D000D40F49085200013E4D4604EB4303E3D1C7
:1018E0001A4327D146084FEA6C0101F17E511CF0E2
:1018F000010F01F5C00118BF46F0004601EB075388
:10190000324643EC182BB0EE480AF0EE680ABDEC04
:10191000028BBDE8F883B8F1000FD0DB05F10109B7
:10192000CEE79442C4D91D46B7E7C20F02EB43038A
:10193000400093E7431C39D000F001031818D1E7A9
:1019400023F000441443DED0002B36D11A46C10ADE
:10195000153A40050029FAD011F4801329D1490025
:101960000133CC02FBD5C3F10105C3F1200420FAF9
:1019700004F4521921439840A2F57E7721F07F4369
:1019800023F47003073FD20743F480133FF566AF9B
:10199000CBE751EC100BFDF7A9F902460B4651ECD1
:1019A000180BFCF7F1FF41EC180BACE70CF1010C44
:1019B00099E7202401250023D9E751EC100B0B46B1
:1019C000FCF7E0FF02460B46FDF7BAFA41EC180BB4
:1019D00099E700BF000000002DE9F04F5BEC10AB71
:1019E0002DED028BB0EE418AF0EE618A2BF00044BF
:1019F000B4F1795F85B071DA50465946FDF710FCB5
:101A0000002800F0FD8052465B4650465946FDF7DF
:101A10006DF981A3D3E9002306460F46FDF766F969
:101A20007FA3D3E90023FCF7AFFF32463B46FDF727
:101A30005DF97DA3D3E90023FCF7A4FF32463B46C2
:101A4000FDF754F97AA3D3E90023FCF79DFF324652
:101A50003B46FDF74BF978A3D3E90023FCF792FF4F
:101A600032463B46FDF742F975A3D3E90023FCF764
:101A70008BFF32463B46FDF739F980468946002305
:101A80000022C3F6E07330463946FDF72FF942468F
:101A9000CDE900014B4630463946FDF727F953ECB6
:101AA000182B04460D4650465946FDF71FF90246CD
:101AB0000B4620462946FCF765FF02460B46DDE94A
:101AC0000001FCF75FFF0B4600210246C3F6F071F0
:101AD0000020FCF757FF41EC100B83E052465B46B9
:101AE00050465946FDF702F94BA3D3E900230646B9
:101AF0000F46FDF7FBF84AA3D3E90023FCF744FFA8
:101B000032463B46FDF7F2F847A3D3E90023FCF742
:101B100039FF32463B46FDF7E9F845A3D3E90023F8
:101B2000FCF732FF32463B46FDF7E0F842A3D3E92B
:101B30000023FCF727FF32463B46FDF7D7F840A3CA
:101B4000D3E90023FCF720FF3B463246FDF7CEF8F1
:101B500043F23233C3F6D3739C42804689468EDD0E
:101B60000023C3F6E9739C4241DC0021A4F5001375
:101B700000220020C3F6F07114461D46FCF702FF58
:101B8000CDE9020100230022C3F6E0733046394656
:101B9000FDF7ACF822462B46FCF7F4FE4246CDE9B1
:101BA00000014B4630463946FDF7A0F853EC182BA0
:101BB00004460D4650465946FDF798F802460B4636
:101BC00020462946FCF7DEFE02460B46DDE9000111
:101BD000FCF7D8FE02460B46DDE90201FCF7D2FE17
:101BE00041EC100B05B0BDEC028BBDE8F08F9FED12
:101BF000067B00258DED027B0024C3F6D275C1E77C
